:020000040800F2
:1000000000060020E10100086D0E0008ED0D00085B
:10001000450E0008ED0D0008190E0008E301000868
:10002000E3010008E3010008E301000841210008A2
:10003000E3010008E3010008E3010008E301000810
:10004000E3010008E3010008E3010008E301000800
:10005000E3010008E3010008093200083532000816
:10006000613200088D320008B9320008E30100084F
:10007000E3010008E3010008E3010008E3010008D0
:10008000E3010008E3010008E3010008E3010008C0
:10009000E3010008E3010008E3010008E53200087D
:1000A000E3010008E3010008E3010008E3010008A0
:1000B0007D300008E3010008E3010008E3010008C7
:1000C000E3010008E3010008E3010008E301000880
:1000D000E3010008E3010008E3010008E301000870
:1000E0004D330008E3010008E3010008E3010008C4
:1000F000E3010008E3010008E3010008E301000850
:10010000E3010008E3010008E3010008E30100083F
:10011000E3010008E3010008E3010008E30100082F
:10012000E3010008E3010008E3010008E30100081F
:10013000E3010008E3010008E3010008E30100080F
:10014000E3010008E3010008E30100087928000842
:10015000E3010008E3010008E3010008E3010008EF
:10016000E3010008E3010008E3010008E3010008DF
:10017000E3010008E3010008E3010008E3010008CF
:10018000E3010008E3010008E3010008E3010008BF
:10019000E3010008E3010008E3010008E3010008AF
:1001A000E3010008E3010008E3010008E30100089F
:1001B000E3010008E3010008E3010008E30100088F
:1001C000E3010008E3010008E3010008E30100087F
:1001D000E3010008E3010008E3010008E30100086F
:1001E00002E000F000F8FEE772B63A4880F30888B3
:1001F000394880F3098839484EF60851CEF200019B
:10020000086040F20000CCF200004EF63471CEF2ED
:1002100000010860BFF34F8FBFF36F8F40F2000003
:10022000C0F2F0004EF68851CEF200010860BFF334
:100230004F8FBFF36F8F4FF00000E1EE100A4EF6C4
:100240003C71CEF200010860062080F31488BFF3F1
:100250006F8F01F0F5FF01F0D1FF02F073FE4FF058
:1002600055301F491B4A91423CBF41F8040BFAE745
:100270001C49194A91423CBF41F8040BFAE71A495C
:100280001A4A1B4B9A423EBF51F8040B42F8040B2A
:10029000F8E700201749184A91423CBF41F8040B87
:1002A000FAE701F0AFFF02F0A1FE144C144DAC428E
:1002B00003DA54F8041B8847F9E700F041F8114CC1
:1002C000114DAC4203DA54F8041B8847F9E701F0FA
:1002D00097BF000000060020002200200000000858
:1002E00000000020000600207837000800220020CF
:1002F0004022002040220020A82D0020E00100081C
:10030000E0010008E0010008E00100082DE9F04FDD
:100310002DED108AC1F80CD0C3689D46BDEC108A43
:10032000BDE8F08F002383F311882846A047002002
:1003300001F012FBFEE701F08DFA00DFFEE700009E
:1003400038B501F0CDFE054601F0F0FE0446D8B9FF
:100350000F4B9D421AD001339D4218BF044641F213
:10036000883504BF01240025002001F0C3FE0CB134
:1003700000F076F800F010FD00F09EFB284600F03B
:10038000BFF800F06DF8F9E70025EDE70546EBE76B
:10039000010007B008B500F061FBA0F1200358424E
:1003A000584108BD07B541F21203022101A8ADF87A
:1003B000043000F071FB03B05DF804FB38B5202376
:1003C00083F311881748C3680BB101F04BFB164A41
:1003D000144800234FF47A7101F008FB002383F3E3
:1003E0001188124C236813B12368013B23606368B2
:1003F00013B16368013B63600D4D2B7833B96368BB
:100400007BB9022000F042FC322363602B78032B7F
:1004100007D163682BB9022000F038FC4FF47A73DF
:10042000636038BD40220020BD0300085C2300202B
:1004300054220020084B187003280CD8DFE800F085
:1004400008050208022000F017BC022000F00ABCD8
:10045000024B00225A607047542200205C23002087
:10046000234B244A10B51C46196801313FD0043390
:100470009342F9D16268A24239D31F4B9B6803F1C2
:10048000006303F540439A4231D2002000F02EFB76
:100490000220FFF7CFFF194B1A6C00221A64196E65
:1004A0001A66196E596C5A64596E5A665A6E5A69B0
:1004B00042F080025A615A6922F080025A615A69F8
:1004C0001A6942F000521A611A6922F000521A6148
:1004D0001B6972B64FF0E0232021C3F8084DD4E920
:1004E000003281F311889D4683F30888104710BDC0
:1004F00000C0000820C00008002200200038024090
:100500002DE9F04F93B0A94B00902022FF210AA8BB
:100510009D6800F0EBFBA64A1378A3B9A54801211A
:10052000C3601170202383F31188C3680BB101F0FD
:1005300099FAA14A9F4800234FF47A7101F056FAC4
:10054000002383F31188009B13B19C4B009A1A601F
:100550009B4A009C1378032B1EBF00231370974AFD
:100560004FF0000A18BF5360D3465646D1460120CB
:1005700000F082FB24B1914B1B68002B00F00F822E
:10058000002000F06BFA0390039B002BF2DB0120AC
:1005900000F068FB039B213B162BE8D801A252F820
:1005A00023F000BF0106000829060008BD06000868
:1005B0006F0500086F0500086F0500084507000873
:1005C000130900082D0800088F080008B708000864
:1005D000DD0800086F050008EF0800086F05000837
:1005E00061090008A10600086F050008A5090008B8
:1005F0000D060008A10600086F0500088F08000816
:100600000220FFF7C7FE002840F0F381009B022183
:10061000BAF1000F08BF1C4605A841F21233ADF82D
:10062000143000F039FAA2E74FF47A7000F016FAAD
:10063000071EEBDB0220FFF7ADFE0028E6D0013FEE
:10064000052F00F2D881DFE807F0030A0D101336FA
:1006500005230593042105A800F01EFA17E053486E
:100660000421F9E757480421F6E757480421F3E746
:100670004FF01C08404600F03BFA08F104080590D2
:10068000042105A800F008FAB8F12C0FF2D10120DE
:1006900000FA07F747EA0B0B5FFA8BFB4FF00009F4
:1006A00000F070FB26B10BF00B030B2B08BF0024EE
:1006B000FFF778FE5BE745480421CDE7002EA5D083
:1006C0000BF00B030B2BA1D10220FFF763FE0746B3
:1006D00000289BD0012000F009FA0220FFF7AAFEB3
:1006E00000265FFA86F8404600F010FA044688B10A
:1006F000404600F01BFA01360028F2D1BA46044603
:1007000041F21213022105A8ADF814303E4600F064
:10071000C3F92CE70120FFF78DFE2546234B9B688C
:10072000AB4207D9284600F0E3F9013040F066817A
:100730000435F3E7224B00251D70204BBA465D605F
:100740003E46ADE7002E3FF461AF0BF00B030B2BE1
:100750007FF45CAF0220FFF76DFE322000F07EF9DF
:10076000B0F10008FFF652AF18F003077FF44EAF68
:100770000E4A926808EB050393423FF647AFB8F57F
:10078000807F3FF743AF124B0193B84522DD4FF412
:100790007A7000F063F90390039A002AFFF636AFEF
:1007A000019B039A03F8012B0137EDE7002200209B
:1007B0005823002040220020BD0300085C230020B5
:1007C0005422002004220020082200200C220020B5
:1007D00058220020C820FFF7DDFD074600283FF41F
:1007E00015AF1F2D11D8C5F1200242450AAB25F0E7
:1007F000030028BF424683490192184400F050FA92
:10080000019A8048FF2100F071FA4FEAA8037D4960
:100810000193C8F38702284600F070FA06460028C4
:100820003FF46EAF019B05EB830539E70220FFF72C
:10083000B1FD00283FF4EAAE00F0A2F900283FF431
:10084000E5AE0027B846704B9B68BB4218D91F2FF6
:1008500011D80A9B01330ED027F0030312AA1344C8
:1008600053F8203C05934046042205A900F000FB04
:1008700004378046E7E7384600F03AF90590F2E79A
:10088000CDF81480042105A800F006F908E700233C
:10089000642104A8049300F0F5F800287FF4B6AEB4
:1008A0000220FFF777FD00283FF4B0AE049800F077
:1008B0004FF90590E6E70023642104A8049300F0B3
:1008C000E1F800287FF4A2AE0220FFF763FD0028C4
:1008D0003FF49CAE049800F04BF9EAE70220FFF7E2
:1008E00059FD00283FF492AE00F05AF9E1E70220EA
:1008F000FFF750FD00283FF489AE05A9142000F051
:1009000055F904210746049004A800F0C5F83946BB
:10091000B9E7322000F0A2F8071EFFF677AEBB075A
:100920007FF474AE384A926807EB090393423FF6AE
:100930006DAE0220FFF72EFD00283FF467AE27F0D2
:1009400003074F44B9453FF4ABAE484600F0D0F83A
:100950000421059005A800F09FF809F10409F1E7CA
:100960004FF47A70FFF716FD00283FF44FAE00F009
:1009700007F9002844D00A9B01330BD008220AA9AA
:10098000002000F0BBF900283AD02022FF210AA85D
:1009900000F0ACF9FFF706FD1C4800F0E3FF13B0D0
:1009A000BDE8F08F002E3FF431AE0BF00B030B2BA4
:1009B0007FF42CAE0023642105A8059300F062F8B3
:1009C000074600287FF422AE0220FFF7E3FC8046B2
:1009D00000283FF41BAEFFF7E5FC41F2883000F041
:1009E000C1FF059800F000FA464600F0CBF93C46FE
:1009F000BDE5064654E64FF0000907E6BA467FE635
:100A000037467DE65822002000220020A086010003
:100A100070B50F4B1B780133DBB2012B0C4611D89C
:100A20000C4D29684FF47A730E6AA2FB033201461B
:100A300022462846B047844204D1074B00221A7050
:100A4000012070BD4FF4FA7000F08CFF0020F8E731
:100A500010220020502500209023002007B50023FD
:100A6000024601210DF107008DF80730FFF7D0FF96
:100A700020B19DF8070003B05DF804FB4FF0FF3094
:100A8000F9E700000A4608B50421FFF7C1FF80F02E
:100A90000100C0B2404208BD30B4054C2368DD6996
:100AA000044B0A46AC460146204630BC604700BFB6
:100AB00050250020A086010070B501F003FA094E10
:100AC000094D3080002428683388834208D901F01A
:100AD000F3F92B6804440133B4F5404F2B60F2D393
:100AE00070BD00BF922300206423002001F0ACBA47
:100AF00000F1006000F540400068704700F10060C0
:100B0000920000F5404001F02BBA0000054B1A6836
:100B1000054B1B889B1A834202D9104401F0CCB9C3
:100B200000207047642300209223002038B5074D31
:100B300004462868204401F0C7F928B928682044F1
:100B4000BDE8384001F0D8B938BD00BF64230020AB
:100B500010F003030AD1B0F5047F05D200F1005074
:100B6000A0F51040D0F80038184670470023FBE786
:100B700000F10050A0F51040D0F8100A70470000B6
:100B8000064991F8243033B10023086A81F82430F3
:100B90000822FFF7B3BF0120704700BF6823002081
:100BA000014B1868704700BF002004E070B52A4B65
:100BB0001B68C3F30B0204461B0C62B140F21340E6
:100BC000824230D040F2194082422ED040F2214081
:100BD00082422CD10322214D0C2000FB0252556889
:100BE00042F20102934224D0B3F5805F23D041F258
:100BF0000102934221D041F2030293421FD041F2FD
:100C00000702934214BF3F233123013C0C44013DB2
:100C10000A46A24215D215F9016F501C9EB100F888
:100C2000016C0246F5E70122D5E70222D3E70C4D1D
:100C3000D6E73323E9E74123E7E75A23E5E75923DA
:100C4000E3E7104605E02C258442157001D9901C7D
:100C50005370401A70BD00BF002004E078340008D3
:100C60004C340008022802BF024B4FF080729A6198
:100C7000704700BF00080240022802BF024B4FF439
:100C800080729A61704700BF00080240022801BFCD
:100C9000024A536983F4807353617047000802402D
:100CA00010B50023934203D0CC5CC4540133F9E760
:100CB00010BD000010B5013810F9013F3BB191F9AA
:100CC00000409C4203D11AB10131013AF4E71AB154
:100CD00091F90020981A10BD1046FCE70346024621
:100CE000D01A12F9011B0029FAD1704702440346B9
:100CF000934202D003F8011BFAE770472DE9F8434D
:100D00001F4D144695F824200746884652BBDFF84D
:100D100070909CB395F824302BB92022FF214846CF
:100D20002F62FFF7E3FF95F82400C0F10802A2420A
:100D300028BF2246D6B24146920005EB8000FFF75D
:100D4000AFFF95F82430A41B1E44F6B2082E1744BA
:100D50009044E4B285F82460DBD1FFF711FF00284E
:100D6000D7D108E02B6A03EB82038342CFD0FFF791
:100D700007FF0028CBD10020BDE8F8830120FBE766
:100D800068230020024B1A78024B1A70704700BF8C
:100D9000902300201022002010B50F4C0F4800F0C7
:100DA000F7F821460D4800F01FF924680C48626DE1
:100DB000D2F8043843F00203C2F8043800F0D2FD40
:100DC0000849204600F016FA626DD2F8043823F084
:100DD0000203C2F8043810BD6C350008502500200D
:100DE00040420F00743500087047000000B59BB00A
:100DF000EFF3098168226846FFF752FFEFF305839E
:100E0000044B9A6BDA6A9A6A9A6A9A6A9A6A9A6A36
:100E10009B6AFEE700ED00E000B59BB0EFF30981AF
:100E200068226846FFF73CFFEFF30583044B9A6B9B
:100E30009A6A9A6A9A6A9A6A9A6A9B6AFEE700BFF5
:100E400000ED00E000B59BB0EFF309816822684631
:100E5000FFF726FFEFF30583034B5A6B9A6A9A6AF2
:100E60009A6A9A6A9B6AFEE700ED00E0FEE70000DE
:100E700030B5094D0A4491420DD011F8013B58405C
:100E8000082340F30004013B2C4013F0FF0384EAE5
:100E90005000F6D1EFE730BD2083B8ED026843681B
:100EA0001143016003B118477047000013B5446B4C
:100EB000D4F894341A681178042915D1217C0229B8
:100EC00012D11979128901238B4013420CD101A947
:100ED00004F14C0001F03CFFD4F89444019B2179CB
:100EE0000246206800F0CEF902B010BD143001F0C7
:100EF000BFBE00004FF0FF33143001F0B9BE000058
:100F00004C3001F091BF00004FF0FF334C3001F046
:100F10008BBF0000143001F08DBE00004FF0FF3198
:100F2000143001F087BE00004C3001F05DBF0000BE
:100F30004FF0FF324C3001F057BF000000207047E7
:100F400010B5D0F894341A6811780429044617D1E2
:100F5000017C022914D15979528901238B40134213
:100F60000ED1143001F020FE024648B1D4F894446A
:100F70004FF4807361792068BDE8104000F070B9CB
:100F800010BD0000406BFFF7DBBF000070470000A2
:100F90007FB5124B036000234360C0E90233012593
:100FA00002260F4B057404460290019300F184025F
:100FB000294600964FF48073143001F0D1FD094B9F
:100FC0000294CDE9006304F523724FF4807329463F
:100FD00004F14C0001F098FE04B070BDA834000884
:100FE000850F0008AD0E00080B68202282F31188DF
:100FF0000A7903EB820290614A79093243F82200B0
:101000008A7912B103EB8203986102230374C0F85A
:101010009414002383F311887047000038B5037FD0
:10102000044613B190F85430ABB9201D01250221BC
:10103000FFF734FF04F1140025776FF0010100F091
:10104000B9FC84F8545004F14C006FF00101BDE884
:10105000384000F0AFBC38BD10B501210446043063
:10106000FFF71CFF0023237784F8543010BD0000E5
:1010700038B504460025143001F08AFD04F14C0017
:10108000257701F059FE201D84F854500121FFF707
:1010900005FF2046BDE83840FFF752BF90F84430C6
:1010A00003F06003202B07D190F84520212A4FF050
:1010B000000303D81F2A06D800207047222AFBD13C
:1010C000C0E90E3303E0034A82630722C26303646C
:1010D000012070471122002037B5D0F894341A68E7
:1010E0001178042904461AD1017C022917D11979F3
:1010F000128901238B40134211D100F14C0528467F
:1011000001F0DAFE58B101A9284601F021FED4F819
:101110009444019B21790246206800F0B3F803B0A3
:1011200030BD0000F0B500EB810385B09E69044638
:101130000D46FEB1202383F3118804EB8507301D93
:101140000821FFF7ABFEFB685B691B6806F14C00EA
:101150001BB1019001F00AFE019803A901F0F8FD0E
:10116000024648B1039B2946204600F08BF8002335
:1011700083F3118805B0F0BDFB685A691268002A34
:10118000F5D01B8A013B1340F1D104F14402EAE798
:10119000093138B550F82140DCB1202383F31188A0
:1011A000D4F894241368527903EB8203DB689B69BB
:1011B0005D6845B104216018FFF770FE294604F10F
:1011C000140001F0FBFC2046FFF7BAFE002383F376
:1011D000118838BD7047000001F0A8B801230370E2
:1011E0000023C0E90133C36183620362C3624362C7
:1011F0000363704738B50446202383F31188002524
:10120000C0E90355C0E90555416001F09FF802238C
:10121000237085F3118838BD70B500EB8103054656
:101220005069DA600E46144618B110220021FFF70B
:101230005DFDA06918B110220021FFF757FD31466E
:101240002846BDE8704001F04BB90000826802F00A
:10125000011282600022C0E90422826101F0CCB94F
:10126000F0B400EB81044789E4680125A4698D404E
:101270003D43458123600023A2606360F0BC01F020
:10128000E7B90000F0B400EB81040789E4680125A8
:1012900064698D403D43058123600023A260636043
:1012A000F0BC01F061BA000070B5022300250446CD
:1012B0000370C0E90255C0E90455C564856180F832
:1012C000345001F0A9F863681B6823B12946204611
:1012D000BDE87040184770BD037880F85030052392
:1012E000037043681B6810B504460BB1042198478E
:1012F0000023A36010BD000090F8502043680270E6
:101300001B680BB1052118477047000070B590F8B5
:101310003430044613B1002380F8343004F1440221
:10132000204601F08BF963689B68B3B994F84430A8
:1013300013F0600535D00021204601F0DDFB0021CF
:10134000204601F0CFFB63681B6813B106212046DD
:101350009847062384F8343070BD2046984700280B
:10136000E4D0B4F84A30E26B9A4288BFE36394F960
:101370004430E56B002B4FF0200380F20381002DF9
:1013800000F0F280092284F8342083F311880021D0
:10139000D4E90E232046FFF775FF002383F311885D
:1013A000DAE794F8452003F07F0343EA022340F292
:1013B0000232934200F0C58021D8B3F5807F48D037
:1013C0000DD8012B3FD0022B00F09380002BB2D11F
:1013D00004F14C02A2630222E2632364C1E7B3F585
:1013E000817F00F09B80B3F5407FA4D194F8463014
:1013F000012BA0D1B4F84C3043F0020332E0B3F536
:10140000006F4DD017D8B3F5A06F31D0A3F5C063EE
:10141000012B90D8636894F846205E6894F84710D2
:10142000B4F848302046B047002884D04368A3630E
:101430000368E3631AE0B3F5106F36D040F602425A
:1014400093427FF478AF5C4BA3630223E3630023F2
:10145000C3E794F84630012B7FF46DAFB4F84C30FD
:1014600023F00203C4E90E55A4F84C30256478E754
:10147000B4F84430B3F5A06F0ED194F8463084F838
:101480004E30204601F020F863681B6813B101213B
:1014900020469847032323700023C4E90E339CE7BA
:1014A00004F14F03A3630123C3E72378042B10D176
:1014B000202383F311882046FFF7C8FE85F31188A7
:1014C0000321636884F84F5021701B680BB12046DC
:1014D000984794F84630002BDED084F84F30042330
:1014E000237063681B68002BD6D0022120469847E2
:1014F000D2E794F848301D0603F00F0120460AD5C4
:1015000001F08EF8012804D002287FF414AF2B4B91
:101510009AE72B4B98E701F075F8F3E794F846301B
:10152000002B7FF408AF94F8483013F00F01B3D0CC
:101530001A06204602D501F0F3FAADE701F0E6FA0B
:10154000AAE794F84630002B7FF4F5AE94F84830C3
:1015500013F00F01A0D01B06204602D501F0CCFAF3
:101560009AE701F0BFFA97E7142284F8342083F356
:1015700011882B462A4629462046FFF771FE85F33F
:101580001188E9E65DB1152284F8342083F31188CF
:101590000021D4E90E232046FFF762FEFDE60B2270
:1015A00084F8342083F311882B462A4629462046A6
:1015B000FFF768FEE3E700BFD8340008D034000826
:1015C000D434000838B590F834300446002B3ED0AF
:1015D000063BDAB20F2A34D80F2B32D8DFE803F0FB
:1015E0003731310822323131313131313131373710
:1015F000C56BB0F84A309D4214D2C3681B8AB5FB54
:10160000F3F203FB12556DB9202383F311882B46A7
:101610002A462946FFF736FE85F311880A2384F807
:1016200034300EE0142384F83430202383F31188FF
:1016300000231A4619462046FFF712FE002383F3C3
:10164000118838BD036C03B198470023E7E70021F8
:10165000204601F051FA0021204601F043FA636868
:101660001B6813B10621204698470623D7E70000E0
:1016700010B590F83430142B044629D017D8062B17
:1016800005D001D81BB110BD093B022BFBD80021AE
:10169000204601F031FA0021204601F023FA636868
:1016A0001B6813B1062120469847062319E0152B25
:1016B000E9D10B2380F83430202383F311880023F1
:1016C0001A461946FFF7DEFD002383F31188DAE797
:1016D000C3689B695B68002BD5D1036C03B1984745
:1016E000002384F83430CEE7024B0022C3E90033F4
:1016F0009A60704794230020002303748268054B8E
:101700001B6899689142FBD25A680360426010607E
:10171000586070479423002008B5202383F3118874
:10172000037C032B05D0042B0DD02BB983F3118838
:1017300008BD436900221A604FF0FF334361FFF791
:10174000DBFF0023F2E7D0E9003213605A60F3E7D1
:10175000002303748268054B1B6899689142FBD88B
:101760005A680360426010605860704794230020FC
:10177000054B19690874186802681A60536018618B
:1017800001230374FEF7C2BD9423002030B54B1C27
:101790000B4D87B0044610D02B690A4A01A800F00F
:1017A00025F92046FFF7E4FF049B13B101A800F0E0
:1017B00059F92B69586907B030BDFFF7D9FFF8E731
:1017C000942300201917000838B50C4D41612B698E
:1017D00081689A689142044603D8BDE83840FFF713
:1017E0008BBF1846FFF7B4FF01232C610146237419
:1017F0002046BDE83840FEF789BD00BF9423002095
:10180000044B1A681B6990689B68984294BF00203B
:10181000012070479423002010B5084C23682069EC
:101820001A6822605460012223611A74FFF790FF46
:1018300001462069BDE81040FEF768BD94230020F2
:1018400008B5FFF7DDFF18B1BDE80840FFF7E4BFBA
:1018500008BD0000FFF7E0BFFEE7000010B50C4C2C
:10186000FFF742FF00F0B4F80A498022204600F05A
:101870003BF8012344F8180C037400F071FC0023BA
:1018800083F3118862B60448BDE8104000F04CB8FC
:10189000BC230020DC340008EC34000800F01CB944
:1018A000EFF3118020B9EFF30583202282F3118832
:1018B0007047000010B530B9EFF30584C4F3080495
:1018C00014B180F3118810BDFFF7BAFF84F31188BB
:1018D000F9E70000034A516853685B1A9842FBD845
:1018E000704700BF001000E0826002220282704751
:1018F0008368A3F17C0243F80C2C026943F83C2C6A
:10190000426943F8382C074A43F81C2CC26843F854
:10191000102C022203F8082C002203F8072CA3F154
:10192000180070472503000810B5202383F31188A1
:10193000FFF7DEFF00210446FFF746FF002383F395
:101940001188204610BD0000024B1B6958610F2012
:10195000FFF70EBF94230020202383F31188FFF7A5
:10196000F3BF000008B50146202383F31188082047
:10197000FFF70CFF002383F3118808BD49B1064B24
:1019800042681B6918605A60136043600420FFF7C7
:10199000FDBE4FF0FF30704794230020036898424B
:1019A00006D01A680260506059611846FFF7A4BE5D
:1019B0007047000038B504460D462068844200D1C7
:1019C00038BD036823605C604561FFF795FEF4E76E
:1019D000054B03F11402C3E905224FF0FF31002249
:1019E000C3E90712704700BF9423002070B51C4E56
:1019F000C0E9032305460C4601F090FA334653F83C
:101A0000142F9A420DD13062C5E901242A600A2CB4
:101A10002CBF00190A30C6E90555BDE8704001F039
:101A20006BBA316A431AE31838BF1C469368A34265
:101A300002D9081901F06EFA73699A6894420CD8B9
:101A40005A68AC602B606A6015609A685D60121B12
:101A50009A604FF0FF33F36170BD1B68A41AECE786
:101A60009423002038B51B4C636998420DD0D0E90F
:101A7000003213605A6000228168C2609A680A448A
:101A80009A604FF0FF33E36138BD2246036842F8A5
:101A9000143F002193425A60C16003D1BDE8384031
:101AA00001F032BA9A688168256A0A449A6001F0A6
:101AB00035FA63699A68411B8A42E5D9AB181D1A49
:101AC000092D206A98BF01F10A02BDE83840104490
:101AD00001F020BA942300202DE9F041184C002792
:101AE00004F11406656901F019FA236AAA68C11A9B
:101AF0008A4215D813442362D5E9003213605A6034
:101B00006369D5F80C80EF60B34201D101F0FCF9B4
:101B100087F311882869C047202383F31188E1E700
:101B20006169B14209D013441B1ABDE8F0410A2B88
:101B30002CBFC0180A3001F0EDB9BDE8F08100BF3C
:101B40009423002000207047FEE70000704700004B
:101B50004FF0FF307047000002290CD0032904D059
:101B60000129074818BF00207047032A05D80548F7
:101B700000EBC2007047044870470020704700BF68
:101B8000D0350008202200208435000870B59AB0B6
:101B90000546084601A9144600F0C2F801A8FFF75F
:101BA0009DF8431C5B00C5E9003400222370032329
:101BB0006370C6B201AB02341046D1B28E4204F15A
:101BC000020401D81AB070BD13F8011B04F8021CFE
:101BD00004F8010C0132F0E708B5202383F31188E3
:101BE0000348FFF779FA002383F3118808BD00BF8B
:101BF0005025002090F8443003F01F02012A07D13D
:101C000090F845200B2A03D10023C0E90E3315E0DC
:101C100003F06003202B08D1B0F848302BB990F8BE
:101C20004520212A03D81F2A04D8FFF737BA222AD1
:101C3000EBD0FAE7034A82630722C2630364012000
:101C4000704700BF1822002007B5052917D8DFE824
:101C500001F0191603191920202383F31188104A63
:101C600001900121FFF7D8FA01980E4A0221FFF7EF
:101C7000D3FA0D48FFF7FCF9002383F3118803B072
:101C80005DF804FB202383F311880748FFF7C6F9AA
:101C9000F2E7202383F311880348FFF7DDF9EBE730
:101CA00024350008483500085025002038B50C4D73
:101CB0000C4C0D492A4604F10800FFF767FF05F1B7
:101CC000CA0204F110000949FFF760FF05F5CA7266
:101CD00004F118000649BDE83840FFF757BF00BFC0
:101CE000182A002020220020043500080E350008A4
:101CF0001935000870B5044608460D46FEF7EEFF9C
:101D0000C6B22046013403780BB9184670BD32467E
:101D10002946FEF7CFFF0028F3D10120F6E70000A7
:101D20002DE9F04705460C46FEF7D8FF2B49C6B211
:101D30002846FFF7DFFF08B10636F6B228492846E5
:101D4000FFF7D8FF08B11036F6B2632E0BD8DFF8D4
:101D50008C80DFF88C90234FDFF894A02E7846B962
:101D60002670BDE8F08729462046BDE8F04701F01F
:101D700065BB252E2ED1072241462846FEF79AFF45
:101D800070B9194B224603F10C0153F8040B42F8C9
:101D9000040B8B42F9D11B78137007350D34DDE746
:101DA000082249462846FEF785FF98B90F4BA21C2A
:101DB000197809090232C95D02F8041C13F8011BE5
:101DC00001F00F015345C95D02F8031CF0D118342E
:101DD0000835C3E704F8016B0135BFE7F0350008AB
:101DE0001935000806360008F8350008107AFF1F7C
:101DF0001C7AFF1FBFF34F8F024AD368DB03FCD46A
:101E0000704700BF003C024008B5094B1B7873B90E
:101E1000FFF7F0FF074B1A69002ABFBF064A5A6056
:101E200002F188325A601A6822F480621A6008BD92
:101E3000762C0020003C02402301674508B50B4B7F
:101E40001B7893B9FFF7D6FF094B1A6942F000429D
:101E50001A611A6842F480521A601A6822F4805299
:101E60001A601A6842F480621A6008BD762C00205D
:101E7000003C02400B28F0B516D80C4C0C492378D6
:101E80007BB90C4D0E460C234FF0006255F8047BD5
:101E900046F8042B013B13F0FF033A44F6D101232B
:101EA000237051F82000F0BD0020FCE7A82C002092
:101EB000782C002018360008014B53F8200070479A
:101EC000183600080C2070470B2810B5044601D9BD
:101ED000002010BDFFF7CEFF064B53F82430184406
:101EE000C21A0BB90120F4E712680132F0D1043BA9
:101EF000F6E700BF183600080B2838B5044628D886
:101F0000FFF7CEFCFFF776FFFFF77EFF124AF323C1
:101F1000D360E300DBB243F4007343F002031361C8
:101F2000136943F48033136105462046FFF762FFCF
:101F3000FFF7A0FF094B53F8241000F0E9F82846FA
:101F4000FFF77CFFFFF7B6FC2046BDE83840FFF7FF
:101F5000BBBF002038BD00BF003C0240183600085F
:101F600012F001032DE9F04105460E4614464BD10F
:101F70008218B2F1016F61D8314B1B6813F0010375
:101F80005CD0304FFFF78CFCFFF73EFFF323FB6084
:101F9000FFF730FF314640F20128032C18D824F017
:101FA0000104284E0C446D1A40F20118A142336915
:101FB00005EB01072AD123F001033361FFF73EFF50
:101FC000FFF778FC0120BDE8F081043C0435E4E72C
:101FD000AB07E4D13B6923F440733B613B6943EABF
:101FE00008033B6151F8046B2E60BFF34F8FFFF77E
:101FF00001FF2B689E42E8D03B6923F001033B615F
:10200000FFF71CFFFFF756FC0020DCE723F44073CA
:102010003361336943EA080333610B883B80BFF3C4
:102020004F8FFFF7E7FE3F8831F8023BBFB2BB425C
:10203000BCD0336923F001033361E1E71846C2E7FE
:1020400000380240003C0240084908B50B7828B12E
:102050001BB9FFF7D9FE01230B7008BD002BFCD084
:10206000BDE808400870FFF7E9BE00BF762C0020ED
:1020700010B50244064BD2B2904200D110BD441CB0
:1020800000B253F8200041F8040BE0B2F4E700BFBF
:10209000502800400F4B30B51C6F240407D41C6F30
:1020A00044F400741C671C6F44F400441C670A4C21
:1020B000236843F4807323600244084BD2B29042F9
:1020C00000D130BD441C00B251F8045B43F82050ED
:1020D000E0B2F4E7003802400070004050280040B1
:1020E00007B5012201A90020FFF7C2FF019803B044
:1020F0005DF804FB13B50446FFF7F2FFA04205D0DC
:10210000012201A900200194FFF7C4FF02B010BD15
:1021100070470000034B1A681AB9034AD2F87428B2
:102120001A607047AC2C00200030024008B5FFF761
:10213000F1FF024B1868C0F3407008BDAC2C0020C2
:10214000EFF3098305494A6B22F001024A636833C1
:1021500083F30988002383F31188704700EF00E0C0
:10216000202080F3118862B60C4B0D4AD96821F407
:10217000E0610904090C0A43DA60D3F8FC2009493C
:1021800042F08072C3F8FC200A6842F001020A6043
:102190001022DA7783F82200704700BF00ED00E0DC
:1021A0000003FA05001000E010B5202383F3118826
:1021B0000E4B5B6813F4006314D0F1EE103AEFF3AA
:1021C0000984683C4FF08073E361094BDB6B236645
:1021D00084F30988FFF714FB10B1064BA36110BD0F
:1021E000054BFBE783F31188F9E700BF00ED00E042
:1021F00000EF00E0370300083A03000870470000D2
:10220000FEE700000A4B0B480B4A90420BD30B4BE6
:10221000DA1C121AC11E22F003028B4238BF0022C0
:102220000021FEF763BD53F8041B40F8041BECE7E4
:10223000B8370008A82D0020A82D0020A82D0020C8
:102240007047000070B5D0E915439E6800224FF03A
:10225000FF3504EB42135101D3F800090028BEBF3B
:10226000D3F8000940F08040C3F80009D3F8000B10
:102270000028BEBFD3F8000B40F08040C3F8000B2D
:10228000013263189642C3F80859C3F8085BE0D2DC
:102290004FF00113C4F81C3870BD00001D4B03EB58
:1022A00080022DE9F043D2F80CC05D6DDCF81420FB
:1022B000461CD2F800E005EB063605EB40185168E5
:1022C00071450AD3D5F83438012202FA00F023EA26
:1022D0000000C5F83408BDE8F083BCF81040AEEB50
:1022E0000103A34228BF2346D8F81849A4B2B3EB90
:1022F000840FF0D89468A4F1040959F8047F37607A
:10230000A4EB09071F44042FF7D81C440B44946026
:102310005360D4E7B02C0020890141F02001016115
:1023200003699B06FCD41220FFF7D4BA10B5054C04
:102330002046FEF753FF4FF0A0436365024BA365B1
:1023400010BD00BFB02C00206C36000870B50378BB
:10235000012B054650D12A4B446D98421BD1294B85
:102360005A6B42F080025A635A6D42F080025A65FD
:102370005A6D5A6942F080025A615A6922F080020D
:102380005A610E2143205B6900F0D4FB1E4BE360D1
:102390001E4BC4F800380023C4F8003EC02323605D
:1023A0006E6D4FF40413A3633369002BFCDA012331
:1023B00033610C20FFF78EFA3369DB07FCD412205F
:1023C000FFF788FA3369002BFCDA0026A66028465E
:1023D000FFF738FF6B68C4F81068DB68C4F814684E
:1023E000C4F81C684BB90A4BA3614FF0FF3363611B
:1023F000A36843F00103A36070BD064BF4E700BF80
:10240000B02C00200038024040140040030020029D
:10241000003C30C0083C30C0F8B5446D0546002192
:102420002046FFF779FFA96D00234FF001128F6856
:10243000C4F834384FF00066C4F81C284FF0FF3061
:1024400004EB431201339F42C2F80069C2F8006BEB
:10245000C2F80809C2F8080BF2D20B686A6DEB6586
:10246000636210231361166916F01006FBD1122067
:10247000FFF730FAD4F8003823F4FE63C4F80038CC
:10248000A36943F4402343F01003A3610923C4F874
:102490001038C4F814380A4BEB604FF0C043C4F84E
:1024A000103B084BC4F8003BC4F81069C4F800396D
:1024B000EB6D03F1100243F48013EA65A362F8BDEB
:1024C0004836000840800010426D90F84E10D2F857
:1024D000003823F4FE6343EA0113C2F80038704762
:1024E0002DE9F84300EB8103456DDA68166806F0C4
:1024F0000306731E022B05EB41130C4680460FFAB0
:1025000081F94FEA41104FF00001C3F8101B4FF062
:10251000010104F1100398BFB60401FA03F39169B5
:102520008EBF334E06F1805606F5004600293AD09C
:10253000578A04F15801490137436F50D5F81C18E8
:102540000B43C5F81C382B180021C3F81019536928
:102550000127611EA7409BB3138A928B9B08012A17
:1025600088BF5343D8F85C20981842EA034301F12E
:10257000400205EB8202C8F85C0021465360284601
:10258000FFF7CAFE08EB8900C3681B8A43EA84533D
:10259000483464011E432E51D5F81C381F43C5F83A
:1025A0001C78BDE8F88305EB4917D7F8001B21F428
:1025B0000041C7F8001BD5F81C1821EA0303C0E747
:1025C00004F13F0305EB83030A4A5A60284621467B
:1025D000FFF7A2FE05EB4910D0F8003923F40043C1
:1025E000C0F80039D5F81C3823EA0707D7E700BF41
:1025F0000080001000040002826D1268C265FFF7BF
:1026000021BE00005831436D49015B5813F400406E
:1026100004D013F4001F0CBF0220012070470000FB
:102620004831436D49015B5813F4004004D013F462
:10263000001F0CBF022001207047000000EB810149
:10264000CB68196A0B6813604B68536070470000D1
:1026500000EB810330B5DD68AA691368D36019B94E
:10266000402B84BF402313606B8A1468426D1C4466
:10267000013CB4FBF3F46343033323F0030302EBA5
:10268000411043EAC44343F0C043C0F8103B2B68F9
:1026900003F00303012B09B20ED1D2F8083802EB84
:1026A000411013F4807FD0F8003B14BF43F08053F7
:1026B00043F00053C0F8003B02EB4112D2F8003B5C
:1026C00043F00443C2F8003B30BD00002DE9F04167
:1026D000244D6E6D06EB40130446D3F8087BC3F817
:1026E000087B38070AD5D6F81438190706D505EB44
:1026F00084032146DB6828465B689847FA071FD5A4
:10270000D6F81438DB071BD505EB8403D968CCB9A0
:102710008B69488A5A68B2FBF0F600FB16228AB928
:102720001868DA6890420DD2121AC3E900242023F7
:1027300083F311880B482146FFF78AFF84F3118841
:10274000BDE8F081012303FA04F26B8923EA020356
:102750006B81CB68002BF3D021460248BDE8F041E5
:10276000184700BFB02C002000EB810370B5DD6876
:10277000436D6C692668E6604A0156BB1A444FF403
:102780000020C2F810092A6802F00302012A0AB2E6
:102790000ED1D3F8080803EB421410F4807FD4F86C
:1027A000000914BF40F0805040F00050C4F8000908
:1027B00003EB4212D2F8000940F00440C2F80009CD
:1027C000D3F83408012202FA01F10143C3F83418A6
:1027D00070BD19B9402E84BF4020206020682E8A29
:1027E0008419013CB4FBF6F440EAC44040F00050C8
:1027F0001A44C6E7F8B504461E48456D05EB441378
:10280000D3F80869C3F80869F10717D5D5F8103867
:10281000DA0713D500EB8403D9684B691F68DA68BF
:10282000974218D2D21B00271A605F60202383F3DF
:1028300011882146FFF798FF87F31188330617D5D3
:10284000D5F834280123A340134211D02046BDE817
:10285000F840FFF723BD012303FA04F2038923EABA
:10286000020303818B68002BE8D021469847E5E7F7
:10287000F8BD00BFB02C00202DE9F74F984C666DD5
:102880007569B3691D4015F48058756107D02046FD
:10289000FEF70AFD03B0BDE8F04FFFF785BC002D41
:1028A00012DAD6F8003E8E489F071EBFD6F8003ECB
:1028B00023F00303C6F8003ED6F8043823F00103E2
:1028C000C6F80438FEF718FD280505D58448FFF73B
:1028D000B9FC8348FEF700FDA9040CD5D6F80838EA
:1028E00013F0060FF36823F470530CBF43F4105336
:1028F00043F4A053F3602A0704D56368DB680BB187
:1029000077489847EB0274D4AF0227D5D4F8549097
:10291000DFF8CCB100274FF0010A09EB4712D2F8DB
:10292000003B03F44023B3F5802F11D1D2F8003BD4
:10293000002B0DDA62890AFA07F322EA03036381A6
:1029400004EB8703DB68DB6813B1394658469847C8
:10295000A36D01379B68FFB29F42DED9E80617D509
:10296000676D3A6AC2F30A1002F00F0302F4F01224
:10297000B2F5802F00F08880B2F5402F08D104EB2B
:1029800083030022DB681B6A07F5805790426DD1F4
:102990002903D6F8184813D5E20302D50020FFF723
:1029A00095FEA30302D50120FFF790FE670302D531
:1029B0000220FFF78BFE260302D50320FFF786FED9
:1029C0006D037FF567AFE00702D50020FFF712FF28
:1029D000A10702D50120FFF70DFF620702D50220F3
:1029E000FFF708FF23077FF555AF0320FFF702FF2E
:1029F00050E7636DDFF8E8B0019300274FF0010A5C
:102A0000A36D9B685FFA87F999453FF67DAF019BFF
:102A100003EB4913D3F8002902F44022B2F5802FCA
:102A200022D1D3F80029002A1EDAD3F8002942F077
:102A30009042C3F80029D3F80029002AFBDB606D1F
:102A40004946FFF769FC22890AFA09F322EA0303DF
:102A5000238104EB8903DB689B6813B14946584620
:102A600098474846FFF71AFC0137C9E7910708BFA6
:102A7000D7F80080072A98BF03F8018B02F1010202
:102A800098BF4FEA182881E7023304EB830207F569
:102A900080575268D2F818C0DCF80820DCE9001C26
:102AA000A1EB0C0C002188420AD104EB830463687B
:102AB0009B699A6802449A605A6802445A6067E7C0
:102AC00011F0030F08BFD7F800808C4588BF02F8CB
:102AD000018B01F1010188BF4FEA1828E3E700BF2D
:102AE000B02C0020436D03EB4111D1F8003B43F4BF
:102AF0000013C1F8003B7047436D03EB4111D1F85F
:102B0000003943F40013C1F800397047436D03EBFB
:102B10004111D1F8003B23F40013C1F8003B70478A
:102B2000436D03EB4111D1F8003923F40013C1F8D0
:102B30000039704700F1604303F561430901C9B2F0
:102B400083F80013012200F01F039A4043099B0001
:102B500003F1604303F56143C3F880211A607047B5
:102B600030B5039C0172043304FB0325C0E906530E
:102B7000049B03630021059BC160C0E90000C0E91C
:102B80000422C0E90842C0E90A11436330BD0000D5
:102B9000416A0022C0E90411C0E90A22C2606FF054
:102BA0000101FEF707BF0000D0E90432934201D1D2
:102BB000C2680AB9181D7047002070470369196080
:102BC000C2680132C260C2691344826903619342E0
:102BD00024BF436A03610021FEF7E0BE38B5044616
:102BE0000D46E3683BB16269131D1268A36213448A
:102BF000E362002007E0237A33B929462046FEF736
:102C0000BDFE0028EDDA38BD6FF00100FBE70000E3
:102C1000C368C269013BC36043691344826943616D
:102C2000934224BF436A436100238362036B03B171
:102C30001847704770B52023044683F31188866ACD
:102C40003EB9FFF7CBFF054618B186F31188284639
:102C500070BDA36AE26A13F8015BA362934202D3D8
:102C60002046FFF7D5FF002383F31188EFE700002C
:102C70002DE9F84F04460E46174698464FF02009B6
:102C800089F311880025AA46D4F828B0BBF1000FBB
:102C900009D141462046FFF7A1FF20B18BF31188EF
:102CA0002846BDE8F88FD4E90A12A7EB050B521AA3
:102CB000934528BF9346BBF1400F1BD9334601F122
:102CC000400251F8040B43F8040B9142F9D1A36A76
:102CD00040334036A3624035D4E90A239A4202D3F6
:102CE0002046FFF795FF8AF31188BD42D8D289F3B9
:102CF0001188C9E730465A46FDF7D2FFA36A5B4404
:102D00005E44A3625D44E7E710B5029C01720433A0
:102D100004FB0321C0E906130023C0E90A33039B27
:102D20000363049BC460C0E90000C0E90422C0E959
:102D30000842436310BD0000026AC260426AC0E9F3
:102D400004220022C0E90A226FF00101FEF732BE20
:102D5000D0E904239A4201D1C26822B9184650F83A
:102D6000043B0B607047002070470000C368C269D5
:102D70000133C3604369134482694361934224BFB2
:102D8000436A43610021FEF709BE000038B50446DE
:102D90000D46E3683BB123691A1DA262E269134440
:102DA000E362002007E0237A33B929462046FEF784
:102DB000E5FD0028EDDA38BD6FF00100FBE700000B
:102DC00003691960C268013AC260C269134482692A
:102DD0000361934224BF436A036100238362036B50
:102DE00003B118477047000070B520230D46044614
:102DF000114683F31188866A2EB9FFF7C7FF10B119
:102E000086F3118870BDA36A1D70A36AE26A01335C
:102E10009342A36204D3E16920460439FFF7D0FF4F
:102E2000002080F31188EDE72DE9F84F04460D46A8
:102E3000904699464FF0200A8AF311880026B3463F
:102E4000A76A4FB949462046FFF7A0FF20B187F394
:102E500011883046BDE8F88FD4E90A073A1AA8EB82
:102E60000607974228BF1746402F1BD905F140039C
:102E700055F8042B40F8042B9D42F9D1A36A403346
:102E8000A3624036D4E90A239A4204D3E16920467A
:102E90000439FFF795FF8BF311884645D9D28AF3A1
:102EA0001188CDE729463A46FDF7FAFEA36A3B446E
:102EB0003D44A3623E44E5E7D0E904239A4217D19A
:102EC000C3689BB1836A8BB1043B9B1A0ED013601D
:102ED000C368013BC360C3691A44836902619A42B3
:102EE00024BF436A036100238362012318467047AD
:102EF0000023FBE700F088B84FF0804300225863BE
:102F00001A610222DA6070474FF080430022DA60D3
:102F1000704700004FF08043586370474FF0804384
:102F2000586A70474B6843608B688360CB68C360A6
:102F30000B6943614B6903628B6943620B680360F1
:102F40007047000008B5264B26481A6940F2FF1169
:102F50000A431A611A6922F4FF7222F001021A610F
:102F60001A691A6B0A431A631A6D0A431A651E4AD4
:102F70001B6D1146FFF7D6FF02F11C0100F58060C2
:102F8000FFF7D0FF02F1380100F58060FFF7CAFFBC
:102F900002F1540100F58060FFF7C4FF02F17001F7
:102FA00000F58060FFF7BEFF02F18C0100F5806044
:102FB000FFF7B8FF02F1A80100F58060FFF7B2FF4C
:102FC00002F1C40100F58060FFF7ACFF02F1E001FF
:102FD00000F58060FFF7A6FFBDE8084000F09AB852
:102FE00000380240000002407836000808B500F0C2
:102FF00007FAFEF733FCFFF78DF8BDE80840FEF74F
:1030000055BE000070470000104B1A6C42F00102E0
:103010001A641A6E42F001021A660D4A1B6E93681A
:1030200043F0010393604FF0804353229A624FF0C4
:10303000FF32DA6200229A615A63DA605A60012232
:103040005A6108211A601C20FFF774BD0038024045
:10305000002004E04FF0804208B51169D3680B40AE
:10306000D9B2C9439B07116107D5202383F3118887
:10307000FEF714FC002383F3118808BD08B5FFF7A1
:10308000E9FFBDE80840FFF78FB800001F4B1A6941
:103090006FEAC2526FEAD2521A611A69C2F3080289
:1030A0001A614FF0FF301A695A69586100215A6954
:1030B00059615A691A6A62F080521A621A6A02F0F9
:1030C00080521A621A6A5A6A58625A6A59625A6A6D
:1030D0001A6C42F080521A641A6E42F080521A66DC
:1030E0001A6E0B4A106840F480701060186F00F47C
:1030F0004070B0F5007F1EBF4FF48030186719672D
:10310000536823F40073536000F05AB9003802404A
:1031100000700040334B4FF080521A64324A4FF433
:10312000404111601A6842F001021A601A68910762
:10313000FCD59A6822F003029A602A4B9A6812F032
:103140000C02FBD1196801F0F90119609A601A6844
:1031500042F480321A601A689203FCD55A6F42F02A
:1031600001025A671F4B5A6F9007FCD51F4A5A60DD
:103170001A6842F080721A601B4A53685904FCD5E1
:10318000184B1A689201FCD5194A9A60194B1A68B3
:10319000194B9A42194B21D1194A1168194A914287
:1031A0001CD140F205121A60144A136803F00F0391
:1031B000052BFAD10B4B9A6842F002029A609A688A
:1031C00002F00C02082AFAD15A6C42F480425A6486
:1031D0005A6E42F480425A665B6E704740F2057246
:1031E000E1E700BF0038024000700040085440078B
:1031F00000948838002004E011640020003C024064
:1032000000ED00E041C20F41084A08B5516913685A
:103210000B4003F00103536123B1054A13680BB15E
:1032200050689847BDE80840FEF7BEBF003C01402B
:10323000282D0020084A08B5516913680B4003F097
:103240000203536123B1054A93680BB1D0689847D4
:10325000BDE80840FEF7A8BF003C0140282D002033
:10326000084A08B5516913680B4003F00403536121
:1032700023B1054A13690BB150699847BDE808406E
:10328000FEF792BF003C0140282D0020084A08B5F7
:10329000516913680B4003F00803536123B1054AD9
:1032A00093690BB1D0699847BDE80840FEF77CBF31
:1032B000003C0140282D0020084A08B551691368D8
:1032C0000B4003F01003536123B1054A136A0BB19D
:1032D000506A9847BDE80840FEF766BF003C0140D1
:1032E000282D0020174B10B55A691C68144004F4AF
:1032F00078725A61A30604D5134A936A0BB1D06A57
:103300009847600604D5104A136B0BB1506B984771
:10331000210604D50C4A936B0BB1D06B9847E2059C
:1033200004D5094A136C0BB1506C9847A30504D51A
:10333000054A936C0BB1D06C9847BDE81040FEF77E
:1033400033BF00BF003C0140282D00201A4B10B5B0
:103350005A691C68144004F47C425A61620504D521
:10336000164A136D0BB1506D9847230504D5134AC7
:10337000936D0BB1D06D9847E00404D50F4A136EDE
:103380000BB1506E9847A10404D50C4A936E0BB153
:10339000D06E9847620404D5084A136F0BB1506F82
:1033A0009847230404D5054A936F0BB1D06F984713
:1033B000BDE81040FEF7F8BE003C0140282D00207B
:1033C000062108B50846FFF7B5FB06210720FFF7E1
:1033D000B1FB06210820FFF7ADFB06210920FFF70E
:1033E000A9FB06210A20FFF7A5FB06211720FFF7FE
:1033F000A1FBBDE8084006212820FFF79BBB000089
:1034000008B5FFF743FE00F00BF8FDF7E5FEFDF70A
:10341000BDFDFFF7F7FDBDE80840FFF76BBD0000FD
:103420000023054A19460133102BC2E9001102F1AD
:103430000802F8D1704700BF282D0020034611F87C
:10344000012B03F8012B002AF9D1704753544D3357
:1034500032463F3F3F00000053544D333246343034
:10346000780053544D3332463432780053544D3340
:103470003246343436585800000000004C340008FE
:103480003F00000013040000583400083F00000013
:1034900019040000623400083F000000210400000D
:1034A0006C3400083F00000000000000090F000815
:1034B000F50E0008310F00081D0F0008290F000845
:1034C000150F0008010F0008ED0E00083D0F000861
:1034D0000000000001000000000000006D61696E46
:1034E0000000000069646C6500000000E43400081E
:1034F000D8230020502500200100000059180008A2
:10350000000000004172647550696C6F74002542C0
:103510004F415244252D424C002553455249414CC0
:103520002500000002000000000000002511000836
:103530009111000840004000E8290020F8290020EF
:103540000200000000000000030000000000000076
:10355000D51100080000000010000000082A00201B
:10356000000000000100000000000000B02C00205E
:1035700001010200491C0008591B0008F51B000846
:10358000D91B0008430000008C35000809024300E5
:10359000020100C0320904000001020201000524FA
:1035A0000010010524010001042402020524060084
:1035B00001070582030800FF09040100020A000058
:1035C00000070501024000000705810240000000DD
:1035D00012000000D835000812011001020000405E
:1035E000091241570002010203010000040309040B
:1035F00025424F41524425007370656564796265C8
:103600006566347633003031323334353637383905
:103610004142434445460000004000000040000095
:103620000040000000400000000001000000020017
:103630000000020000000200000002000000020082
:103640000000020000000200000000000D1300084E
:10365000C51500087116000840004000102D00201C
:10366000102D002001000000202D0020800000000F
:103670004001000003000000000180420000000043
:10368000AAAAAAAA00010040FFFF00000000000053
:1036900000A00A000000000100000000AAAAAAAAD7
:1036A00000000001FFFF000000000000000000001B
:1036B0000000010000000000AAAAAAAA0000000061
:1036C000FFFE0000000000000000000000000000FD
:1036D00000000000AAAAAAAA00000000FFFF000044
:1036E00000000000000000000000000000000000DA
:1036F000AAAAAAAA00000000FFFF00000000000024
:10370000000000000000000000000000AAAAAAAA11
:1037100000000000FFFF00000000000000000000AB
:103720000000000000000000AAAAAAAA00000000F1
:10373000FFFF00000000000000000000000000008B
:10374000000000000A00000000000000030000006C
:103750000000000000000000000000000000000069
:103760000000000000000000000000000000000059
:1037700000000000000000003A040000000000000B
:1037800000400F0000000000FF009600000000084D
:10379000009600000000080004000000EC3500085E
:1037A0000000000000000000000000000000000019
:1037B0000000000000000000FFFFFFFFFFFFFFFF11
:1037C000FFFFFFFFFFFFFFFFFFFFFFFFFFFFFFFF09
:1037D000FFFFFFFFFFFFFFFFFFFFFFFFFFFFFFFFF9
:1037E000FFFFFFFFFFFFFFFFFFFFFFFFFFFFFFFFE9
:1037F000FFFFFFFFFFFFFFFFFFFFFFFFFFFFFFFFD9
:10C0000000060020A9D2000855A90908B1A809080E
:10C010001DA90908B1A80908E9A80908ABD20008B8
:10C02000ABD20008ABD20008ABD2000829CC0B0879
:10C03000ABD20008ABD20008ABD20008ABD20008EC
:10C04000ABD20008ABD20008ABD20008ABD20008DC
:10C05000ABD20008ABD20008C1D70B08E9D70B0858
:10C0600011D80B0839D80B0861D80B08C1800B0810
:10C07000E9800B0815810B0841810B086D810B08C5
:10C0800095810B08C1810B0845800B08ABD20008D5
:10C09000ABD20008ABD20008ABD2000889D80B089D
:10C0A000ABD20008ABD20008ABD20008ABD200087C
:10C0B000ABD20008D5D90B08E9D90B08ABD20008E0
:10C0C000ABD200084D870B08F5880B08ABD20008EF
:10C0D000ABD200085DD90B0871D90B0885D90B08C4
:10C0E000EDD80B08ABD20008ABD200080DDA0B0874
:10C0F00011DA0B0825DA0B0829DA0B08ED810B0899
:10C10000ABD20008ABD20008FDD90B08ABD20008B7
:10C1100099D90B08ADD90B08ABD20008ABD20008F7
:10C1200019820B0841820B086D820B0899820B085B
:10C13000C5820B08ABD20008ABD20008ABD2000816
:10C14000ABD20008ABD20008ABD2000855D30B0825
:10C15000ED820B0819830B0845830B08C1D90B0826
:10C16000ABD20008ABD20008ABD20008ABD20008BB
:10C17000ABD20008ABD20008ABD20008ABD20008AB
:10C18000ABD20008ABD20008ABD20008ABD200089B
:10C19000ABD20008ABD20008ABD20008ABD200088B
:10C1A000ABD20008ABD20008ABD20008ABD200087B
:10C1B000ABD20008ABD20008ABD20008ABD200086B
:10C1C000ABD20008ABD20008ABD20008ABD200085B
:10C1D000ABD20008ABD20008ABD20008ABD200084B
:10C1E00025F50008E5250108EDAC0108F9FA01087C
:10C1F000E97B020879F003084D790508557F0508A9
:10C2000065FD0508CD5F060891670608C96A06083E
:10C2100035CB0608B1E90608E57F070895F0070861
:10C22000EDFD07081D9B0908DD9F0908696E0A08D6
:10C23000CDCF0A08E5F50A088D000B089D2C0B08E8
:10C2400065320B0800000000000000000000000044
:10C2500081F0004102E000BF83F0004330B54FEAB7
:10C2600041044FEA430594EA050F08BF90EA020F24
:10C270001FBF54EA000C55EA020C7FEA645C7FEAB7
:10C28000655C00F0E2804FEA5454D4EB5555B8BFDA
:10C290006D420CDD2C4480EA020281EA030382EA4B
:10C2A000000083EA010180EA020281EA0303362DDD
:10C2B00088BF30BD11F0004F4FEA01314FF4801CB0
:10C2C0004CEA113102D0404261EB410113F0004FC2
:10C2D0004FEA03334CEA133302D0524263EB430379
:10C2E00094EA050F00F0A780A4F10104D5F1200E17
:10C2F0000DDB02FA0EFC22FA05F2801841F1000172
:10C3000003FA0EF2801843FA05F359410EE0A5F145
:10C3100020050EF1200E012A03FA0EFC28BF4CF076
:10C32000020C43FA05F3C01851EBE37101F000452C
:10C3300007D54FF0000EDCF1000C7EEB00006EEB39
:10C340000101B1F5801F1BD3B1F5001F0CD34908C3
:10C350005FEA30004FEA3C0C04F101044FEA44521A
:10C3600012F5800F80F09A80BCF1004F08BF5FEAA1
:10C37000500C50F1000041EB045141EA050130BD81
:10C380005FEA4C0C404141EB0101013C28BFB1F593
:10C39000801FE9D291F0000F04BF01460020B1FADE
:10C3A00081F308BF2033A3F10B03B3F120020CDAB1
:10C3B0000C3208DD02F1140CC2F10C0201FA0CF08F
:10C3C00021FA02F10CE002F11402D8BFC2F1200CF4
:10C3D00001FA02F120FA0CFCDCBF41EA0C019040AA
:10C3E000E41AA2BF01EB0451294330BD6FEA0404F3
:10C3F0001F3C1CDA0C340EDC04F11404C4F12002DE
:10C4000020FA04F001FA02F340EA030021FA04F3EF
:10C4100045EA030130BDC4F10C04C4F1200220FA46
:10C4200002F001FA04F340EA0300294630BD21FA84
:10C4300004F0294630BD94F0000F83F4801306BF4A
:10C4400081F480110134013D4EE77FEA645C18BF3E
:10C450007FEA655C29D094EA050F08BF90EA020FD5
:10C4600005D054EA000C04BF1946104630BD91EACD
:10C47000030F1EBF0021002030BD5FEA545C05D1D0
:10C480004000494128BF41F0004130BD14F580040F
:10C490003CBF01F5801130BD01F0004545F0FE4183
:10C4A00041F470014FF0000030BD7FEA645C1ABFB8
:10C4B000194610467FEA655C1CBF0B46024650EAEF
:10C4C000013406BF52EA033591EA030F41F400211B
:10C4D00030BD00BF90F0000F04BF0021704730B5A1
:10C4E0004FF4806404F132044FF000054FF0000176
:10C4F00050E700BF90F0000F04BF0021704730B537
:10C500004FF4806404F1320410F0004548BF40420B
:10C510004FF000013EE700BF42004FEAE2014FEA60
:10C5200031014FEA02701FBF12F07F4393F07F4F3B
:10C5300081F06051704732F07F4208BF704793F03E
:10C540007F4F04BF41F40021704730B54FF4607451
:10C5500001F0004521F000411CE700BF50EA010254
:10C5600008BF704730B54FF000050AE050EA0102FD
:10C5700008BF704730B511F0004502D5404261EB6D
:10C5800041014FF4806404F132045FEA915C3FF4AE
:10C59000D8AE4FF003025FEADC0C18BF03325FEA4B
:10C5A000DC0C18BF033202EBDC02C2F1200300FAFC
:10C5B00003FC20FA02F001FA03FE40EA0E0021FA21
:10C5C00002F11444BDE600BF70B54FF0FF0C4CF40F
:10C5D000E06C1CEA11541DBF1CEA135594EA0C0FC1
:10C5E00095EA0C0F00F0DEF82C4481EA030621EAFC
:10C5F0004C5123EA4C5350EA013518BF52EA033537
:10C6000041F4801143F4801338D0A0FB02CE4FF0E8
:10C610000005E1FB02E506F00042E0FB03E54FF018
:10C620000006E1FB03569CF0000F18BF4EF0010E10
:10C63000A4F1FF04B6F5007F64F5407404D25FEA0C
:10C640004E0E6D4146EB060642EAC62141EA5551BF
:10C650004FEAC52040EA5E504FEACE2EB4F1FD0C01
:10C6600088BFBCF5E06F1ED8BEF1004F08BF5FEA7F
:10C67000500E50F1000041EB045170BD06F0004631
:10C6800046EA010140EA020081EA0301B4EB5C04DE
:10C69000C2BFD4EB0C0541EA045170BD41F48011D6
:10C6A0004FF0000E013C00F3AB8014F1360FDEBFFB
:10C6B000002001F0004170BDC4F10004203C35DAD7
:10C6C0000C341BDC04F11404C4F1200500FA05F35A
:10C6D00020FA04F001FA05F240EA020001F00042FB
:10C6E00021F0004110EBD37021FA04F642EB060171
:10C6F0005EEA430E08BF20EAD37070BDC4F10C049B
:10C70000C4F1200500FA04F320FA05F001FA04F25E
:10C7100040EA020001F0004110EBD37041F100014A
:10C720005EEA430E08BF20EAD37070BDC4F1200555
:10C7300000FA05F24EEA020E20FA04F301FA05F2BD
:10C7400043EA020321FA04F001F0004121FA04F265
:10C7500020EA020000EBD3705EEA430E08BF20EA35
:10C76000D37070BD94F0000F0FD101F0004640006F
:10C7700041EB010111F4801F08BF013CF7D041EAF1
:10C78000060195F0000F18BF704703F000465200F5
:10C7900043EB030313F4801F08BF013DF7D043EAC6
:10C7A0000603704794EA0C0F0CEA135518BF95EA7C
:10C7B0000C0F0CD050EA410618BF52EA4306D1D103
:10C7C00081EA030101F000414FF0000070BD50EA22
:10C7D000410606BF1046194652EA430619D094EAAC
:10C7E0000C0F02D150EA013613D195EA0C0F05D196
:10C7F00052EA03361CBF104619460AD181EA0301EA
:10C8000001F0004141F0FE4141F470014FF00000A1
:10C8100070BD41F0FE4141F4780170BD70B54FF03C
:10C82000FF0C4CF4E06C1CEA11541DBF1CEA1355BC
:10C8300094EA0C0F95EA0C0F00F0A7F8A4EB05049E
:10C8400081EA030E52EA03354FEA013100F0888095
:10C850004FEA03334FF0805545EA131343EA12635E
:10C860004FEA022245EA111545EA10654FEA002613
:10C870000EF000419D4208BF964244F1FD0404F5CC
:10C88000407402D25B084FEA3202B61A65EB030528
:10C890005B084FEA32024FF480104FF4002CB6EBE5
:10C8A000020E75EB030E22BFB61A754640EA0C0065
:10C8B0005B084FEA3202B6EB020E75EB030E22BFA5
:10C8C000B61A754640EA5C005B084FEA3202B6EBE6
:10C8D000020E75EB030E22BFB61A754640EA9C00A5
:10C8E0005B084FEA3202B6EB020E75EB030E22BF75
:10C8F000B61A754640EADC0055EA060E18D04FEA33
:10C90000051545EA16754FEA06164FEAC30343EAD2
:10C9100052734FEAC2025FEA1C1CC0D111F4801F9F
:10C920000BD141EA00014FF000004FF0004CB6E798
:10C9300011F4801F04BF01430020B4F1FD0C88BF37
:10C94000BCF5E06F3FF6AFAEB5EB030C04BFB6EB42
:10C95000020C5FEA500C50F1000041EB045170BD35
:10C960000EF0004E4EEA113114EB5C04C2BFD4EB62
:10C970000C0541EA045170BD41F480114FF0000EE6
:10C98000013C90E645EA060E8DE60CEA135594EA62
:10C990000C0F08BF95EA0C0F3FF43BAF94EA0C0F65
:10C9A0000AD150EA01347FF434AF95EA0C0F7FF4DA
:10C9B00025AF104619462CE795EA0C0F06D152EA2E
:10C9C00003353FF4FDAE1046194622E750EA410612
:10C9D00018BF52EA43067FF4C5AE50EA41047FF423
:10C9E0000DAF52EA43057FF4EBAE12E74FF0FF3C88
:10C9F00006E000BF4FF0010C02E000BF4FF0010C59
:10CA00004DF804CD4FEA410C7FEA6C5C4FEA430CD1
:10CA100018BF7FEA6C5C1BD001B050EA410C0CBF20
:10CA200052EA430C91EA030F02BF90EA020F002082
:10CA3000704710F1000F91EA030F58BF994208BFE9
:10CA400090422CBFD8176FEAE37040F001007047A6
:10CA50004FEA410C7FEA6C5C02D150EA013C07D1FD
:10CA60004FEA430C7FEA6C5CD6D152EA033CD3D048
:10CA70005DF8040B704700BF8446104662468C4642
:10CA80001946634600E000BF01B5FFF7B7FF002875
:10CA900048BF10F1000F01BD4DF808EDFFF7F4FF9E
:10CAA0000CBF012000205DF808FB00BF4DF808ED29
:10CAB000FFF7EAFF34BF012000205DF808FB00BF4C
:10CAC0004DF808EDFFF7E0FF94BF012000205DF86E
:10CAD00008FB00BF4DF808EDFFF7CEFF94BF012023
:10CAE00000205DF808FB00BF4DF808EDFFF7C4FF1C
:10CAF00034BF012000205DF808FB00BF4FEA410C65
:10CB00007FEA6C5C02D150EA013C0AD14FEA430C47
:10CB10007FEA6C5C02D152EA033C02D14FF0000084
:10CB200070474FF0010070474FEA410212F50012C2
:10CB300015D211D56FF47873B3EB625212D94FEA64
:10CB4000C12343F0004343EA505311F0004F23FA4E
:10CB500002F018BF404270474FF00000704750EAA3
:10CB6000013005D111F0004008BF6FF00040704760
:10CB70004FF00000704700BF4A0011D212F50012BA
:10CB800011D20DD56FF47873B3EB62520ED44FEA25
:10CB9000C12343F0004343EA505323FA02F07047A5
:10CBA0004FF00000704750EA013002D14FF0FF30E3
:10CBB00070474FF0000070474FEA4102B2F1E04386
:10CBC00024BFB3F5001CDCF1FE5C0DD901F0004C74
:10CBD0004FEAC0024CEA5070B2F1004F40EB8300C4
:10CBE00008BF20F00100704711F0804F21D113F1F0
:10CBF0003872BCBF01F00040704741F480114FEA29
:10CC00005252C2F11802C2F1200C10FA0CF320FAB1
:10CC100002F018BF40F001004FEAC1234FEAD323CE
:10CC200003FA0CFC40EA0C0023FA02F34FEA430338
:10CC3000CCE77FEA625307D150EA01331EBF4FF0C1
:10CC4000FE4040F44000704701F0004040F0FE40DC
:10CC500040F40000704700BF80F0004002E000BFD9
:10CC600081F0004142001FBF5FEA410392EA030FD7
:10CC70007FEA226C7FEA236C6AD04FEA1262D2EB21
:10CC80001363C1BFD218414048404140B8BF5B4226
:10CC9000192B88BF704710F0004F40F4000020F0BF
:10CCA0007F4018BF404211F0004F41F4000121F0D5
:10CCB0007F4118BF494292EA030F3FD0A2F101021F
:10CCC00041FA03FC10EB0C00C3F1200301FA03F15D
:10CCD00000F0004302D5494260EB4000B0F5000F80
:10CCE00013D3B0F1807F06D340084FEA310102F13F
:10CCF0000102FE2A51D2B1F1004F40EBC25008BFF1
:10CD000020F0010040EA03007047490040EB0000BA
:10CD1000013A28BFB0F5000FEDD2B0FA80FCACF1BB
:10CD2000080CB2EB0C0200FA0CF0AABF00EBC250E8
:10CD300052421843BCBFD0401843704792F0000FD6
:10CD400081F4000106BF80F400000132013BB5E729
:10CD50004FEA41037FEA226C18BF7FEA236C21D09F
:10CD600092EA030F04D092F0000F08BF0846704704
:10CD700090EA010F1CBF0020704712F07F4F04D1D2
:10CD8000400028BF40F00040704712F100723CBFE5
:10CD900000F50000704700F0004343F0FE4040F40F
:10CDA000000070477FEA226216BF08467FEA2363CD
:10CDB0000146420206BF5FEA412390EA010F40F4B8
:10CDC000800070474FF0000304E000BF10F0004304
:10CDD00048BF40425FEA000C08BF704743F09643EB
:10CDE00001464FF000001CE050EA010208BF704706
:10CDF0004FF000030AE000BF50EA010208BF70478D
:10CE000011F0004302D5404261EB41015FEA010CA1
:10CE100002BF84460146002043F0B64308BFA3F199
:10CE20008053A3F50003BCFA8CF2083AA3EBC2537B
:10CE300010DB01FA02FC634400FA02FCC2F120029A
:10CE4000BCF1004F20FA02F243EB020008BF20F0D1
:10CE50000100704702F1200201FA02FCC2F1200237
:10CE600050EA4C0021FA02F243EB020008BF20EA2C
:10CE7000DC7070477BB972B90029BEBF00204FF04B
:10CE8000004106E008BF00281CBF6FF000414FF0D2
:10CE9000FF3000F007BAADF1080C6DE904CE0029AF
:10CEA00009DB002B1ADB00F095F8DDF804E0DDE982
:10CEB000022304B07047404261EB4101002B1BDBB1
:10CEC00000F088F8DDF804E0DDE9022304B0404218
:10CED00061EB4101524263EB43037047524263EB03
:10CEE000430300F077F8DDF804E0DDE9022304B045
:10CEF000404261EB41017047524263EB430300F053
:10CF000069F8DDF804E0DDE9022304B0524263EB86
:10CF10004303704753B94AB9002908BF00281CBF12
:10CF20004FF0FF314FF0FF3000F0BCB9ADF1080C0D
:10CF30006DE904CE00F04EF8DDF804E0DDE90223EF
:10CF400004B07047430803F05533C01A830803F058
:10CF5000333300F03330184400EB101000F00F3082
:10CF600000EB002000EB0040000E704707EE900A37
:10CF7000F5EEC07AF1EE10FA01D400F00BB8F1EE44
:10CF8000677A08B517EE900A00F004F8404261EBAA
:10CF9000410108BDD0B5FFF7BFFA0C4B0022064691
:10CFA0000F46FFF711FBFFF7E7FD0446FFF792FA84
:10CFB000074B0022FFF708FB02460B463046394676
:10CFC000FFF74AF9FFF7D8FD2146D0BD0000F03D3C
:10CFD0000000F0412DE9F047089D04468E46002BE5
:10CFE0004DD18A42944669D9B2FA82F252B101FA1D
:10CFF00002F3C2F1200120FA01F10CFA02FC41EA2D
:10D00000030E94404FEA1C48210CBEFBF8F61FFAB1
:10D010008CF708FB16E341EA034306FB07F199424C
:10D020000AD91CEB030306F1FF3080F01F819942FF
:10D0300040F21C81023E63445B1AA4B2B3FBF8F0D9
:10D0400008FB103344EA034400FB07F7A7420AD960
:10D050001CEB040400F1FF3380F00A81A74240F288
:10D0600007816444023840EA0640E41B00261DB1F3
:10D07000D4400023C5E900433146BDE8F0878B4228
:10D0800009D9002D00F0EF800026C5E900013046E7
:10D090003146BDE8F087B3FA83F6002E4AD18B42C1
:10D0A00002D3824200F2F980841A61EB030301206B
:10D0B0009E46002DE0D0C5E9004EDDE702B9FFDE57
:10D0C000B2FA82F2002A40F09280A1EB0C014FEA02
:10D0D0001C471FFA8CFE0126200CB1FBF7F307FB5F
:10D0E000131140EA01410EFB03F0884208D91CEB02
:10D0F000010103F1FF3802D2884200F2CB8043469F
:10D10000091AA4B2B1FBF7F007FB101144EA01447D
:10D110000EFB00FEA64508D91CEB040400F1FF310C
:10D1200002D2A64500F2BB800846A4EB0E0440EAFA
:10D1300003409CE7C6F12007B34022FA07FC4CEA03
:10D14000030C20FA07F401FA06F31C43F9404FEAF6
:10D150001C4900FA06F3B1FBF9F8200C1FFA8CFE0B
:10D1600009FB181140EA014108FB0EF0884202FA5F
:10D1700006F20BD91CEB010108F1FF3A80F0888020
:10D18000884240F28580A8F102086144091AA4B2DD
:10D19000B1FBF9F009FB101144EA014100FB0EFE5E
:10D1A0008E4508D91CEB010100F1FF346CD28E458D
:10D1B0006AD90238614440EA0840A0FB0294A1EB1E
:10D1C0000E01A142C846A64656D353D05DB1B3EB7B
:10D1D000080261EB0E0101FA07F722FA06F3F140AB
:10D1E0001F43C5E9007100263146BDE8F087C2F152
:10D1F0002003D8400CFA02FC21FA03F391400143CA
:10D200004FEA1C471FFA8CFEB3FBF7F007FB103602
:10D210000B0C43EA064300FB0EF69E4204FA02F4AE
:10D2200008D91CEB030300F1FF382FD29E422DD901
:10D23000023863449B1B89B2B3FBF7F607FB163336
:10D2400041EA034106FB0EF38B4208D91CEB0101B6
:10D2500006F1FF3816D28B4214D9023E6144C91A36
:10D2600046EA004638E72E46284605E70646E3E646
:10D270001846F8E64B45A9D2B9EB020864EB0C0E50
:10D280000138A3E74646EAE7204694E74046D1E75F
:10D29000D0467BE7023B614432E7304609E764440D
:10D2A000023842E7704700BF02E000F000F8FEE7F6
:10D2B00072B6374880F30888364880F309883648C4
:10D2C0003649086040F20000CCF200004EF634719E
:10D2D000CEF200010860BFF34F8FBFF36F8F40F2B3
:10D2E0000000C0F2F0004EF68851CEF20001086056
:10D2F000BFF34F8FBFF36F8F4FF00000E1EE100AC6
:10D300004EF63C71CEF200010860062080F31488CE
:10D31000BFF36F8FAFF0E6FCAEF0BEFD4FF05530BF
:10D320001F491B4A91423CBF41F8040BFAE71D49D3
:10D33000184A91423CBF41F8040BFAE71A491B4ACC
:10D340001B4B9A423EBF51F8040B42F8040BF8E71E
:10D3500000201849184A91423CBF41F8040BFAE7F3
:10D36000AFF0C4FCAEF0ECFD144C154DAC4203DA4A
:10D3700054F8041B8847F9E702F0C4F8114C124D29
:10D38000AC4203DA54F8041B8847F9E7AFF0ACBCB1
:10D39000000600200022002000C0000808ED00E088
:10D3A0000000002000060020E0520E0800220020AD
:10D3B000CC2B0020D02B002060540120E0C10008BD
:10D3C00044C2000844C2000844C200082DE9F04FDE
:10D3D0002DED108AC1F80CD0C3689D46BDEC108AB3
:10D3E000BDE8F08F002383F311882846A047002072
:10D3F000AEF0D8FAFEE7AEF045F900DFFEE7000038
:10D4000001F0FF01102A2BDB10F0070F08D010F8F5
:10D41000013B013A8B422DD010F0070F42B3F6D1F9
:10D42000F0B441EA012141EA014122F007047FF012
:10D4300000070023F0E80256083C85EA010586EA69
:10D44000010685FA47F5A3FA87F586FA47F6A5FAA5
:10D4500087F68EB9EED1F0BC01F0FF0102F00702B1
:10D4600032B110F8013B013A83EA010313B1F8D15C
:10D470000020704701387047002D06BF354603383D
:10D48000073815F0010F07D1013015F4807F02BF76
:10D49000013015F4C03F0130F0BC0138704700BFC7
:10D4A00010F8012B11F8013B012A28BF9A42F7D04E
:10D4B000D01A7047034613F8012B002AFBD1181A23
:10D4C0000138704738B50022002304460D46FFF7A7
:10D4D000EDFA28B920462946BDE8384000F00AB8E0
:10D4E000204605F1004100F005F8404261EB4101A2
:10D4F00038BD00BFD0B50C4B002206460F46FFF7E3
:10D5000063F8FFF739FB0446FEF7E4FF074B002200
:10D51000FFF75AF802460B4630463946FEF79CFEA6
:10D52000FFF72AFB2146D0BD0000F03D0000F0418E
:10D53000036800221B6818477FB503914021054608
:10D540007CF01AFA039A18B90124204604B070BD81
:10D55000134E039296F9DA31002BF5D05FF020FDDF
:10D56000437A039A53B95FF01BFD847A039A2CB96E
:10D570000C4B402128467CF007FAE6E7D6F8283B1A
:10D58000B6F9DC11B3F906309942DDDD064B0093A4
:10D590004021064B28467CF0F7F90024D5E700BF70
:10D5A000D84B0020E8510C0807520C08F5510C0824
:10D5B000F0B50D469DB0202104467CF0DDF9002831
:10D5C00000F09D804F4E96F9DA31ABB1D6F8282B9A
:10D5D000B6F9DC31B2F90A1003F10A02914203DD17
:10D5E00040F28D32934207DC474B2A4620212046E9
:10D5F0007CF0CAF9002080E096F9C931022B05D1F0
:10D60000424B2A46202120467CF0BEF9B6F89C31D8
:10D61000A3F57A739BB241F6583293420DD83C4F32
:10D6200096ED827AD7F89039D3ED097AB4EEE77A9D
:10D63000F1EE10FA03DD374BD7E7374BD5E796ED20
:10D64000837AD3ED0B7AB4EEE77AF1EE10FAF2DCDE
:10D65000B6F9D631002B01DC304BC6E796F86822CC
:10D660000D2A06D80123934013F4215F01D02C4BDF
:10D67000BBE72C480EF00CFE012806D1D7F89C0918
:10D6800083F0DEF998B101281AD00021602204A8A5
:10D690000391B3F049FA2449D7F89809642303AAFF
:10D6A00082F0B6FD00BB03AB0093204B02E0204BA1
:10D6B0000093204B2A46202120467CF065F999E70B
:10D6C00096F83C3B73B11C4819214AF08DFE48B1D5
:10D6D0001948D6F8B46119214AF0ACFE8642D4DD6F
:10D6E000164BE5E7164BE3E71649D7F89009642394
:10D6F00003AA7FF04DFC0028D5D01DB0F0BD01205D
:10D70000FBE700BFD84B002010520C0823520C0836
:10D71000D86B00205B520C084B520C0875520C0859
:10D720008A520C08F485002004530C0808530C0896
:10D73000CF520C08AA520C08E8380020EE520C0810
:10D74000DF520C081A530C0807B5044884F0FAFCA1
:10D7500000F0010003B05DF804FB00BF4C75002031
:10D760002DE9F043474F0446D7F8EC0E0368A5B007
:10D770001B690D469847814614F01CFB002180462A
:10D7800060220CA80B91B3F0CFF964230BAA494691
:10D79000404613F011FE064648B93B4A0BAB2946FA
:10D7A00020467CF0F9FA304625B0BDE8F08307F159
:10D7B000A00068F095FEB9F1000F03D194F91E3076
:10D7C000012B0AD1314811F0FDFA80B9304A2946BF
:10D7D00020467CF0E1FA0026E5E710F0060FE2D0E3
:10D7E000A7F5005011F0EEFA08B92A4AEFE703A9AD
:10D7F000404613F017FC28B19DF80D305B0601D5AB
:10D80000254AE4E7D7ED7E7AF5EEC07AF1EE10FA1C
:10D810004FF00003C7DD089309930A930DF1200927
:10D8200007AB019305AA06AB04A9CDF800904046CA
:10D8300013F0D6FF48462EF017FCD7ED7E7AB4EEF3
:10D84000E70AF1EE10FA01DB144AC0E79DED057A14
:10D85000F4EEC77AF1EE10FA01D8114AB7E79DED60
:10D86000047AF4EEC77AF1EE10FA01D80D4AAEE769
:10D870009DED067AF4EEC77AF1EE10FA93D80A4AD3
:10D88000A5E700BFD84B002020530C08D82B002060
:10D8900029530C0840530C0866530C0874530C08A9
:10D8A00089530C089F530C08B5530C0808B5064B58
:10D8B00093F8053F9B0704D5044A7CF06DFA0020DD
:10D8C00008BD0120FCE700BFD84B0020CC530C085A
:10D8D00070B50C4C0546D4F8EC0E03685B690E4637
:10D8E000984710B10124204670BDA4F5005011F0F6
:10D8F0007BFA04460028F5D1034A314628467CF0DD
:10D900004BFAF0E7D84B0020DC530C082DE9F04629
:10D91000464ED6F8103F93F8CB509BB081468A46CE
:10D9200065B9434B1B68986A03685B6B984704466C
:10D9300040B9404A514648467CF02EFA28461BB072
:10D94000BDE8F0865FF02CFB202160F0E1FA58B1D1
:10D950005FF026FB1F2160F0DBFA88B3364A5146A0
:10D9600048467CF019FA002496F8E23E03F01403CE
:10D97000142B05D1314A514648467CF00DFA00245B
:10D98000514648467DF0C0F8002188424FF06002C1
:10D9900002A808BF0C460191B3F0C6F8D6F8100FE4
:10D9A000036801AA1B6864219847054680B9244A88
:10D9B00001AB514648467CF0EFF92C462546BDE7C1
:10D9C0005FF0EEFAA52160F0A3FA0028C6D1CBE7FC
:10D9D000002CF3D0D9F808303BB9D9F800305146C3
:10D9E0005B6B484698470446E8E751464846FFF7D0
:10D9F000DFFD514607464846FFF758FF3840C4B29E
:10DA000051464846FFF798FD514604404846FFF707
:10DA10005FFF5146044048467CF0E6F95146044019
:10DA200048467DF089F80440C8E700BFD84B002085
:10DA3000F8870020F0530C0807540C0821540C08F8
:10DA400039540C0808B5FFF761FF054A92F8E01E4B
:10DA500060F3041182F8E01E024A907108BD00BF15
:10DA6000D84B0020B5890020F7B505460F467BF05E
:10DA7000BFFF044678B1022128467BF07DFF0646B1
:10DA800048B1154884F05EFBC205C0F30723C0F31C
:10DA9000002403D53446204603B0F0BD9B07F9D5DA
:10DAA0000D4884F05DFB0D4B03F51463D3ED007A54
:10DAB000F8EEE77A30EE670ADFED097AB0EEC00AD9
:10DAC000B4EEE70AF1EE10FAE4DD064B3A46022125
:10DAD00028467BF059FFDEE74C750020D86B00200C
:10DAE0000000C84244540C08F8B504460F467CF0C8
:10DAF0001BFA1021054620467BF03EFF58B1204618
:10DB0000FFF722FE064630B9044B3A461021204664
:10DB10007BF03AFF35462846F8BD00BF58540C0844
:10DB200070B505460E467BF0CBFE044678B18021E9
:10DB300028467BF021FF50B1074B93F8653443B181
:10DB4000064B3246802128467BF01EFF00242046EB
:10DB500070BD0446FBE700BFD85B00206C540C0886
:10DB600038B50D4D0446D5F89C0982F069FF0128AF
:10DB700010D0D5F89C0982F063FF022804D020461B
:10DB8000BDE838407BF09EBE04480EF081FB0128C2
:10DB9000F5D138BD0020FCE7D86B0020F4850020CB
:10DBA000F0B5114C85B0D4F8203B0093D4F8243B59
:10DBB0000193D4F8283B02936A46D4F82C3B039394
:10DBC00006460F467CF052FF3946054630467BF04C
:10DBD00035FF94F8E03E284060F3C303C3F3C00070
:10DBE00084F8E03E05B0F0BDD84B00202DE9F843A5
:10DBF00006462648DFF8A480DFF8A4900F4668F0B8
:10DC00006FFC0446D8F8EC0E03681B69984705467C
:10DC100030B914F0060F03D1D8F8203F022B09D1F8
:10DC2000394630467BF0DCFF054618B9002489F8F8
:10DC300007400AE039463046FFF792FD04460028C7
:10DC4000F4D02DB9012389F807302046BDE8F883C8
:10DC5000082130467BF090FE0028F3D00C4821F0DC
:10DC60006BFF0028EED00B4B93F8E423B02101FBAF
:10DC70000233B3F8EE21B8F9CA319A42E2DD064B1D
:10DC80003A46082130467BF07FFECFE7784C0020F3
:10DC9000F82C0020D82B002080540C08D84B0020F2
:10DCA000B58900202DE9F3410F46054614F082F8AE
:10DCB000804613F079F9044640B94F4A01212846BD
:10DCC0007CF06AF8204602B0BDE8F0814B4ED6F8F1
:10DCD000EC0E036839469B699847044658B9D6F854
:10DCE000EC0E03681B6C9847454A03460121284601
:10DCF0007CF052F8E6E7AB68002BE3D01021284611
:10DD00007BF03AFE10B3D8ED937A98ED920A20EEAC
:10DD1000270AB0F0A7FCDFED3B7AB6F99C3120EE84
:10DD2000270ADFED397A20EE270A07EE903AF8EE5F
:10DD3000E77AB4EEE70AF1EE10FA07DD334B012281
:10DD4000102128467BF020FE0024BBE74021284616
:10DD50007BF012FE28B3012F1CD0232F1AD0042FE2
:10DD600018D0D6F8283B2A48B3F9083000EE103A0C
:10DD7000B8EEC00A00F0C0FBB5EEC00AF1EE10FA32
:10DD80001DDD244B00930122234B402128467BF0CC
:10DD9000FBFDD9E7D6F8EC0E0368DB6B984700284B
:10DDA000DFD01E4B1B68D86A0368DB6998470128DF
:10DDB000014619D11A4A28467BF0EEFFC4E7D6F88F
:10DDC000EC0E03685B69984730B1D6F8283BB3F98D
:10DDD0000830002BE5DDD4E7D6F8EC0E03681B68AD
:10DDE00098470B28DDD1F0E73946284602B0BDE858
:10DDF000F0417CF061BB00BF90540C08D84B002070
:10DE0000A1540C08E02E65420000C842B5540C082D
:10DE1000D82B002007520C08BD540C08F8870020AE
:10DE2000C9540C0870B505460E46FFF799FC084B1F
:10DE30000446D87131462846FFF74AFD314600288E
:10DE4000284608BF00247CF0EDFC204070BD00BFD8
:10DE5000B5890020F8B54E4F3B78002B40F09580F7
:10DE60004C4CD4F8105F95F8CB5001263E7015B19C
:10DE70003B702846F8BD7CF007FF054630B9464A9E
:10DE80003870137843F001031370F2E753F020FF6A
:10DE9000314652F009FFA4F5005006F0CFFC3F4B8D
:10DEA0001E710B2645F0EEFF013E45F089FF16F08E
:10DEB000FF06F7D13A4800F06BFF13F07BFFD0F874
:10DEC0000022C4F8382F90F87C32DA074BD413F0D4
:10DED000E9FA53F0FDFE3C2153F092FC04F6F8639E
:10DEE00000221A6000212E4800F0E6FF2C4810F0B6
:10DEF00069FF01462B4888F097F82B4B1B68D86ABE
:10DF0000036801211B689847D4F8100F03689B6AC7
:10DF100098470121D4F8100F85F0CEF853F0D8FEC1
:10DF20000646D4F8EC0E03681B68984794F85C2109
:10DF30000146304653F094F8194806F071FC4FF052
:10DF400021FE4FF05DF900233B708CF039FD174B3B
:10DF5000C3F8A809B4F8E23E23F4087343F02003A1
:10DF6000A4F8E23E85E79B07BCD431460C4804F098
:10DF700029FD0F4884F0F4F8DFED0E7A20EE270A31
:10DF800004F6F86383ED000AACE7002571E700BFF3
:10DF9000D02B0020D84B0020D4890020B589002048
:10DFA000D82B00209C550020F8870020D86B00203B
:10DFB0004C7500200AD7233C2DE9F043374DD5F8A6
:10DFC000103F93F8CB3087B0002B64D062B10129A9
:10DFD00001D0232908D195F9E03E002B04DB002471
:10DFE000204607B0BDE8F0837CF004FF044600281B
:10DFF000F5D013F0DFFE07461AF0D0FB8046384616
:10E0000012F0E4FCD8B198F92430022B17D1002685
:10E010004FF00009F1B203AA38460191CDF80C90F7
:10E02000CDF81090CDF8149013F062F8019918B162
:10E0300003AA40461AF062F80136032EEAD11848C6
:10E04000012106F063FE1648012106F095FD00212E
:10E05000D5F8100F85F030F8124830F005FD53F078
:10E0600037FE002152F020FE0F4B1B68D86A036870
:10E0700000211B68984795F8E23ED5F8EC1E0B4846
:10E080006FF3451385F8E23E0B1A594259413C3073
:10E090008AF02EFCA4E70124A2E700BFD84B0020A1
:10E0A000D82B002028800020F8870020C481002081
:10E0B00010B5064CD4F8EC0E03685B6A984718B1AB
:10E0C000D4F8103F93F8CB0010BD00BFD84B002010
:10E0D00030B52DED028B89B00C46B0EE408AFFF7CB
:10E0E000E7FF0546002838D0B4EE488AF1EE10FA72
:10E0F0007CBFDFED1C8ADFED1C7A226863689FED30
:10E100001A0A68BFDFED198A029278BF68EE288A82
:10E1100002A878BF68EEA78AD4ED027A0393F1EEE5
:10E12000677ACDED047A2DF0A1FBB4EE488A002287
:10E130000123F1EE10FACDE900238DED050ACDEDB6
:10E14000060A9FED0A0A0A488DED071AF0EE680AE2
:10E1500068BF134605A90CF07FF9284609B0BDEC4D
:10E16000028B30BDE02E65420000C8420000000076
:10E170009884002007B50191FFF79AFF30B101990B
:10E18000044803B05DF804EB00F0F6BA03B05DF8A4
:10E1900004FB00BFD82B0020014868F02DBB00BF56
:10E1A000784C002008B500F5005090F8E03EC3F32D
:10E1B00040128A420BD061F3451380F8E03E31B142
:10E1C00053F086FDBDE808400F2153F019BB08BD90
:10E1D00070B500F500560546D6F8203F8B420C4638
:10E1E00012D0012911D0022916D059B953F070FD6F
:10E1F0001B2153F005FB0D4A05F533500621043071
:10E2000056F0B0FDC6F8204F70BD53F061FD1A21E5
:10E2100053F0F6FA064AEFE7012100F04DFE53F005
:10E2200057FD1D2153F0ECFA024AE5E734550C087E
:10E2300049550C0844550C0810B500F500520C4621
:10E2400092F8053F03F00101A14209D064F30003F5
:10E2500082F8053FDB0704D405F0D8FE024B9C7220
:10E2600010BD06F0ABF8F9E7B589002000F50050C5
:10E2700090F8053F61F3410380F8053F014B1973A6
:10E28000704700BFB589002010B504465EF088FED7
:10E2900020215FF03DFE04F50053003893F8E22E94
:10E2A00018BF012060F3820283F8E22E10BD000047
:10E2B00010B504464FF066FC04F50052436FD2F8E7
:10E2C000102F04F58044D360D4F890299366D4F8D5
:10E2D0009829C2F8FC32D4F8900903685B6D98471E
:10E2E000D4F890090368BDE810409B6D1847000002
:10E2F00070B52DED028B00F500550446D5F8103FA2
:10E3000093F8CB30002B74D095F9E03E002B70DBF6
:10E3100000F5A04393F87433002B6AD1D5F8EC0EC6
:10E3200003685B699847002863D1334BD3F8EC0E40
:10E3300003681B6898470B285BD004F580469FED67
:10E340002F7AD6F89839D3EDDB7AF0EEE77AF4EE4F
:10E35000C77AF1EE10FA4CD5D5F8100F443056F0CC
:10E3600073F90346DFED260A93ED000A9F20B7EE0E
:10E37000001A2AF08FF8B5EEC00AF1EE10FA38DD77
:10E3800004F59240743083F0F7FEDFED1E7AB0EEB4
:10E39000C00AB4EEE70AF1EE10FA2AD504F580546B
:10E3A000D6F89009D4F8B83407EE903A0368D3F859
:10E3B0009830B8EEE78A984738EE400ADFED127AD7
:10E3C000B0EEC00AB4EEE70AF1EE10FA11D5D4F8B7
:10E3D000BC3440F2E63203F2F313934209D8BDECA9
:10E3E000028BD5F8100F9FED090ABDE8704086F04A
:10E3F0004DB9BDEC028B70BDD84B0020000000343D
:10E4000000000000000070420000FA430AD7233CDD
:10E4100008B500F50050D0F8100F03681B69984745
:10E42000F6EE007A20EE270AB5EEC00AF1EE10FAF9
:10E4300048BF9FED010A08BD0000000038B52DED72
:10E44000028B00F580450446D5F89039DFED110ABE
:10E4500093ED370A04F500547120B7EE001A2AF044
:10E4600019F8D4F8100FD5F8985903681B69B0EE65
:10E47000408A984738EE400ABDEC028BDFED067A01
:10E4800005F50575284620EE270ABDE8384073F0EB
:10E4900079BB00BF0000000000007A4400F5805006
:10E4A00000F5A26300F21C50D3ED005AD2ED007AC1
:10E4B000D0ED006A91ED006A26EEE77A67EEA57A64
:10E4C000A6EE257AE6EE267A81ED007AC2ED007A94
:10E4D0007047000000F50050B0F9743A33B9B0F954
:10E4E000D6010028B8BF404280B2704783EAE3708B
:10E4F000A0EBE370F8E7000070B52DED028B00F59E
:10E50000005482B094F8051F11F00106054605D0AD
:10E510009FED2D0A02B0BDEC028B70BD8DED010A9E
:10E520005EF03EFD037F002BF2D0DFED288ADFEDA9
:10E53000260A9DED010AB0EE681A4E2029F0AAFFC6
:10E540004FF4C8723146B4F9DE01B0EE408A29F0CA
:10E55000DFFFA4F8DE01284610F0E4F9B4F9DE315B
:10E5600007EE900AB8EEE77A07EE903AF8EEE77A0F
:10E5700077EE676AB4EEE68AF1EE10FA0DD528461A
:10E58000FFF7A8FF07EE900A38EE668AB8EEE70AB2
:10E5900020EE088A88EE260ABCE777EE877AB4EE8A
:10E5A000E78AF1EE10FAB3DDB4F9D63100EE103A95
:10E5B00038EE678AB8EEC00A78EEE77A20EE088A6D
:10E5C00088EE270AA6E700BF0000000000007A449A
:10E5D00000207047002070477047000000F507508A
:10E5E0002C30704700487047F8840C0800F5005044
:10E5F000D0F8EC0E03681B68184700000348086059
:10E600003021117008221A60704700BFF4580C08BE
:10E6100000F50050D0F8EC0E0368DB6C18470000E2
:10E6200000F50050D0F8EC0E03689B6C1847000012
:10E6300000F5005300F5A840D3F8EC3E14301B1A47
:10E64000584258417047000010B500F500500C4684
:10E65000D0F8EC0E0368DB6D984707EE900A9FED4B
:10E66000057AF8EE677A012067EE877AC4ED007AC2
:10E6700010BD00BF0AD7233C10B500F500500C4672
:10E68000D0F8EC0E03689B6D984707EE900A9FED5B
:10E69000057AF8EEE77A012067EE877AC4ED007A12
:10E6A00010BD00BF0AD7233C10B500F500500C4642
:10E6B000D0F8EC0E03681B6E9847DFED047A20EE6D
:10E6C000270A012084ED000A10BD00BF0AD7233CB1
:10E6D00061F098B811F082BA65F06EB860F038BC9D
:10E6E0004FF09AB927F010BE52F060BC17F0E2B8B4
:10E6F0005EF0A8B85CF062BA0FF0C0BD10F008BAC6
:10E7000006F03CBD11F000BA05F0D6BC05F02ABAFF
:10E7100005F050B962F02ABE0EF056BCFFF7E8BD16
:10E720000FF0E4BE10F04CB903F0CCB80FF06CBEA3
:10E730000FF0EABD5EF082BB22F09CBC06F0EAB8A6
:10E7400002F09ABC10F05AB906F0CEBC04F026B91B
:10E7500006F028BE05F0C0B906F08AB90FF01ABD60
:10E76000FFF7A6BD28F0EEB805F0A6BE09F0D4BEAE
:10E7700009F0CEBD09F062BD1FB500F50053044697
:10E78000D3F8EC0E039103685B6A984760B1DFED44
:10E79000070A0399002304F5B1400093B0EE600A24
:10E7A0001A4640300BF0AEFC04B010BD0000000073
:10E7B00010B52DED028B00F500530446D3F8EC0E96
:10E7C00003685B6AB0EE408A984720B90024BDEC2C
:10E7D000028B204610BD9FED080A04F5B14028EEDB
:10E7E000000A40300AF058FF04460028EED00348E3
:10E7F0000121FFF7D7FCEAE70000C842D82B002030
:10E800000A4A92F9E02E002A0B4605DA00228A60B5
:10E810004A600A600120704700F58040D0F89029D6
:10E82000783207CA83E80700F4E700BFD84B00201E
:10E8300070B51F4B036000F500530446D3F8740E07
:10E840001C4AC3F8C42C08B119F0E0F91A4B236034
:10E8500004F5805393F8842E42B9D3F8805E2DB12D
:10E86000284626F0A1FB284619F0CCF904F58E5075
:10E870000C307AF0B5FB04F58650143060F09CFD46
:10E8800004F6C44504F66446B54204D0183D284653
:10E8900025F0DEFFF8E7094BC4F8983804F6941029
:10E8A00055F0AEFB04F5106055F0AAFB204670BD94
:10E8B000C45C0C0820660D0828440D08480A0D08A1
:10E8C00038B5474B044640F8043B61F0BBF804F10F
:10E8D000100016F06FFC04F168004EF02BFE04F5FA
:10E8E000907021F051F804F5866015F0C1FA04F239
:10E8F000545019F08DF904F6980027F0B9FB04F58F
:10E90000446060F07DFE04F5516049F093FC04F52D
:10E910007C6052F019F904F58650143060F034FD33
:10E9200004F58850103017F063FF04F58E500C305A
:10E930007AF042FB04F58F5008304FF0BDF904F532
:10E9400091501C3062F05CFA04F5805304F5935248
:10E950000025104683F86052224B10301A6045F0B3
:10E960009DF8294604F5965011F020FD04F5C85095
:10E97000103073F0C5F904F5E850143077F062FBFD
:10E9800004F5F1500C3079F071FC04F5F4501030BE
:10E990007AF0A6F804F5F750083011F009FB04F5F9
:10E9A0000150083073F062FE04F50250203067F029
:10E9B0003BFC04F5005304F5055083F85C510A4D07
:10E9C00034307AF0CDFE2B6813B108488BF0C6FFC7
:10E9D0002046074948F016FA2C60204638BD00BF93
:10E9E00028440D0830930020948A002058550C08C4
:10E9F00050430D0810B50FF00DFF5EF0D1FA03681B
:10EA0000BDE810405B681847FFF7F4BF10B5044637
:10EA100006F0CAF8204610F0FDF9204603F010FE7B
:10EA20002046BDE8104003F073BF0000FFF7EEBFC3
:10EA300070B500F53C553C350446284616F094FA6E
:10EA400019F0ACFE90F9213093B390F840337BB3CA
:10EA500004F5005304F25456D3F8100F443055F027
:10EA6000F3FD0346DFED130A93ED000A9F20B7EE96
:10EA7000001A29F00FFD94F98835012B284608BFAC
:10EA800086ED0E0A002116F035F8DFED0B7A04F260
:10EA9000AC7494ED287A20EE270ADFED087AA7EE11
:10EAA000270A304684ED280ABDE8704019F086BD7B
:10EAB00070BD00BF00000000CDCCCC3D6666663F57
:10EAC000FFF7B6BF10B50121044610F0DFF960B1C1
:10EAD000114BD3F8EC0E03689B6A984728B920467F
:10EAE00002F0D8F9204602F0E5F94FF40011204673
:10EAF00010F0CCF918B128F09FFF27F0CDF94FF4B2
:10EB00008021204610F0C2F928B128F095FFBDE819
:10EB1000104027F0CFB810BDD84B0020FFF7D2BF70
:10EB200070B500F580450446D5F890099FED540A6C
:10EB300086B06C302CF09AFE03A904F596508DED4A
:10EB4000030ACDED040A8DED051A11F0DBFA02215E
:10EB5000204610F09BF970B10121204610F096F983
:10EB600048B9484BD3F8EC0E03689B6A984710B934
:10EB7000204602F08FF90121204610F087F948B9AC
:10EB8000404BD3F8EC0E03689B6A984710B92046B7
:10EB900002F090F90121204610F078F910B92046D2
:10EBA00002F0E0F94FF40031204610F06FF930B177
:10EBB00004F50053D3F8100F03685B6C98474021AD
:10EBC000204610F063F960B104F57C60019051F0CB
:10EBD00081FB04F58053019893F9D4300BB151F0C7
:10EBE000BBFC4FF48061204610F050F918B104F5D9
:10EBF0007C6051F009FC2021204610F047F958B103
:10EC000004F50056D6F8EC0E03681B699847C0B1AE
:10EC1000D5F8980980F038FA8021204610F036F9AE
:10EC2000E0B128F009FF27F069F81021204610F024
:10EC30002DF910B3D5F8900906B0BDE870407CF00E
:10EC400069BF20460CF016F90028E1D1D6F8EC0E89
:10EC500003685B6998470028DAD0DDE74FF480212C
:10EC6000204610F013F90028DBD14FF40021204694
:10EC700010F00CF90028D4D1D7E706B070BD00BF62
:10EC8000E02E6542D84B0020FFF74ABF10B50121A6
:10EC9000044610F0FBF810B1204602F063F9802121
:10ECA000204610F0F3F858B14FF48021204610F0C0
:10ECB000EDF828B928F0C0FEBDE8104026F0FABFF4
:10ECC00010BD0000FFF7E2BF10B5044605F0C2FC1E
:10ECD000204605F025FB204605F000FD204610F0FB
:10ECE000A1FF2046BDE8104003F086BCFFF7ECBF53
:10ECF00070B54FF6FF71044610F0C8F804F50055E2
:10ED000028B1D5F8E02E0721204602F05BF9D5F8AE
:10ED1000103F93F8CB307BB92046FFF7B5FAD5F812
:10ED2000100F95F8F221036895F868121B6A98474E
:10ED3000D5F8100F85F076FC5FF034FE5FF0C0FB75
:10ED4000204610F061FF95F8E03E0F4A04F580443C
:10ED5000DB43D4F89059C3F3C01353712B681E6F73
:10ED60004EF010FF4EF078FB2846B047D4F8984993
:10ED70004EF008FF04F505744EF06EFB2046BDE82A
:10ED8000704072F065BD00BFB5890020FFF7B0BFCD
:10ED90002DE9F04100F5805600F5005406F5A26318
:10EDA00004F624781B68C8F8003006F21C5304F6F9
:10EDB00028771B683B600546D6F8C00400F58C40F8
:10EDC000503029F03BFB04F57363C4F82C0FD8F8DE
:10EDD00000201A6004F634743B6823604FF6FF711C
:10EDE000284610F053F838B1D6F8C0242846092137
:10EDF000BDE8F04102F0BEB8BDE8F08110B500F505
:10EE00000053D3F8204F002C55D093F8E12ED107B2
:10EE100051D56FF3000283F8E12ED3F8242BD3F8F9
:10EE2000201BB2F90820012C06EE902AB1F9084007
:10EE30000BBF03F6247203F57362D2ED007AD2EDB4
:10EE4000007A0CBF03F6287203F63472D2ED005A32
:10EE50000CBFF8EEE66AF8EEE66A07EE104A25EE19
:10EE6000E66AB8EEC77A00F58050A7EE276A00F58B
:10EE7000A26200F21C5067EEA67AD2ED006AE7EEBD
:10EE8000257A90ED007A27EE877AA6EE267ABDEEF7
:10EE9000C77A17EE104A0C8192ED007AD3F8243B22
:10EEA00067EE877A90ED007AE6EE477AFDEEE77A34
:10EEB00017EE902A1A8110BD38B505462DED028B4C
:10EEC00000F5005471B128460FF032FBD4F82C3F06
:10EED0001B1A03F2F31340F2E63293420CD8BDEC56
:10EEE000028B38BDD4F8203F022BF8D10FF002FB83
:10EEF000B0F57A7FE7D2F2E7C4F82C0F00F58C402A
:10EF00005030642390FBF3F308EE103ADFED0B7AF8
:10EF1000B8EEC88A28EE278AB0EE480AAFF0E8F9C2
:10EF200004F5736383ED000AB0EE480AAFF036FBD8
:10EF300004F6347484ED000AD1E700BF35FA8E3C44
:10EF4000012100F5965012F0A7BE0000FFF7F8BFB0
:10EF500010B504460FF0ECFC102120460FF096FF90
:10EF600070B1204601F0E4FE4FF4001120460FF08E
:10EF70008DFF28B928F060FDBDE8104026F08CBF59
:10EF800010BD0000FFF7E4BFF8B50446254606F0C3
:10EF900031F9224B45F83C3B214BA465C4E91734B9
:10EFA000204BC4E91934204BE36604F1800018F0CB
:10EFB0006BFA04F19C0018F067FA04F1B80018F03D
:10EFC00063FA4FF6FF76194BC4F8CC30A4F8D06042
:10EFD00004F1D40018F058FA4FF0FF37144B1549DC
:10EFE000C4F8307128461D6047F00CFFA4F8787013
:10EFF000A4F8946004F5A27018F046FA04F5B07015
:10F0000018F042FA04F5BE7018F03EFA002384F8B6
:10F010009031C4F8B4312046F8BD00BF7CB00C0874
:10F020006DE7000871E7000875E700080000FFFFC2
:10F030008489002008180D0810B5044606F0DAF897
:10F040000A4B23600123A38704F1400018F01CFA47
:10F0500004F1500018F018FA04F1600018F014FAE6
:10F0600004F1700018F010FA204610BD24B80C0806
:10F070002DE9F043044689B0FFF722FCA34B23603F
:10F0800004F50850143004F5005502F0CBF804F5EF
:10F090000753203304F52C57C5F8343B062385F875
:10F0A000383B4FF07C5805A907F14400CDF8148097
:10F0B00055F02CFB07F15C008AF0BEFB04F592468C
:10F0C0000023743604F52E5785F8743B192304A9E0
:10F0D00085F8803BC5F87C6B07F10C00CDF81080FB
:10F0E00055F014FB07F124008AF0A6FB4FF001084D
:10F0F000182304F52F5004F5315785F8C83B043721
:10F1000085F8BC8BC5F8C46B1C305FF04FFD3846EA
:10F110007AF0E2FB06AE7E4BC5F8443C3146381D22
:10F120008DF8188048F08CFC04F531503C307AF0B2
:10F13000BDFB784B784FC5F87C3C04F53250314626
:10F140001430069755F0E2FA04F53250314620307B
:10F15000069755F0DBFA04F5325031462C3004F5B1
:10F160003358069708F1040855F0D0FA6B4BC5F8F0
:10F17000C43C08F108008AF05FFB04F5335704F53E
:10F180003559303709F114093846143759F02AFF38
:10F190004F45F9D10723C5F8783E0023A5F87C3EFA
:10F1A0004FF4CB7018F02CFDC5F8740E04F53A50EE
:10F1B0008AF042FB04F53B5004308AF03DFB584B8B
:10F1C0001A680AB9C3F8008004F5B547554BC5F86D
:10F1D000C43C283704F53B50C5F8EC7E30307BF05A
:10F1E00029FE05F624734FF07E58C3F8008005F51C
:10F1F00073654D4B07934D4BC5F800800694009303
:10F2000004F53C5096E80C004FF400713C3015F0CA
:10F2100039FB04F5515028306AF092FF04F5924012
:10F2200003A94430CDF80C8055F096FA04F59240CD
:10F2300003A95830CDF80C8055F068FA04F59240D7
:10F2400004F58045643018F01FF905F674130026A4
:10F250001E605E609E6004F5934304F593401E605B
:10F260005E609E6004F59653C5F88C39002385F8DE
:10F27000AD394FF40041303016F0A2F804F5944057
:10F28000303069F0EBF804F594406C3048F00EFD36
:10F29000274BC5F86C3A274B274904F5954004F5F0
:10F2A0009548186008F1200847F0ACFDFF2385F869
:10F2B000B03A85F8B83A2149404647F0A3FD204BC3
:10F2C0001D6815B11F488BF049FB04F5954040308F
:10F2D000C3F800804FF0C0FD1B4B1C48186004F5BC
:10F2E000A64264322B464FF0140C9DB20CFB050174
:10F2F0000133097C0029F8D1154B1D80154BD3F83B
:10F300000080B8F1000F29D01348DCE7C45C0C087A
:10F31000E0540C0820550C080000A04020660D08A1
:10F32000B08D0020445D0C0869E70008B45C0C084F
:10F3300030550C0834930020A4720D0830CF0D080E
:10F34000C49300206C550C08508A0020F89E0C08CD
:10F350004E8A00200C8A00208D550C0804F5A6402A
:10F360001A6003A9564B0393783055F0CFF904F592
:10F37000A74004F5A045183005F03CFF514BC5F8F7
:10F38000983304F5A740583005F034FF04F5AB4935
:10F390004D4BC5F8D83304F5A84009F16C09143079
:10F3A000FFF7F2FD484605F025FF484BC5F8EC3560
:10F3B00009F13C0087F024FF454BC5F8283604F5D9
:10F3C000AF402C3005F016FF424BC5F8AC3704F5C2
:10F3D000AF40703005F00EFF3F4BC5F8F03704F535
:10F3E000B04085F82C88303005F004FF3B4BC5F861
:10F3F000303804F5B0406C3005F0FCFE384BC5F8F1
:10F400006C3805F6A80304F5B1401E605E609E608E
:10F41000403005F0EFFE334BC5F8C03804F5B2407C
:10F42000C5F8FC88043005F0E5FE2F4BC5F804391B
:10F4300004F5B2404C3005F0DDFE2C4BC5F84C39DC
:10F4400004F5B340083005F0D5FE294BC5F88839DE
:10F4500004F5B44318461E605E601C30FFF7ECFDF7
:10F46000384605F0C7FE234BC5F8A83A04F5B54069
:10F47000643005F0BFFE204BA5F8208B04F5B640A4
:10F48000C5F8E43A3430FFF7D7FD1C4BC5F8343BE0
:10F49000012385F8BD3B05F6C43304F5B7401E6073
:10F4A0005E609E60503005F0A5FE154BC5F8D03B60
:10F4B00005F5416520462E606E6009B0BDE8F08319
:10F4C000CDCC4C3D78AD0C081CAE0C0820B10C081E
:10F4D000B0B10C086CB20C080CB30C08ACB30C083F
:10F4E00044B40C08E4B40C0874B50C080CB60C0851
:10F4F000ACB60C0880B90C081CBB0C08DCB80C08B6
:10F50000E0BB0C0838B5054B1C6823680A461D682B
:10F51000034B01462046A847002038BDF88700204D
:10F52000D82B002010B58AF055FD064C064B18600C
:10F530002046FFF79DFD2046044A0549BDE81040DE
:10F54000AEF0B0BDD82B0020F887002058EB00208B
:10F5500031E800080120704790F890308B4286BF58
:10F5600000EB8100D0F894000020704790F89030B4
:10F570008B4286BF00EB8100D0F8940000207047DA
:10F58000FA207047014B93F8A2017047D84B002036
:10F59000034BD3F8200F431E58425841704700BF19
:10F5A000D84B0020034BD3F8200F831E58425841FC
:10F5B000704700BFD84B0020034BD3F8100F08B1A1
:10F5C00083F072BE01487047D84B0020305D0C08B4
:10F5D00070B5036A374D43F4E0520262426A42F466
:10F5E000E0524262826A42F4E0528262D5F898297F
:10F5F0000446E2B143F4F8430362D5F898097FF07A
:10F6000003F938B1636A43F480436362A36A43F445
:10F610008043A362D5F898097FF018FA38B1636A7D
:10F6200043F400536362A36A43F40053A362224B82
:10F630001D6845B11921284648F0D6FE18B1236A45
:10F6400043F4807323621D4E96F83C3B6BB1636AB2
:10F6500043F48073636245B11921284648F0FCFEEB
:10F6600018B1A36A43F48073A362154B93F858331F
:10F67000013B012B0BD8D4E9082343F480036362D8
:10F68000A36A42F4800243F480032262A362236AE5
:10F6900043F080432362636A43F080436362D6F899
:10F6A000103F93F8C1301BB9A36A43F08043A362B3
:10F6B00070BD00BFD86B00205C8A0020D84B0020B2
:10F6C000D87B002013B54FF44470CDE9002118F029
:10F6D00091FA044628B1DDE900215CF0BDF9024B46
:10F6E0002360204602B010BD885F0C0800207047E0
:10F6F000704700000320704708207047014B93F8C3
:10F70000A4017047D84B0020034B93F95C020038EA
:10F7100018BF0120704700BFD84B0020014B93F960
:10F72000A6017047D84B00207047000070470000CA
:10F7300008B50C4BD3F8980970B910230A4AD2F8CF
:10F74000102F43F0400022B192F8CB200AB143F0D1
:10F75000C00040F0010008BD7FF056F80028ECD052
:10F760001823EBE7D86B0020D84B002038B5C578BC
:10F770000B46352D044628BF352535220021184675
:10F78000B1F0D2F92A4604F10C01BDE83840B1F0DD
:10F7900081B900001FB5184C94F83610A4F58C7090
:10F7A00010F0F2FB78B194F83610A4F58C7010F0DC
:10F7B000EDFB40B194F83610A4F58C7004B0BDE8B0
:10F7C000104010F0E5BB002301930293039312F065
:10F7D000F1FA01A912F0C8F820B101A82CF044FCFC
:10F7E00004B010BD21F084FC90F8C432B02202FBBA
:10F7F000030090ED2F0AF3E7D84B002008B50D4B1E
:10F80000D3F8100FA8B1443054F01EFF034693ED17
:10F81000000ADFED090A9F20B7EE001A28F03AFE31
:10F82000DFED067A20EE270ABDEEC00A10EE103A90
:10F8300018B208BDD84B0020000000000000C842EC
:10F840002DE9F04FDFF8D880344F8DB00446042501
:10F8500008F5005617F8019BB8F9FC3109F1FF3A99
:10F8600043FA0AF3D90742D5207C56F009FA8346B9
:10F87000207C57F009F900F121039B4505D2207C3B
:10F880000DB0BDE8F04F55F077BCBAF1030F2ED89C
:10F89000DFE80AF00234393ED6F8900903689B6825
:10F8A000984700F194035A69D3F800A0D3F804E014
:10F8B000D8681969D3F818C008925A6A1B6ACDF83B
:10F8C0002520CDF8293062222123CDE9003206908F
:10F8D0000791207CCDF80CA0192303AAC221CDF8F2
:10F8E00010E0CDF814C08DF8249056F033FA013DA5
:10F8F00015F0FF05AED10DB0BDE8F08FD6F8900938
:10F900000368DB68CCE7D6F8900903681B69C7E792
:10F91000D6F8983903F52A73C5E700BF54600C0880
:10F92000D84B002013B504460748019108F038FC75
:10F9300030B90199204602B0BDE8104057F0C8BA6E
:10F94000042002B010BD00BFEC7F0020014808F089
:10F9500081BA00BFEC7F00205AF0DEBF10B588B03E
:10F96000044658F041FC0C4BD3F8100F38B90B4A41
:10F970000621204608B0BDE8104058F01DBC69467D
:10F980001E2283F095FC064A6B460621204658F05D
:10F9900013FC08B010BD00BFD84B00207C5D0C08E4
:10F9A000EEAA0C08034A92F81C3B013382F81C3B78
:10F9B00057F01EBDD84B002007B50846019117F03F
:10F9C0006BFE38B10448019902F0C8FC002003B076
:10F9D0005DF804FB0420FAE704880020162A10B41E
:10F9E0000C4605D0542A03D05DF8044B57F08EBA6C
:10F9F0000323237001205DF8044B704710B5074BBB
:10FA000093F9C02A40F6CD3440F6CD13002A08BF42
:10FA10001C4657F021FC204310BD00BFD86B0020CE
:10FA200010B5044618F0EEF8204610BD10B50C4C89
:10FA300094F9E03E002B0FDBD4F8EC0E0368DB6C8E
:10FA4000984758B9D4F8EC0E03689B6C9847002887
:10FA50000CBF0220032010BD0120FCE70420FAE7C0
:10FA6000D84B002010B44C69012C05D101465DF83B
:10FA7000044B034802F0ECBF5DF8044B57F0D2BCD6
:10FA8000D82B00202DE9F341B1F90430002B0646B4
:10FA90000C46154635DB4FF00008CDE900281A4F1B
:10FAA000B1F902209FED190AD7F8201B4FF47A73A1
:10FAB0005BF00CFA0123CDE900539FED140AB4F971
:10FAC0000020D7F8241B4FF47A7330465BF0FEF920
:10FAD0009FED0F0AB4F90420D7F8281B434630469F
:10FAE000CDE900585BF0F2F9CDE900589FED070A27
:10FAF000B4F90620D7F82C1B4FF47A7330465BF02C
:10FB0000E5F902B0BDE8F081D84B00200000FA44CE
:10FB100000007A44044B187820B9044B93F8E20EA5
:10FB2000C0F38010704700BF54890020D84B0020DC
:10FB30000C4B93F865248AB9A3F5805213F8FB3C6B
:10FB40009B060BD192F9E03E002B09DB92F8E13ED7
:10FB500013F0200F14BF04200120704705207047C8
:10FB600003207047D85B002008B5074B93F9F031AC
:10FB7000032B03D0BDE8084058F096BB034A02218E
:10FB800058F01AFB042008BDD84B0020945D0C08E7
:10FB9000094BD3F86022920701D457F0A9B903F5B5
:10FBA000005303F6681393ED000ADFED047AB8EE14
:10FBB000C00A20EE270A7047D84B00200AD7233C02
:10FBC00010B594B0044603A817F05EFC1C4BD3F8A4
:10FBD000EC0E036803A95B6D984778B3002103A876
:10FBE00017F01CFD50B3247C8AF0EAFE059BDDED86
:10FBF000047A0893069B09930023F8EEE77A9FEDB9
:10FC0000117A0B930C930D930E930F931093119302
:10FC100012934FF6F853ADF84C300023962267EE5E
:10FC2000877A8DF84E303323CDE90032079007AA4A
:10FC300057212046CDED0A7A56F08CF814B010BD4D
:10FC4000D84B00200AD7233C30B52DED0A8B774CDA
:10FC50000546D4F8EC0E036899B05B6A9847002813
:10FC60005BD004F54054D4F8FC38062B00F2C98070
:10FC7000DFE803F00404045788AB53006C489FEDA1
:10FC80006D8A0AF007FC9FED6C0A01684268836880
:10FC90000D930BA80B910C922BF0E8FDF0EE489A17
:10FCA000B0EE40CAF0EE60BAB0EE419AB0EE48AAAB
:10FCB000F0EE488AF0EE48AAB0EE48BA40F6F854A2
:10FCC0002D7C8AF07DFE00231593169301238C2250
:10FCD0008DF85E303323CDE900320B90B1EE499AB6
:10FCE000F1EE688AB1EE488A0BAA552128468DEDBF
:10FCF0000CCACDED0DBA8DED0E9A8DED0FBACDED8E
:10FD000010AACDED118A8DED12AACDED139A8DEDCD
:10FD1000148AADF85C4056F01DF819B0BDEC0A8BA2
:10FD200030BD43480AF0B6FB9FED430A01684268C4
:10FD300083680D930BA80B910C922BF097FD3C4818
:10FD4000F0EE60BAB0EE419AB0EE40CA0AF0A6FBFF
:10FD50009FED390A2BF08AFD3548B0EE40BAF0EE3F
:10FD600060AAF0EE418A0AF09DFB9FED330A2BF06A
:10FD70007DFD4FF44064B0EE40AAF0EE609AB0EE24
:10FD8000418A9DE72A489FED2B9A0AF087FB9FED59
:10FD90002A0A2BF06BFD2648B0EE40BAF0EE60AABE
:10FDA000F0EE418A0AF07EFB9FED230A2BF05EFD08
:10FDB000F0EE49BAB0EE40AAF0EE609AB0EE418A99
:10FDC000B0EE49CA40F607447AE71948DFED198AD0
:10FDD0000AF068FB9FED180A2BF048FDF0EE68AAC8
:10FDE000B0EE40AAF0EE609AB0EE418AB0EE68BA8A
:10FDF000B0EE689AF0EE68BAB0EE68CA40F63F44DA
:10FE00005EE79FED0C8A0024F0EE489AB0EE48AA17
:10FE1000F0EE488AF0EE48AAB0EE48BAB0EE489A42
:10FE2000F0EE48BAB0EE48CA4AE700BFD84B00200F
:10FE300098840020000000000AD7233C2DE9F041FF
:10FE40002DED068B3B4D95F8E13E99068CB00446AE
:10FE50006AD505F500579FED380AD7F89009DFED10
:10FE6000378A6C302BF002FD8DED041A21EE281A32
:10FE7000D5F8EC6E8DED020ABDEEC11ACDED030A88
:10FE800011EE103A1DB2336894F810809B6D304625
:10FE900060EE289A20EEA89A984707EE900AF8EEAE
:10FEA000E77A304667EEA87AFDEEE77A17EE903AE9
:10FEB0001CB23368DB6D984707EE900AB8EE678A8C
:10FEC000D7F89839DFED1E7A93ED0FAA336828EE44
:10FED000288A1B6EB4EEE78AF1EE10FA58BFB0EE36
:10FEE000678A30469847BCEEC88A0023089318EE0C
:10FEF000103AB7222AEE28AA20EE280AADF82C30B4
:10FF00001A23CDE900323E2105AA4046CDED059ADF
:10FF10008DED069A8DED07AA8DED090AADF82850F2
:10FF2000ADF82A4055F016FF0CB0BDEC068BBDE8CD
:10FF3000F08100BFD84B00209F0CB3450AD7233C6B
:10FF400000FF7F472DE9F04F2DED028B1A4B047C0B
:10FF5000D3F890398DB0D3F88480D3F88870D3F873
:10FF60008C60D3F8905093ED258AD3F898B0D3F8ED
:10FF70009CA0D3F8DC908AF023FD00238DF82C3070
:10FF800016222523CDE90032029002AA53212046F1
:10FF90008DED078ACDF820B0CDF824A0CDF82890BB
:10FFA000CDF80C8004970596069555F0D3FE0DB05C
:10FFB000BDEC028BBDE8F08FD86B0020054BD3F869
:10FFC000103F2BB193F8CA00002808BF02207047E9
:10FFD00002207047D84B002008B5034BD3F8EC0E35
:10FFE00003681B68984708BDD84B0020024B93F864
:10FFF000E10EC0F340107047D84B002070B52C4E76
:020000040801F1
:100000002DED028B0546D6F8EC0E91ED018A0368C2
:1000100086B05B6A0C46984750B9BDEEC88A18EEA8
:10002000103ADB0704D4022006B0BDEC028B70BD91
:10003000D4E9040129F0C4FA0028F4D002A817F08A
:1000400023FA02AA214628465AF0B0FE0028EAD038
:10005000184902A817F02CFB03460028E3D1DFED76
:10006000160A00900246B0EE600A144802A90AF08F
:1000700049F8D8B1D6F8EC0E03685B6A9847044695
:1000800008B10020D0E70E480222042105F048FC08
:1000900060B1DFED090A094800942346B0EE600A1A
:1000A000224602A90AF02EF80028EAD10420BBE774
:1000B000D84B00203C7500200000000098840020F0
:1000C000D82B002008B591F82030032B1CD1D1ED9E
:1000D000027A9FED0E7A91ED060A0D4BF0EEE77A6B
:1000E000F4EEC77ADFED0B7AD3F8EC0EF1EE10FAEE
:1000F0004CBF0121002120EE270A0FF0C9F900288A
:1001000014BF0020042008BD0220FCE700000034DA
:10011000D84B00200000C84210B52DED028BD1ED68
:10012000007AF5EEC07AF1EE10FA82B00C4604DAED
:10013000042002B0BDEC028B10BD9FED197AF4EEE5
:10014000C77AF1EE10FAF3D891ED030A9FED158A04
:10015000F0EEC07AF4EEC87AF1EE10FA19D5D4EDCB
:10016000037A1148D4ED010A94ED000AF4EEC87A3E
:10017000D4ED027AFDEEE77AF1EE10FACDED017AD8
:100180009DF90410ACBF0122002202F049F80020C2
:10019000CFE7F7EE000A28F079F80028C8D0DEE7AC
:1001A0000000B443000000340488002091ED010AEF
:1001B000B5EEC00AF1EE10FA08B501DC042008BD66
:1001C0009FED107A104BD1ED007AD3F8EC0E20EEB3
:1001D000070A9FED0E7A0368F4EEC77AF1EE10FA83
:1001E00005DDDB6E98470028E8D00020E7E79FEDAB
:1001F000087AF4EEC77AF1EE10FACCBF9B6E5B6E14
:10020000F0E700BF0000C842D84B00209A9939405F
:100210003333F33F08B5D1ED007A9FED157AF0EE58
:10022000E77AF4EEC77AF1EE10FA1DD5D1ED017A36
:10023000F0EEE77AF4EEC77AF1EE10FA14D50D4835
:100240000222032105F06CFB80B10A480121FDF771
:10025000A9FF094890F85434012B03D000F58A60B7
:100260002EF058FE002000E0022008BD0420FCE72C
:1002700000000034D82B0020D87B002010B5D1ED31
:10028000007AFCEEE77A17EE903A9CB2012C02D08D
:10029000022C06D04CB90648214661F029F900200D
:1002A00010BD044803F07CF9F9E70420F8E700BF2B
:1002B00058760020D82B00201FB5D1ED017A0B7C99
:1002C000FCEEE77ACDED027AD1ED007A0093FCEEF8
:1002D000E77AD1ED030ACDED037A91ED020A9DF89C
:1002E00008309DF80C20014602480DF0BBFE05B019
:1002F0005DF804FBD82B002010B50A4C94F8053F9C
:10030000DB070CD402220521A4F5005005F008FB00
:1003100028B902221146A4F5005005F001FB002087
:1003200010BD00BFD84B002010B5D1ED007AFCEE17
:10033000E77A044617EE903A13F0FF030FD10F4B04
:10034000D3F8EC0E03689B6F984708B1002010BDEE
:100350000B4A2046062157F02FFF0420F7E7012B18
:1003600009D1064BD3F8EC0E0368DB6F98470028E1
:10037000ECD1044AEDE70220E9E700BFD84B0020AA
:10038000B85D0C08C85D0C089FED0B7A01F10C03F9
:10039000F1EC017AF4EE677AF1EE10FA0AD6F0EE9B
:1003A000E77AF4EEC77AF1EE10FA03DC9942EFD166
:1003B000012070470020704700007A4430B52DEDD1
:1003C000028B8DB00023054603930493059311F02F
:1003D000F1FC03A911F0C8FA58B311F0EBFC00F5D9
:1003E0005A7393E8070006AC84E80700DDED060ABF
:1003F0009DED070A2D7CF1EE600AB1EE400AAEF0E9
:1004000099F92046B0EE408A2BF02EFEDFED0B7AF4
:10041000089B0B93012228EE278A0C23CDE900329A
:10042000A82109AA28468DED098A8DED0A0A55F002
:1004300091FC0DB0BDEC028B30BD00BFE02E6542DB
:10044000272938B5054613D008D81B290ED02429F2
:1004500026D02846BDE838405BF06AB8282914D079
:10046000402903D0A1F14203012BF2D8012405E079
:10047000122154F093FE044610B90024204638BDE2
:10048000297C0C484DF01EFFF8E7162154F086FE3B
:1004900004460028F1D0297C06484DF0EDFFEDE739
:1004A0000C2154F07BFE04460028E6D02846FFF7D6
:1004B00085FFE3E79876002038B5194C94F8053F9E
:1004C000DB070D460AD4D4F8103F93F8CB303BB984
:1004D0000122114604F64440FDF7BCFC002038BD63
:1004E00094F9E03E002B4FF0020212DA0521A4F548
:1004F000005005F015FA0028F0D095ED000ADFED68
:10050000097AD4F8EC0E20EE270A01210EF0C0FF84
:10051000E4E70921A4F5005005F002FADEE700BF88
:10052000D84B00200000C84210B5214C94F8053F7C
:10053000DB070ED4D4F8103F93F8CB304BB194F9CD
:10054000E03E002B07DA0122082104F64440FDF7C3
:1005500033FD002010BDD1ED007A9FED167AF0EE4C
:10056000E77AF4EEC77AF1EE10FA0BD512480222C0
:10057000112105F0D5F9A0B9022211460E4805F067
:10058000CFF9E6E7D4F8EC0E03681B689847042817
:10059000DFD0D4F8EC0E03681B6898471428E5D127
:1005A000D7E7064840F6C41108F0D4FAD1E700BFF7
:1005B000D84B002000000034D82B0020848300207A
:1005C00070B58B8BC12B05460C463CD8BB2B0CD889
:1005D000542B6AD02ED8113B99B2052918D921463F
:1005E0002846BDE870405BF03BBEBC3B052BF6D80F
:1005F00001A151F823F000BFE5060108F306010848
:10060000DF050108DF0501088F06010899060108CA
:10061000052BE4D801A151F823F000BFCF06010853
:10062000DF050108DF050108DF06010841060108B2
:10063000AB060108732B22D0B22B24D0552BCED180
:100640000222092145E04AF21146B34237D00AD8C6
:10065000D12B26D0B3F5967F35D0D02BBFD1BDE8B6
:100660007040FFF70BBE4AF21246B34223D04AF263
:100670001346B342B3D1BDE87040FFF755BFBDE8A4
:100680007040FFF749BDBDE87040FFF78FBD2146C0
:10069000BDE87040FFF7B2BC2146BDE87040FFF7EF
:1006A00043BEBDE87040FFF707BE21462846BDE8BF
:1006B0007040FFF707BDBDE87040FFF7FDBEBDE825
:1006C0007040FFF719BEBDE87040FFF7A3BD0222DE
:1006D00005210A4805F024F948B9042070BD02221A
:1006E0000621F6E70221064806F082FAF4E7002028
:1006F000F4E70221024806F045FAEDE7D82B002086
:10070000EC7F002008B591ED007AF6EE007AB4EEA9
:10071000E77AF1EE10FA06DD044801220521FDF723
:100720004BFC002008BD0420FCE700BF1C58002043
:1007300030B52DED028BCD7893B0272D28BF27251E
:100740000C462722002108A8B0F0EEF92A4604F151
:100750000C0108A8B0F09EF9424BD3F8EC0E0368E8
:100760005B6A9847002841D09DF8465068063DD402
:1007700000244FF07E5329060493079406940594B1
:1007800027D504A82AF04AFBEA07019402940394AF
:1007900005F006032ED4002B2ED10D9B01930E9B4A
:1007A00002930F9B0393304809F05AFA9DED100A0B
:1007B000044630B340F2ED40B7EE001AFFEE000AF7
:1007C00027F068FE2848234601AA04A909F050FA38
:1007D0000CE0099B04930A9B05930B9B069304A8CA
:1007E0000C9B07932AF020FB0028CDD113B0BDEC61
:1007F000028B30BD062BD6D001211B4809F0CCF965
:10080000F4E7DFED1A0A4FF49E60B7EE001A27F006
:1008100041FEF6EE000AB0EE408A27F037FDE8B957
:10082000B6EE000A124BB4EEC08AF1EE10FAD3F81D
:100830009C3908DD38EE400A30EE008A93ED070A55
:1008400028EE000ABEE730EE480AD3ED087A30EE13
:10085000000AF0EEE77A27EEC00AB3E79FED030A3D
:10086000B0E700BFD84B00209884002000000000B3
:10087000D86B00202DE9F0439DB0814608460EA9B3
:10088000FEF774FF844BD3F8EC0E03685B6A98475D
:1008900050B19DF86C30012B09D0DA1F022A06D91D
:1008A0007E48012109F078F91DB0BDE8F083BDF85C
:1008B0006840A20504F0070604F0380704F4E07568
:1008C00001D5002DF0D04FF00008CDF81480CDF800
:1008D0001880CDF81C803EBB9FED716A9DED107AAB
:1008E000DDED117ADDED0F6A27EE067A67EEC67A46
:1008F00066EE866A083B012BCDED056A8DED067A22
:10090000CDED077A04D8674806AA05A9FDF7C6FD0C
:100910009DF86C30073B022B06D8634881F01CFC25
:10092000014605A82AF0C2FFCDF82080CDF824802A
:10093000CDF82880F7B9DDED147A129B0893F1EE1B
:10094000677A139B099308A94846CDED0A7AFFF709
:100950001BFD0028A4D09FED520A08A82AF0DAFF58
:100960009DF86C30083B012B04D84E4809AA08A911
:10097000FDF794FDCDF82C80CDF83080CDF8348093
:10098000EDB99FED476A9DED167ADDED177ADDED45
:10099000156A9DF86C3027EE067A67EEC67A66EE29
:1009A000866A083B012BCDED0B6A8DED0C7ACDEDFF
:1009B0000D7A04D83B480CAA0BA9FDF76FFD14F47F
:1009C000806233D1DFED397A9DED180A9DF86C1005
:1009D00020EE270ADFED327A0839012920EE270AB6
:1009E0008CBF0021012114F4006305BFDFED2F7AD5
:1009F000DDED190ADFED2E0A60EEA70A04BFDFED78
:100A0000287A60EEA70AAEB9002F35D1B3FA83F386
:100A1000B2FA82F25B0952090291019300920BAB88
:100A200008AA05A91D4809F025FA3DE79FED200A0F
:100A30000021D8E77FB9B3FA83F35B090120009363
:100A4000B2FA82F3CDE901105B0914480BAA08A998
:100A500009F0A8FC28E7002D7FF422AF0120B3FAAB
:100A600083F3B2FA82F2CDE900105B090B48520918
:100A70000BA909F03FFC17E7002D3FF411AFB3FAC3
:100A800083F3B2FA82F2CDE900165B09520905A997
:100A9000024809F071FA07E7D84B0020988400203B
:100AA0000000C842D82B00204C750020E02E654283
:100AB000000000002DE9F047A2B08046084614A9C6
:100AC000FEF754FE7E4BD3F8EC0E03685B6A984742
:100AD000C0B1BDF88040A30504F0070904F4E07735
:100AE00000D57FB10CAE304616F0CEFCB9F1000F48
:100AF00029D1DDE9150128F063FD30B971480121E4
:100B000009F04AF822B0BDE8F0879DF8841009AAE0
:100B100040465AF035F90028F0D0DDED177A9FED08
:100B20006A7A099B009367EE877A10ADFDEEE77A4B
:100B3000DDE9151217EE903A284616F0C5FC95E847
:100B40000F0086E80F00002514F0380A0695079577
:100B5000089514D1DDED1A7A189B0693F1EE677AA9
:100B6000199B079306A94046CDED087AFFF70CFCC8
:100B70000028C3D09FED540A06A82AF0CBFE0995A1
:100B80000A950B959FB99FED506A9DED1C7ADDED9E
:100B90001D7ADDED1B6A27EE067A67EEC67A66EEF1
:100BA000866A8DED0A7ACDED096ACDED0B7A14F4E3
:100BB000806805BFDFED457A9DED1E0A9FED440A72
:100BC00020EE270A04BFDFED407A20EE270A14F456
:100BD000006405BFDFED3D7ADDED1F0ADFED3C0A65
:100BE00060EEA70A04BFDFED387A60EEA70AB9F11C
:100BF000000F31D1BAF1000F52D13046CDED050AC8
:100C00008DED040A16F070FC03289DED040ADDED5D
:100C1000050A3FF473AF10A93046CDED050A8DEDFE
:100C2000040A10951195129516F0F0FD00283FF476
:100C300065AFB4FA84F46409B8FA88F3DDED050A07
:100C40009DED040ACDF804A000945B0906AA10A942
:100C50001C4809F07FF955E7BAF1000F0FD10123C5
:100C6000B4FA84F4CDE901A36409B8FA88F315480D
:100C700000945B0909AA06A909F094FB42E7002F3A
:100C80007FF43CAF0123CDE90073B8FA88F2B4FADF
:100C900084F30C485B09520909A909F02BFB31E7E1
:100CA000002F3FF42BAFB4FA84F3B8FA88F2CDF8F2
:100CB00000905B0952093146024809F023FA21E706
:100CC000D84B0020988400200000C842E02E6542E6
:100CD0000000000030B48D7A4B7A43EA0523CD7AC8
:100CE00043EA0543562B04460A461BD008D8522B2C
:100CF00012D0542B13D02046114630BC5AF048B9BC
:100D000003F18073863B23F07F43012BF3D8017CF2
:100D1000064830BC4DF078BC30BCFFF709BD30BC94
:100D2000FFF7A8BD30BCFFF7C5BE00BF9876002016
:100D30002DE9F0412DED028B044690B000F5954071
:100D4000002301226946403000934EF0D3F908B9E0
:100D50004D4B009304F50056DFED4C8AD6F8EC0EAF
:100D600003685B69984704F58048002840F0878055
:100D7000D8F89839D3EDDE7A93EDD88AFDEEE77A8C
:100D800028EE288A17EE903A1DB204F52F570C373B
:100D900001A938460DF038FF18B950F099FF3A4BC9
:100DA00001933722002102A8AFF0BEFEA3238DF8E5
:100DB000083095238DF8093089F00AFED8F890396B
:100DC000CDF80B00D6F8100FD3F8DC20D3F8E030C4
:100DD000CDF80F104430CDF81320CDF8173053F074
:100DE00033FC0346DFED2A0A93ED000AB7EE001A42
:100DF0009F2027F04FFB10EE103AD6F8100FCDF8D9
:100E00001B3003681B69984710EE103A04F59246B0
:100E1000CDF81F30743618EE103A3046CDF8233036
:100E200081F09EF920EE280A384610EE103ACDF8EF
:100E30002730D8F84039CDF82B30019BCDF82F3032
:100E40000DF004FF10EE103A3046CDF83330009B21
:100E5000CDF83730ADF83B5081F08EF9BDEEC00AC9
:100E6000372210EE103A02A904F57C60ADF83D304F
:100E70004FF036FF10B0BDEC028BBDE8F0819FED66
:100E8000048A002581E700BF2292CA7F0AD7233C4B
:100E90000000000010B500F58044D4F8900979F006
:100EA000E3FFD4F89819D4F89009BDE810407AF01F
:100EB00041B8000070B54FF4805104460DF0E6FFD4
:100EC00000284ED004F5804604F57C65D6F89009DC
:100ED00003689B689847692100F1940228464FF007
:100EE0008BFDD6F890090368DB6898476A2100F10A
:100EF000940228464FF080FDD6F8900903681B69DC
:100F000098476B2100F1940228464FF075FDD6F802
:100F100098296C21284602F52A724FF06DFD202198
:100F200020460DF0B3FFE0B104F50053D3F8EC0E0A
:100F300003681B69984778B1D6F8982928469032FB
:100F40006E214FF059FDD6F898292846BC32BDE8ED
:100F500070406F214FF050BD204609F08BFF0028F4
:100F6000EAD170BD08B510F025FFBDE8084010F0CB
:100F7000ADBC00007FB50E464FF6FF710446154626
:100F80000DF084FFE0B1102200216846AFF0CCFDE7
:100F9000A3238DF8003095238DF8013003238DF8BD
:100FA000023089F015FD1022CDF80300CDF80710AE
:100FB00004F57C6069468DF80B6003954FF010FFD7
:100FC00004B070BD7FB50E464FF6FF71044615465E
:100FD0000DF05CFFE0B1102200216846AFF0A4FDE7
:100FE000A3238DF8003095238DF8013004238DF86C
:100FF000023089F0EDFC1022CDF80300CDF8071087
:1010000004F57C6069468DF80B6003954FF0E8FEAF
:1010100004B070BD30B52DED048B87B004460D468D
:10102000182200216846B0EE409AF0EE608AB0EED9
:10103000418AAFF079FDA3238DF8003095238DF818
:10104000013006238DF8023089F0C2FC1822CDF859
:101050000300CDF8071004F57C6069468DF80B504D
:101060008DED039ACDED048A8DED058A4FF038FEA3
:1010700007B0BDEC048B30BD10B54FF480110446B1
:101080000DF004FF28B104F59650BDE810400FF0B4
:1010900013B910BD2DE9F0438FB0144605468946BB
:1010A0003122002101A8DDE916769846AFF03CFD1B
:1010B000A3238DF8043095238DF8053008238DF88F
:1010C000063089F085FC2368049363680593A36860
:1010D00006933B68CDF81D307B68CDF82130BB68A6
:1010E000CDF825303368CDF829307368CDF8070086
:1010F000CDF80B10CDF82D303122B3688DF80F905C
:1011000001A905F57C608DF81C80CDF831304FF0D9
:10111000E7FD0FB0BDE8F08370B52DED068B8CB008
:10112000144605460E462C22002101A8B0EE409A36
:10113000F0EE608AB0EE418AB0EE61AAF0EE429A1B
:10114000AFF0F2FCA3238DF8043095238DF8053021
:101150000B238DF8063089F03BFCDFED1A7A94ED15
:10116000007ACDF8070027EE277A29EE279A8DED31
:10117000077A94ED017ACDF80B1027EE277A68EE06
:10118000A78A8DED087A94ED027A8DF80F6028EE2B
:10119000278A67EE277A2C2201A905F57C608DED60
:1011A000049ACDED058A8DED068ACDED097A8DED97
:1011B0000AAACDED0B9A4FF093FD0CB0BDEC068B57
:1011C00070BD00BFE02E6542A020704770B5134B84
:1011D00088B004466946D3F8100F04F57C6504F521
:1011E00000561E2282F064F86A460D4928464FF0E8
:1011F00013FFD6F8EC0E03681B68984796F85C213D
:10120000014628464FF02CFF04F5965011F010F8D7
:1012100004F590701EF0D6FF08B070BDD84B0020CA
:10122000EEAA0C082A4B2B4A70B543600023436199
:101230008361C361C363284B426303644FF0804200
:10124000264B43640446826358305BF029FD244EEC
:10125000244BA365A82560195BF0D8FE6651303594
:10126000B5F56A7FF7D104F56A705DF07BFA00216D
:1012700004F5F66084F00CFC1B4BC4F864389FED59
:101280001B1ADFED1B0A9FED1B0A04F678007AF0AB
:10129000DDFB9FED161A9FED180AF0EE410A04F5EA
:1012A00009607AF0D3FB9FED111A9FED130AF0EE5F
:1012B000410A04F6A8007AF0C9FB20460F4945F020
:1012C000A1FD20460E4945F09DFD204670BD00BFA2
:1012D000183800200000C8410AD7233C0000E04035
:1012E00058A80C086CA80C08008200200000000020
:1012F0009A99993E0000B44300804A43089C0C0828
:10130000689E0C0870B54C4D4C49ADF50E7DD02251
:1013100006465AA8AFF0BEFB0FCD0EAC0FC40FCDE2
:101320000FC40FCD0FC495E80F0084E80F00002410
:101330005AAB18190021B7EE000A103445F030F806
:10134000D02CF5D13E4B0FCB02AC84E80F0001A9A5
:10135000204644F0D9FF90B19DF90430DFED396AA1
:10136000E06807EE103AB8EEC77AF0EE007AE7EEE2
:10137000267AB7EE000A80EE270A46F0EBF8002442
:101380000EAB181900211034B7EE000A45F008F82A
:10139000402CF5D12C49902236A8AFF07BFB0022DF
:1013A000092136A845F0A8F896F97469D6B9274DF1
:1013B0000FCD1EAC0FC40FCD0FC40FCD0FC495E8D9
:1013C0000F0084E80F00324604211EA845F094F86F
:1013D0009FED1F0A1F4846F0BDF81F48B7EE000AF0
:1013E00046F0B8F81D4C9FED1E0A0FCC06AD0FC598
:1013F00094E80F0085E80F00002106A844F0D0FF14
:101400009FED170A0021284644F0CAFF04F110019D
:1014100060221EA8AFF03EFB00241EAB181900216D
:10142000B7EE000A103444F0BBFF602CF5D15CF03D
:10143000ADFF0DF50E7D70BD7C4E0C08AC4D0C085B
:10144000BC4E0C08CDCCCC3DCC4E0C085C4F0C08EF
:1014500000000000F09A0C08FF9A0C089C4F0C0842
:10146000000034422DE9F04790B00DF106011D2037
:101470005DF07EF8002800F09E809DF80630614AFD
:101480000133DBB211210BA88DF8063088F064FB24
:1014900000220DF107010BA844F0BCFC9DF80630BA
:1014A000594A112105460BA888F056FB00220DF180
:1014B00007010BA844F0AEFC9DF80630534A1121F9
:1014C00006460BA888F048FB00220DF107010BA887
:1014D00044F0A0FC9DF806304D4A03F03F03112173
:1014E00007460BA888F038FB00220DF107010BA876
:1014F00044F090FC8046002D5DD0002E5BD0002F84
:1015000059D0002857D0284644F09CFE002852D1DC
:10151000304644F097FE00284DD1384644F092FE04
:10152000002848D1404644F08DFE002843D1394C74
:1015300094E80F000DF10C0C10348CE80F0094E8C7
:101540000F000DF11C0989E80F0002A9604644F064
:10155000DBFE98B3BDF8084002A9484644F0D4FE2B
:1015600000284AD0BDF8083054BB23B340F2E2440F
:101570009C420FFA84FA0FFA83F927D80DF10A0179
:101580003046ADF80A9046F0DBFA0DF10A01284624
:10159000ADF80AA046F0D4FA0DF10A013846ADF8CC
:1015A0000AA046F0CDFA00230DF10A014046ADF83D
:1015B0000A3046F0DFFA10B0BDE8F0870024CBE730
:1015C00040F2D662002B08BF1346D1E70DF10A01A5
:1015D0003046ADF80AA046F0B3FA0DF10A012846EC
:1015E000ADF80A9046F0ACFA0DF10A013846ADF8B4
:1015F0000A9046F0A5FA0123D6E7002CDBD040F292
:10160000D663B5E7109B0C081C9B0C08289B0C08A4
:10161000359B0C081C500C0837B500F50651782294
:10162000203104464DF04AFF00220C21244844F0AA
:1016300063FF2046FFF716FF04F506500022B7EEC1
:10164000000A0221343044F0DFFF012504F5025185
:101650001C4A009500232031452044F051FF1A4ACE
:101660001368D90705D41949156004F501530833E7
:101670000B6004F50850154901221430012544F08F
:1016800091FF134A0095002304F57C61FD2044F08E
:1016900037FF104B1A68D20705D40F4A1D6004F5B6
:1016A0008F54083414600C48012144F097FF45F032
:1016B000AFFD0A4A138843F00103138003B030BD25
:1016C000489B0C0888C90D08FC87002000220020D8
:1016D0004C4B0D08008800200C220020408A00207E
:1016E0000F299DBF302303FB0100503000207047BD
:1016F000014B93F9E7017047D84B0020024B93F858
:10170000050F00F001007047D84B0020044BB3F8E0
:10171000AC31DB075ABF0069C0F3401000207047AE
:10172000D84B0020014BD3F82C0B7047D84B00202E
:1017300008B503689B68984730B9044B93F9040FC8
:10174000B0FA80F0400908BD0020FCE7D84B00202B
:1017500038B50D1E2DDB174C94F8382BEBB29A429E
:1017600027D3D4F8343B0122595DA4F5005004F08E
:10177000D7F8F0B15BF014FC03215CF0C9FBC0B9F1
:101780005BF00EFC0D215CF0C3FB90B994F9CC31F9
:10179000EB40DB075CBF94F9E611E940A4F500508B
:1017A00048BF0221BDE8384058BF01F00101FCF7F5
:1017B0000FBD38BDD84B0020022A10B50C4605D10C
:1017C000BDE810400948352204F0AAB8084BD3F808
:1017D000EC0E03681B689847A04205D15BF0E0FB64
:1017E000BDE810405BF066BB10BD00BFD82B0020E9
:1017F000D84B002029B1022907D1044BC3F8E41EBD
:101800007047024B0122C3F8E42E7047D84B0020EA
:1018100031B1022907D1044B012283F8E82E704729
:10182000014B83F8E81E7047D84B002010B500F537
:101830000053DFED186AD3F8242BD3F8203BB2F91C
:101840000820B3F908309FED147A07EE902AF8EEDD
:10185000E77A0446C7EEA60A012100F5965007EE86
:10186000903AF8EEE77A60EE870A87EEA60A20EE55
:10187000070A10F03DFB50F02BFA26214FF0C0FF75
:1018800004F53350054ABDE810400621043053F0FA
:1018900069BA00BF0000C84235FA8E3C28A60C0881
:1018A00000F58042002382F8AC39044A00F5335039
:1018B00013720621024A043053F054BAB58900204D
:1018C00034A60C08F8B500F58045044695F8AC1927
:1018D000002954D02A4B2B4AD3F8EC0E904204D165
:1018E000D3F8103F93F8CB3023B92046BDE8F84039
:1018F000FFF7D6BF244E95F8AD7904F500530120CB
:1019000093F9E02E3072BFBB002A38DB85F8AD09B1
:101910000139C9B285F8AC19D3F8242BD3F8203B90
:10192000B2F90820DFED196AB3F908309FED187A93
:1019300007EE902AF8EEE77AB1FA81F1C7EEA60A2F
:10194000490904F5965007EE903AF8EEE77A60EE12
:10195000870A87EEA60A20EE070A10F0C9FA95F862
:10196000AC3963B904F5335033720A4ABDE8F84024
:101970000621043053F0F6B9002AC9DAB5E7F8BDFC
:10198000D84B002080860020B589002000007A45D1
:1019900035FA8E3C48A60C086D2900F3E380012936
:1019A00001DC5CF003B98B1E6B2BFAD80FF2040C30
:1019B0005CF823F0C31B0108BD1B0108C31B010811
:1019C000C31B0108A3190108C31B0108A3190108BF
:1019D000A3190108BD1B0108A3190108C31B0108B5
:1019E000BD1B0108BD1B0108A3190108C31B010889
:1019F000C31B0108C31B0108A3190108A31901088F
:101A0000BD1B0108C31B0108BD1B0108A319010868
:101A1000BD1B0108BD1B0108A3190108A31901087A
:101A2000A3190108A3190108A3190108BD1B010886
:101A3000C31B0108A3190108A3190108A319010870
:101A4000C31B0108A3190108BD1B0108A319010844
:101A5000A3190108C31B0108BD1B0108A319010834
:101A6000A3190108A3190108C31B0108C31B01081E
:101A7000C31B0108A3190108A3190108C31B01080E
:101A8000A3190108A3190108C31B0108C31B0108FE
:101A9000C31B0108A3190108A3190108C31B0108EE
:101AA000C31B0108A3190108A3190108A319010800
:101AB000A3190108A3190108A3190108C31B0108F0
:101AC000C31B0108C31B0108C31B0108C31B01087A
:101AD000C31B0108A3190108BD1B0108BD1B010898
:101AE000A3190108A3190108A3190108A3190108E2
:101AF000A3190108A3190108C31B0108BD1B010894
:101B0000A3190108A3190108A3190108A3190108C1
:101B1000A3190108A3190108A3190108A3190108B1
:101B2000A3190108A3190108A3190108A3190108A1
:101B3000A3190108A3190108C31B0108A31901086F
:101B4000A3190108A3190108A3190108A319010881
:101B5000A3190108A3190108A3190108A319010871
:101B6000BD1B0108A12921DC96297FF71AAFA1F13D
:101B700097030A2B3FF615AF0FF2040C5CF823F025
:101B8000C31B0108C31B0108A3190108C31B0108DB
:101B9000A3190108A3190108A3190108A319010831
:101BA000BD1B0108BD1B0108C31B0108B42908D0D7
:101BB000DB2903D0B2297FF4F4AE704700235BF039
:101BC000C7BF704770B563298AB000F3D18001297F
:101BD00004DC0AB0BDE870405BF08ABD8B1E612B4F
:101BE000F7D801A454F823F0E71D0108FB1D0108F4
:101BF0001B1E0108231E0108D31B0108531E0108E8
:101C0000D31B0108D31B0108011F0108D31B0108C6
:101C1000D31B0108091E0108271F0108D31B010857
:101C2000FD1E0108611F01086F1F0108D31B010879
:101C3000D31B01087F1F01088D1F01089B1F01088E
:101C4000D31B0108BD1F0108CF1F0108D31B0108CA
:101C5000D31B0108D31B0108D31B0108D31B0108A8
:101C6000E11F0108FB1F0108D31B0108D31B01085A
:101C7000D31B0108FF1F0108D31B0108D31B010858
:101C8000D31B0108D31B010803200108D31B010843
:101C9000D31B0108D31B0108D31B0108D31B010868
:101CA000D31B0108D31B0108D31B0108D31B010858
:101CB00013200108D31B0108D31B0108731F01085F
:101CC000771F01087B1F0108D31B0108D31B0108E4
:101CD000D31B0108D31B0108D31B0108D31B010828
:101CE000D31B0108D31B0108D31B0108D31B010818
:101CF000072001080B2001080F200108D31B010851
:101D0000172001081B200108D31B01085D200108D2
:101D10001F200108D31B0108D31B0108D31B010896
:101D2000D31B0108D31B0108D31B0108D31B0108D7
:101D3000C3200108D31B0108D31B0108D31B0108D2
:101D4000D31B0108D31B0108D31B0108D31B0108B7
:101D5000D31B0108D31B0108D31B0108D31B0108A7
:101D6000D31B0108D31B0108D31B0108D92001088C
:101D70009F291DDC96297FF72CAFA1F19703082B33
:101D80003FF627AF01A454F823F000BFDD2001087F
:101D9000E1200108D31B0108F5200108D31B01082D
:101DA000D31B0108D31B0108D31B0108D120010854
:101DB000B42900F0D780DB2917D0B2297FF409AF0E
:101DC000002A00F07781022A0FD1AD4BD3F8EC0E38
:101DD00003689B6F984740B959F020FEA94A042137
:101DE00052F0C0FF01E0022A01D001242EE035228A
:101DF0000E21A54803F094FDF7E7111E18BF01213D
:101E0000A148FCF7E5F9F0E7012A04D0022A14BF43
:101E100000210221F4E71146F2E70621FFF7CCFC8E
:101E2000E3E7022AE1D1964DD5F8EC0E0368DB6AB0
:101E3000984704460028D8D0D5F8283BB3F9083095
:101E4000002BD2D1A5F50050FFF7F0FC20460AB0D8
:101E500070BD022AC9D18A4D8C4BD5F8EC2E9A421E
:101E6000C3D0D5F8103F93F8CB30002BBDD005F58B
:101E70004054B4F984342BB9D5F8283BB3F9083071
:101E8000002BB2D01C22002103A805AEAEF04CFE00
:101E9000304615F0F9FAB4F984347D4C93B9162321
:101EA000ADF80E30D4F868397A48642BB8BF642393
:101EB00003A906932AF084FC20B14FF009FF2721E3
:101EC0004FF09EFC04F664130FCB86E80F00D5F8A4
:101ED000283B7048B3F90830002BCCBF10231523E2
:101EE00003A9ADF80E302AF06BFC00283FF47DAF5B
:101EF0004FF0EEFE27214FF083FC76E703218DE7BC
:101F0000022A04D05E4B002283F83C2B6DE7624826
:101F1000192146F069FA04460028F3D0584B0122F3
:101F200083F83C2B92E7012A0BD0022A11D0002A19
:101F30007FF45BAF524B83F810224FF0C9FE2B2188
:101F4000D9E74F4B019283F810224FF0C1FE2C21AC
:101F5000D1E74B4B83F810224FF0BAFE2D21CAE790
:101F60000F215BE74D48114686F08AFE3DE70921C7
:101F700054E7042152E7052150E717214EE7901E50
:101F80004142414146485FF0B3FA2EE7022A7FF40E
:101F90002CAF3D4801F004FB27E7012A06D0022AB6
:101FA00007D0002A7FF421AF1146EBE711460192DA
:101FB000E8E73B4801215FF09BFAEAE7344B911ECA
:101FC000D3F890394A424A4183F820200DE7931E06
:101FD000594259412E4BD3F890097AF043FE04E759
:101FE000274B013A93F8E21E012A8CBF00220122FE
:101FF00062F3041183F8E21EF7E611210EE71221C5
:102000000CE715210AE7002108E7102106E7022165
:1020100004E7012102E7072100E70B21FEE6022A7F
:10202000204B0ED1012483F874434FF051FE4A2116
:102030004FF0E6FB59F0F2FC1B4A062152F092FEEB
:1020400004E7002283F874234FF042FE4B214FF047
:10205000D7FB59F0E3FC154A0621C1E6012A09D055
:10206000022A0AD0002A7FF4C0AE012110480CF0E9
:1020700003FEBAE601920021F8E71146F6E700BF39
:10208000D84B002083A60C08D82B0020EC7F002022
:10209000D86B002028800020E83800200082002033
:1020A00058760020D87B002060A60C0871A60C088A
:1020B000A4570020184BD3F8EC0E0368DB6F984749
:1020C00093E61146FFF796FB144803F0D3FF8CE626
:1020D0001146FFF79DFB88E61B219FE61C219DE62C
:1020E000022A7FF482AE0E48FCF752FE59F096FCAD
:1020F0000C4AB1E711465BF01BFA0B4877F030FC55
:10210000044600283FF471AE034A92F8E33E43F0E0
:10211000020382F8E33E99E6D84B0020707F00204E
:10212000D82B00209CA60C081C58002010B5044693
:10213000044880F013F804F10801BDE8104027F0CE
:10214000BDB900BF4C75002038B504462DED028B9B
:10215000114880F009F8054629F0ECF80F48B0EE78
:10216000408A0CF02FFE90B1DFED0D7AB4EEE78AD5
:10217000F1EE10FA0BDDD5ED000A95ED010AACF099
:10218000D9FADFED087A20EE270A84ED080ABDECC3
:10219000028B94ED080A38BD4C750020D82B002026
:1021A00000401C46E02E6542074B93F9CD01022802
:1021B00005D0032806D0003818BF0120704781F0F1
:1021C0000100704704207047D84B002003688B4201
:1021D00016D00429C0E9001302D007290ED0704799
:1021E000084B9FED097A03F59863D3ED007AF8EE7A
:1021F000E77A67EE877AC0ED087A7047002383623A
:10220000704700BFD83B00200AD7233C08B50246E0
:10221000FFF7CAFFBDE8084001461046FFF7D6BFEA
:1022200070B52DED048B0446F0EE408AB0EE608A66
:102230000D46164688F0C4FB9FED329ADFED329AC8
:10224000E06176B3236843B9304B03F59863D3ED6F
:10225000007AF8EEE77AC4ED097A68EE898A002DF3
:10226000B7EE000AFFEE007AB8BFB0EE670A68EE7C
:10227000808AC4ED058A264BB4EEE98AF1EE10FAA5
:10228000D3F8900930DA79F0CBFC20EE090A84ED1E
:10229000060ABDEC048B20460321BDE87040FFF721
:1022A00095BF94ED090A98EE890A26F09DF8002D55
:1022B00084ED050A0BDAB4EEE90AF1EE10FADADB86
:1022C000DFED147A30EE670A84ED050AD3E7D2D049
:1022D000DFED117AB4EEE70AF1EE10FACBD8DFEDBC
:1022E0000D7A30EE270AEFE779F09AFCB4EE480A4F
:1022F000F1EE10FA48BFB0EE408A28EE098A84ED6C
:10230000068AC6E70000C84200000034D83B00201F
:10231000D86B002000A00C47000000B410B52DEDD4
:10232000028B0446B0EE608AF0EE408A88F048FBEB
:10233000DFED090AE06168EEA08A68EE200AC4EDCC
:10234000098ABDEC028BC4ED0A0A20460621BDE8CD
:102350001040FFF73BBF00BF0000C84208B54A6805
:102360000346084642B98A6832B9C96821B9BDE84E
:1023700008400748FFF74ABF03F1080115F046FA85
:1023800028B1BDE8084002480221FFF71FBF08BD81
:102390000488002008B50721FFF718FF80ED0A0A1E
:1023A00008BD000008B50368032B23D1D0ED057AE2
:1023B0009FED127AF0EEE77AF4EEC77AF1EE10FABA
:1023C0001AD50F4B90ED090A03F59863D3ED007A07
:1023D000F8EEE77A37EEC00A26F006F8DFED097A64
:1023E000B0EEC00AB4EEE70AF1EE10FA94BF012095
:1023F000002008BD0120FCE70020FAE700000034BF
:10240000D83B00200000484330B50368023B85B04C
:102410000446082B6FD8DFE803F0050D30374D6315
:1024200041636300FFF782FE84ED090A94ED090A17
:1024300005B030BD88F0C4FAE369DFED320AE0612F
:10244000C31A07EE903AF8EE677A94ED050A67EE44
:10245000A07AD4ED060AF12020EEA71A67EEE00A72
:1024600026F018F8D4ED057A77EEC07AC4ED057A37
:10247000D4ED097A37EE800AD6E7FFF765FEDFED87
:10248000227A20EE270ACFE7204B03F63873D3EDEC
:10249000007AF8EEE77AC0ED097AC7E71C4DD5F867
:1024A000A4097DF091FF0028C0D0D5F8A4391B6B9A
:1024B0006362BBE788F084FAE3699FED127AD4ED9A
:1024C0000A6AE061C31A07EE903AF8EE677A67EE9F
:1024D000877A94ED097AA6EEA77A84ED097AA5E7C2
:1024E0000B4B9FED0C0AD3F890096C3029F0BEF924
:1024F00084ED091A9AE7064BD3F89839D3F8443398
:10250000D6E700BF6F12833A0000C842D84B0020C4
:10251000D86B00209F0CB3450368092B08D8DFE86F
:1025200003F0050A0505050507070510002383626A
:1025300090ED0A0A7047044BD3F89839D3F8483322
:10254000F5E7C36AF3E700BFD86B0020F8B50023B6
:10255000214FCB6297F8053F204E13F0010F044640
:102560000D462DD1D7F8EC0E03685B6F984738B352
:10257000D7F8EC0E03F08AFBDFED197A85ED0B0A34
:10258000B0EEC00AB4EEE70AF1EE10FA03D4092166
:102590003046FFF71BFE1148FFF736FF0F4884ED6A
:1025A000000AFFF7B9FF336884ED010A0A2B0FD840
:1025B000DFE803F00C1010101010100C100C0C00C1
:1025C0003368092BE7D105480021E2E70223A36025
:1025D0002046F8BD0123FAE7D84B002004880020EC
:1025E00000000034034B01221A6000229A60DA6076
:1025F0001A6170470488002013B501A904460CF045
:1026000081FA04F5804320B9012283F8552A02B0EB
:1026100010BDDDED017ADFED096A03F64822B8EE60
:10262000E77AD2ED007A67EEA67AB4EEE77AF1EEB9
:1026300010FA54BF01220022E7E700BF0000C842A1
:102640002DE9F04F2DED068B00F500578DB097F971
:102650001E32054600F5A04400F5965B33B1D7F86D
:10266000103F93F8CB80B8F1000F0FD10021A4F8F0
:10267000681358460FF004FE94F8691358460DB0DD
:10268000BDEC068BBDE8F04F0FF004BE88F098F962
:1026900005F5804A0190DAF898099FED958A90ED4A
:1026A000DBAA7CF0B1F809AE002800F0CC80DAF8A3
:1026B000983903F55C7393E8070086E80700304615
:1026C0008DED0B8A29F0D0FCB0EE409A28460CF034
:1026D00079FB05F5924909F17409002800F0B680EC
:1026E00048467FF041FD07C886E8070030468DED7B
:1026F0000B8A29F0B9FCF0EE409AD7F8EC0E03688B
:102700001B689847122840F0AA80002384F8683399
:10271000D7F8EC0E03685B69984728B1D7F8283BD7
:10272000B3F90830002B0BDC97F9E03E002B07DAF9
:10273000019BC4F86C3348467FF012FD84EDDC0A3F
:1027400094F868335BB1019BD4F86C03181A41F21A
:102750008833984240F29180002384F86833DAF895
:1027600090099FED640A6C3029F080F88DED090A1C
:10277000CDED0A0A8DED0B1A96E8070006AB03AE05
:102780009FED5D0A83E8070086E80700304629F0E0
:102790006DF82846B0EE408AF0EE608A8DED060AAC
:1027A000CDED070A8DED081A0CF00CFB002874D053
:1027B000DFED527AF4EEE79AF1EE10FA94BF0125BC
:1027C0000025DAF898097CF01FF830B1DFED4B7A7C
:1027D000B4EEE79AF1EE10FA0AD9002D64D1D7F8D9
:1027E000EC0E03681B689847022864D04FF000087D
:1027F000DAF898097CF02AF90546002874D0B5EE7D
:10280000C0AAF1EE10FA6ED5DFED3D7AB4EEE7AA7C
:10281000F1EE10FAACBF0126002648467FF0ACFC72
:1028200066B9DFED387AB0EEC00AB4EEE70AF1EE31
:1028300010FA5BD8002D08BF4FF0000894F8681319
:1028400084F8698315E7B0EE489A3FE728460CF014
:102850008DFA00287FF444AFDFED259A4DE7D7F8D5
:10286000103F93F8CB30002B3FF452AF97F9E03E86
:10287000002BBFF64DAF012348E748467FF070FCC0
:10288000D4EDDC7A30EE670ADFED1F7AB4EEE70AAA
:10289000F1EE10FA3FF760AF61E728460CF066FAF8
:1028A0000546002884D18CE7DAF898097BF0ACFF64
:1028B000002894D19CE7B0EE680AABF019FDF0EE69
:1028C000408AB0EE480AABF013FDDFED107A20EE3F
:1028D000280AB4EEE70AF1EE10FACCBF4FF0010877
:1028E0004FF0000884E700252E4696E7B046A5E79E
:1028F000000000009F0CB345D30237390000FA42B4
:102900000000C8C2000070420000484255CF7D3F21
:1029100038B504460CF056FA04F5965548B92046E9
:102920000CF024FA014620B92846BDE838400EF0E4
:1029300029BF04F50054D4F8EC0E03689B6C98474B
:1029400020B9D4F8EC0E0368DB6C98470146EBE73E
:1029500030B589B00446684614F096FD04F59655E6
:1029600004A814F091FD694628460EF0C5FF98B101
:1029700004A928460FF010F870B1059B0193236855
:102980000022DB6C69462046984728B104F52750A1
:102990000121043083F048FB09B030BD00F58052BE
:1029A00092F83C25D2070BD400F50052D2F8102F34
:1029B00092F8CB1009B1FFF7CBBF03689B6C1847A7
:1029C0007047000030B587B0044602A8019114F0AA
:1029D0005BFD02A904F596500EF08EFF019A18B91E
:1029E0000025284607B030BD236802A9DB6C2046CD
:1029F000984705460028F3D004F5275001210430FC
:102A000083F012FBEDE70000F0B5044685B06846A0
:102A100004F596570E46154614F036FD69463846BD
:102A20000EF0BAFF10B9002005B0F0BD31463846AF
:102A30000EF01AFE0028F6D0002DF5D004F58054D3
:102A4000284694F83C3543F0020384F83C35EBE724
:102A50002DE9F04F2DED0A8BBDB0044624220E4621
:102A600018A80021AEF060F82422002121A8AEF0C1
:102A70005BF8242200212AA8AEF056F804F5005590
:102A80002422002133A8AEF04FF80023CDE90D3306
:102A90000F9395F8E13E13F0080837D143F008038F
:102AA00095F81C2B079285F8E13E15F077FE90F91A
:102AB000213003B390F84033EBB104F25457384659
:102AC00015F07CFDC24694F876355FFA8AF18B42A8
:102AD0001FD9384615F050FD0AF1010A8146002839
:102AE000F1D1C84A0221304655F066FB95F8E13E27
:102AF00069F3C30308E0C44A0221304655F05CFB89
:102B000095F8E13E6FF3C30385F8E13E4FF001080D
:102B10003AE304F531530433012118460BEE903AA1
:102B2000FBF73EF8814608B9B84ADBE720460BF0D0
:102B300071FED5F8283BB3F90890B9F1000F01D028
:102B4000B34AD9E795F9E03E002B01DBB14AC9E76A
:102B5000204601F073FE04F53C533C3318464A46C8
:102B60000CA90CEE103A12F015F8002814BF02233D
:102B700001230393F123CDE913398F210A23CDE9F2
:102B80000031307CADF85490032313AA4D2153F04B
:102B9000E1F8A14B9FEDA18A01225A720621A04AB9
:102BA000304655F009FB039B022B0CBF9D4A9E4A01
:102BB000062130464FF0000955F0FEFA85F8DA910B
:102BC0004946384615F044FC94F876355FFA89F1A9
:102BD0008B420CD913AA38468DED138A8DED148AD9
:102BE0008DED158A09F1010915F0B4FAECE73846C4
:102BF00015F0E4FC4FF0000A4FF07C0B94F87625BA
:102C00005FFA8AF94A4519D94946384615F094F9C8
:102C1000C0B20BFB00403CAA0C2300F2E45003FBC3
:102C2000092C07C8ACF1900C8CE807003CAA02EB19
:102C3000890909ED2F8A0AF1010ADFE741F288319B
:102C40000AA821F051FFD5F8100F9FED749A036880
:102C50009FED76AA9B6ADFED76AA9847D5F8100F0C
:102C6000012180F029FA734B1B680293D86A03682C
:102C700001211B68984787F0A3FE059087F0A0FE0E
:102C8000F0EE499A0690002504F50059079A99F844
:102C90001C3B934240F0D68094F89618384615F0C5
:102CA0006BFC002800F0CE80D9F8103F93F8CB30B1
:102CB0000493002B00F0C68041F288310BA821F06C
:102CC00013FF87F07DFE059BC01A132840F2D780C2
:102CD00087F076FE059020460BF09CFD5BF062FECF
:102CE00082465BF0F9FDD9F8283BD9F8100FB3F90B
:102CF000083000EE103AB8EEC00A20EE0A0A81F061
:102D0000B5FE50465BF0F0FD384615F057FC1CEE62
:102D1000100A12F029F9D9F8283BDFED400AB3F97F
:102D2000083000EE103AB8EEC00AA22020EE0A0ADF
:102D3000B7EE001A25F0AEFBB4EEE90AF1EE10FA98
:102D40001CEE100A4FF000020CA958BFF0EE409A9A
:102D5000F0EE408A11F01EFF08B900230C939DEDA0
:102D60000C8ADFED357AB4EE498AF1EE10FAF4EE12
:102D7000E78A48BFB0EE498AF1EE10FA80F28D8002
:102D80009FED2E9ADFED2E8A4FF0000A94F87635EB
:102D90005FFA8AFB5B4540F294814FF00C0918AB57
:102DA00009FB0BF903EB0900B0EE490A28F05EFDC0
:102DB00059463846CDED110A8DED121A8DED100AE7
:102DC00015F0BAF87C23C0B203FB0040B0EE680AED
:102DD00000F2E45028F04AFD3CAB13A910A8994436
:102DE0008DED130ACDED140A8DED151A28F012FDA4
:102DF0000AF1010A09ED240A49ED230A09ED221A14
:102E0000C4E700BF99A80C0888A80C0897BC0C0858
:102E1000A7A80C08B9A80C08B5890020000000007C
:102E2000C4A80C08D9A80C0807520C086F12833AE2
:102E30000000C842F887002000000034A4707D3FE5
:102E40000AD7233CD9F8100F03689B6A9847D9F832
:102E5000100F002180F030F9029BD86A036800212E
:102E60001B689847002D40F05F813046C94A052114
:102E700055F0A2F92946384615F0EAFA70E1029BAE
:102E8000986A036805215B6898470BA821F038FE13
:102E9000B0EE498AB0EE489AF6E64FF000094FF0DE
:102EA0000C0B04F5B26A94F876255FFA89F39A421E
:102EB00022D919463846089315F03EF8089B0BFBBB
:102EC00003F13CAB5A18A2F16C034FF07C0CC0B27A
:102ED000CDE908320CFB00A018AB1944543028F09F
:102EE000AFFC089B099A09F1010902ED1B0AC3ED29
:102EF000010A83ED021AD6E7039B012B4FF0000A6B
:102F000046D19FEDA5BA9FEDA59A4FF00C0B94F812
:102F100076355FFA8AF5AB4240F286800BFB05F509
:102F20003CAB03EB0509A9F14803089321ABB0EED4
:102F3000680A581928F0AAFC089B09ED120AC3ED8B
:102F4000010A83ED021A33ABB0EE4B0A581928F090
:102F50008DFC2AAB58198DED100AB0EE490ACDED63
:102F6000110A8DED121A28F081FC13A910A88DED1D
:102F7000130ACDED140A8DED151A28F061FC0AF143
:102F8000010A09ED090A49ED080A09ED071ABEE729
:102F90009FED819A9FED81BAF0EE088A94F876351C
:102FA0005FFA8AF94B4564D99DED0C0AB4EEE80A44
:102FB000F1EE10FA35DB0C2303FB09F93CAB03EB14
:102FC000090521AB03EB090028F060FC33AB45EDAC
:102FD000110A05ED101A05ED120A03EB0900B0EE17
:102FE000490A28F043FC2AAB03EB09008DED100AD7
:102FF000B0EE4B0ACDED110A8DED121A28F036FC19
:1030000013A910A88DED130ACDED140A8DED151A34
:1030100028F016FC05ED090A45ED080A05ED071A2A
:10302000049D0AF1010AB9E74FF000094FF00C0ABC
:1030300094F876355FFA89F5AB4241D933AB0AFB98
:10304000053029F011F81BEE900AF0EE408A76F078
:1030500083FC07EE900AB8EE677A3CABC8EE877A3D
:1030600003EB850509F1010967EEAA7A45ED2F7A90
:10307000DEE74FF0000A4FF00C0B94F876355FFA5C
:103080008AF94B451DD933AB0BFB093028F0ECFF17
:10309000C8EE297A0AF1010A1BEE900A67EE808ACF
:1030A00076F05AFC07EE900AB8EE677A3CABC8EEB1
:1030B000877A03EB890967EEAA7A49ED2F7ADCE774
:1030C000049D87F07DFC069BC01AB0F5FA7F27D9D6
:1030D00087F076FC04F50053DDED0D7AD3F8283B3C
:1030E0000C9A1B891392FCEEE77A339A1492ADF88E
:1030F0005C30349A159217EE903A359A1692ADF8E4
:103100005E30F0221423CDE90032B121069013AADB
:10311000307C52F01FFE6FF06DFA317C6FF064F975
:103120000BA821F0EDFCB5E60399384615F090F9AF
:1031300000254FF00C0A94F87635E9B28B4207D996
:1031400033AB0AFB0132384615F004F80135F2E7DB
:10315000384615F011F8124A0621304655F02CF881
:10316000104B002520465D7201F05AFB04F5075014
:103170001A3043F01DFF99F8E13E65F3C30389F867
:10318000E13E0AA821F0BCFC40463DB0BDEC0A8BF4
:10319000BDE8F08F2D1C0E08A4707D3F0AD7233C9C
:1031A000E1A80C08B58900207FB54D4BD3F8E83A6B
:1031B000DB07044600F1928000F50055D5F8103F7A
:1031C00093F8C120002A40F0898093F8CB30002B7F
:1031D00000F0818095F9E03E002B7CDB00F5A043F8
:1031E00093F87433002B79D100F580469FED3D0AAA
:1031F000D6F890096C3028F039FBCDED020A60EE6C
:10320000A00ADFED397A8DED010AE0EE000A8DEDBE
:10321000031AF4EEE70AF1EE10FA5CDCD6F8903906
:103220009FED327AD3ED377AF4EEC77AF1EE10FAE9
:1032300004D5D5F8103F1B7A002B4CD0B5EE007AA0
:10324000F4EEC77AF1EE10FA45D404F592407430EA
:103250007EF092FFDFED267AB4EEE70AF1EE10FA87
:1032600039D8D6F890399FED237AD3ED367A67EEC8
:10327000877AB3EE0E7AF4EEC77AF1EE10FA2ADA14
:103280001D4AB4F9A410138801339BB2138019B9F5
:10329000B4F8A210A4F8A410B4F8A41099421DD850
:1032A000002616804EF014FD012219214EF0C8FAB6
:1032B000D5F8100F03685B699847431C04F5335039
:1032C0000E4A3146043051F04DFDD5F8103F012231
:1032D00083F8C12002E0084B00221A8004B070BDC0
:1032E000D84B00209F0CB3454054094A6666663FA0
:1032F000000000B4E02E65423E880020F8A80C08CB
:10330000F0B52DED028B4B4BD3F8E83A9B0785B017
:1033100004461FD400F58046DFED478AD6F89009B1
:1033200003681B699847D0ED017AF4EEE87AF1EE74
:1033300010FA0FDB04F5005304F5A645D3F8102F5F
:1033400092F8C110783549B1002303A928460393A8
:1033500051F07CF905B0BDEC028BF0BD92F8CB20AA
:10336000002AF1D093F9E03E002BEDDB04F5A047F5
:1033700097F87433002BE7D1D6F8900903681B69DE
:103380009847D0F8A430D6F89009039303681B69D6
:10339000984704F58C7200F1A401284651F0C4F955
:1033A000DDED037AB0EEC08AF0EEE77AF4EEC87A8B
:1033B000F1EE10FA03D503A9284651F047F9D6F8E3
:1033C000900903681B699847D0ED040AF4EEE80AF7
:1033D000F1EE10FABEDBF6EE087A60EEA77AF4EEB4
:1033E000C87AF1EE10FA1DD587F0EAFAD7F88433DF
:1033F00042F21072C31A9342ACD9DFED107AC7F8CB
:10340000840368EE277A04F5335417EE900AF9F72F
:1034100083F80434CDE90001094A0021204651F027
:10342000A1FC97E79DED030A24F030FF0028DBD1D3
:1034300090E700BFD84B0020000000340000C842D5
:1034400014A90C0810B5044600F595405EF062F82A
:1034500004F595400121BDE81040203066F02CBDF8
:10346000F8B500F58045044695F9803A53B300F568
:10347000005695F8942A96F8E03EDB43C3F3C01358
:1034800063F3C30200F5954700F5924085F8942A4E
:1034900074307EF071FEDFED3E7A384620EE670A2A
:1034A0005EF0B8F804F5A04393F8743353B9384686
:1034B0005EF05CF8D6F8103F93F8CB301BB9354B73
:1034C00000221A80F8BD95F8943ADB07FAD4D6F8B2
:1034D000EC0E03689B6B98470028F0D096F9E03E0D
:1034E000002BECDB2B4E33884BB9B5F9863A33B160
:1034F000642213FB02F3D5F868299A42E2DB3846CE
:103500005EF0A4F8D5F890399FED237AD3ED367AA2
:1035100067EE877AB3EE0E7AF4EEC77AF1EE10FA20
:1035200005D83388002BCDD0013B3380CAE7B4F9EE
:10353000A4301BB9B4F8A230A4F8A4303388B4F88E
:10354000A420B4F9A400154993423CBF0133338051
:103550003388D5F84029012B01D10A60B2E7096808
:103560009142ACDD18B9B4F8A220A4F8A420B4F8B4
:10357000A4209A42A6D8002333804EF0A9FB022251
:103580000C214EF05DF92046BDE8F840FFF75ABF28
:103590000AD7233C3C880020E02E65423888002072
:1035A00008B500F5804292F9803A6BB300F50053FC
:1035B00093F9E03E002B0EDA00F53350134A062152
:1035C000043051F0CFFB4EF083FB0322BDE80840EE
:1035D0000F214EF035B9B2F9863A8BB1D2F868298D
:1035E000642113FB01F39A420ADA00F53350084ACA
:1035F0000121043051F0B6FB4EF06AFB0222E5E7F0
:10360000BDE80840FFF71EBF08BD00BF2CA90C088D
:103610003EA90C0870B52DED028B00F500555B4EF0
:10362000D5F8103F93F8CB308CB0044633B195F900
:10363000E03E002B02DB95F9F6312BB900233380F5
:103640000CB0BDEC028B70BD00F5A04393F8743351
:10365000002BF3D101F054FB00287ED1D5F8EC0EFD
:1036600003689B6B98470028E8D004F592404430EB
:1036700051F00EF828F0F8FCF0EE087AB4EEE70A04
:10368000F1EE10FAF0EE408AD8DA04F5805303F533
:10369000A16203F20C53D3ED007A92ED000A20EE02
:1036A000270AAAF0DFFFDFED3A7A20EE270AB2EE12
:1036B0000E7AB4EEC70AF1EE10FABFD904F58043D2
:1036C000D3F8903993ED368A28EE278AF3EE0E7AF6
:1036D000B4EEE78AF1EE10FAB0D9002309A904F597
:1036E000965009930A930B930EF062F900283DD18E
:1036F0003388B4F9A42001339BB23380002A40D030
:10370000B4F8A420B3EB420F9ADB4EF0E1FA0122A9
:103710000C214EF095F81F4B002218EE900ACDE9CF
:103720000623F8F7F9FE1C4BCDE90401002218EE40
:10373000100ACDE90223F8F7EFFE04F53354043400
:10374000CDE90001154A2046002151F00BFB012272
:103750000C211348FAF730FC72E7D5F8EC0E036839
:10376000DB6C984700287FF479AF67E709A828F059
:103770007BFCF2EE047AB4EEE70AF1EE10FAB7DB66
:103780005CE7B4F8A220A4F8A420B9E734880020AC
:10379000E02E65420000084000003E4054A90C089D
:1037A0001C580020F0B52DED028B8BB00023079341
:1037B0000893099305AB019307AB0446009302AA53
:1037C00004AB03A900F596500EF00AF804F5005674
:1037D000054686F8B80C28B9002528460BB0BDEC84
:1037E000028BF0BD87F0E0F8D6F8BC3C9FED2E7A56
:1037F000C31A07EE903AF8EE677A074667EE877AC3
:1038000004F5325006AA02A91430CDED067A50F024
:103810008BFF04F5325006AA03A920308DED020A71
:1038200050F082FF04F5325006AA04A92C308DED29
:10383000030A50F079FF96ED7E8AC6F8BC7CB5EE9F
:10384000C08AF1EE10FAC7D9DDED080A9DED070A2E
:10385000AAF0D4FDDDED090AAAF0D0FDDDED037A72
:1038600038EE087AB4EEC08AF1EE10FAB4EEE77AD8
:1038700094BF01230023F1EE10FA0AD80233DDEDE4
:10388000027AB4EEE78AF1EE10FA0AD8002BA3D040
:10389000A3E7B4EEE78AF1EE10FA9CBF0133DBB286
:1038A000EDE7012B99D897E7BD37863570B500F560
:1038B0000055044695F8053F43F0040385F8053F9D
:1038C0004EF006FA012211214DF0BAFFD5F8103F53
:1038D00093F8CB30002B41D0D5F8EC0E03681B6871
:1038E000984709280AD1204607F0C4FA30B104F5F8
:1038F000B2400430BDE8704007F0A4BA184BD3F8CA
:10390000EC0E03681B69984740B995F9F531032B14
:1039100024D10621204607F099FA0DE095F9F5111A
:103920000229F6D195F8053FDB07F2D4062220469E
:1039300001F0F6FF0028ECD00A4BD5F8EC0E01227E
:103940005A7303681B6C9847034604F53350064AC4
:10395000BDE870400221043051F004BA70BD00BFD0
:10396000D84B0020B589002088A90C0808B500F5BF
:10397000005292F8053F590717D56FF3820382F87A
:10398000053F0A4B5A7B42B1002200F533505A736F
:103990000221074A043051F0E5F94EF099F9BDE8EB
:1039A0000840002211214DF04BBF08BDB589002011
:1039B000ACA90C08F0B5054685B0684605F59657E4
:1039C00013F062FD694638460DF0E6FF80B105F55B
:1039D0000053D3ED7E7A384CF5EEC07AF1EE10FA52
:1039E00008D8364A002328462380D373FFF7BEFF4A
:1039F00005B0F0BD2846FFF7D5FE064628460BF079
:103A0000B5F910B928460BF08DF9A378002E18BF30
:103A100000200343DBB2A370002BE9D06378A8BB7E
:103A200083BB23780133DBB2082B237003D14EB361
:103A300038460DF041FF2378092B02D138460DF0AE
:103A400033FF2378092B1DD94FF4857323804EF063
:103A50003FF9022210214DF0F3FE86F0B1FF6368BA
:103A6000C01A47F23053984209D905F53350144A29
:103A70000221043051F076F986F0A2FF60602846FA
:103A8000FFF714FF0D4B6278DA73B1E72678002E4A
:103A9000F8D0013EF6B22670002BF3D0002EF1D103
:103AA00066704EF015F9324610214DF0C9FE2846D9
:103AB000FFF75CFFE6E700BF40880020B5890020E3
:103AC000C4A90C0800F5005393F8053F5B0701D526
:103AD000FFF7ECBE7047000073B5044601A900F57E
:103AE000965004F500550DF0C5FCD5F8803C834296
:103AF00006460CD004F58043D3F8900979F054FCC5
:103B0000C5F8806C4EF0E4F83E214DF079FE04F5E6
:103B1000805695F9841C96F9D02596F8D0359142B7
:103B20001BD0FF2B19D004F58043D3F8900979F00E
:103B30003BFC96F8D03585F8843C4EF0C9F895F8F2
:103B4000842C18214DF07CFE042104F5335095F9A6
:103B5000843C034A084451F005F902B070BD00BF2F
:103B6000D4A90C082DE9F0438FB0054686F028FF54
:103B70000023059306930793089309930A930B93E5
:103B80000C930D9304AB019305F5965903AB009389
:103B900007460BAB08AA05A948460DF001FEDFED6C
:103BA000477A9DED077AB4EEE77AF1EE10FA064611
:103BB00030DB9DED0A7AB4EEE77AF1EE10FAACBF95
:103BC0000124002405F50058484698F8B83C002B1D
:103BD00008BF00260DF0F6FD8146EEB94C4698F977
:103BE000843A012B29D164B1D8F8103F93F8CB4027
:103BF0003CB1D8F8EC0E03685B69984780F001048B
:103C0000E4B298F8882CCABBCCB9C8F88C7C0FB049
:103C1000BDE8F0830024D5E7002CDFD005F5325055
:103C2000203050F011FD90ED007AF7EE007AB4EEFE
:103C3000E77AF1EE10FAD2DCD0E70024E1E7D8F819
:103C40008C3CF81AB0F57A7FE1D9012405F5804360
:103C5000C8F8902C88F8884CD3F8983983F80C442D
:103C60004EF036F822461D214DF0EAFD144A05F5C6
:103C700033500221043051F075F8C8E714B1C8F888
:103C8000907CC4E7D8F8900C43F69823381A9842F1
:103C9000BDD905F58043C8F88C4C88F8884CD3F81A
:103CA000983983F80C44C8F8904C4EF011F822462D
:103CB0001D214DF0C5FD034AD9E700BF00000034C7
:103CC000ECA90C0806AA0C080B4B10B501220446FF
:103CD0005A7286F075FE04F5A042D2F86033C31A1A
:103CE000142B08D9C2F8600304F593501030BDE8D6
:103CF000104040F065B810BDB58900202DE9F743AC
:103D0000044604F5005500F50750002330300DF14E
:103D100007018DF8073043F0C1FED5F8100F90F978
:103D2000C030026883B3083BDBB2012B96692BD904
:103D30003221B04704F1100011F0B2FA1F4B04F524
:103D400033581F684FF0000908F10408F86A036847
:103D5000DB69984701281CD186F032FE41F2873397
:103D6000A0EB09029A42064605D9154A06214046AB
:103D700050F0F8FFB1462046FFF7A6FFB86A036887
:103D800003215B689847E1E79369B5F80412984707
:103D9000D0E70121D5F8100F7FF08EF9D5F8100F7C
:103DA0000368DB6A98475AF09BFAF86A03681B6855
:103DB000012103B0BDE8F043184700BFF887002099
:103DC00024AA0C0870B5044600F533502DED028B83
:103DD000174A184E9FED188A0621043050F0C2FF92
:103DE0002046FFF78BFF2046FFF76EFF20460AF0C4
:103DF00011FD3368986A036803215B6898475AF09D
:103E0000D1FD05465AF068FD04F50053D3F8282B80
:103E1000D3F8100FB2F9082000EE102AB8EEC00A4D
:103E200020EE080A80F022FE28465AF05DFDDAE70F
:103E300048AA0C08F88700206F12833A2DE9F04752
:103E4000044600F533502DED028B2A4ADFF8AC9082
:103E50000621043050F086FF2046FFF74FFF5AF04E
:103E6000A1FD04F5005605465AF036FDB7EE000AEE
:103E7000D6F8100F80F0FAFD28465AF035FD86F08E
:103E80009FFD41F2873A074686F09AFDC01B5045D8
:103E9000D9F8008017D99FED188A28465AF01CFDE2
:103EA000B0EE480AD6F8100F80F0E0FD28465AF030
:103EB0001BFD2046FFF708FFD8F828000368032100
:103EC0005B689847E9E728465AF006FDB7EE000A16
:103ED000D6F8100F80F0CAFD28465AF005FD20469E
:103EE000FFF7F2FED8F82800036803215B689847C3
:103EF000CAE700BF78AA0C0800000000F88700207D
:103F00002DE9F34100F500550446D5F8103F93F92B
:103F1000C030032B29D0354F652600F5A048013E5F
:103F200016F0FF060CD0D8F85C334BB93B68986AA2
:103F3000036814215B68984720460AF06BFCEEE7A3
:103F400004F5315001210430F9F72AFE95F9F031DA
:103F500070B953B1092B08D08DF8070004F507504C
:103F60000DF10701303043F099FD02B0BDE8F0815A
:103F7000032B34D8DFE803F002252D30D5F8283B99
:103F8000B3F9082040F2B5339A422ADD04F5075010
:103F900001250DF1070130308DF8075043F07EFD0B
:103FA00004F53350124A0221043050F0DBFE114B6D
:103FB0005D720E4B1C68A06A036805215B68984718
:103FC000F9E7D5F8283BB3F9082040F2B5339A4217
:103FD00007DD2046FFF7F6FE2046FFF72FFF092BEF
:103FE000C3D000238DF80730B8E700BFF887002062
:103FF0009CAA0C08B58900200B4600F5335004211B
:10400000014A084450F0AEBEBCAA0C0810B50446E4
:104010004DF05EFE002205214DF012FC04F53350F8
:104020000421BDE81040024A084450F09BBE00BF86
:10403000C8AA0C0813B50B464AB1042100F5335049
:1040400000920844044A50F08DFE02B010BD02B048
:10405000BDE81040FFF7D0BFE0AA0C0808B5042166
:1040600000F53350054A084450F07CFE4DF030FE18
:10407000BDE80840002208214DF0E2BBF4AA0C087C
:1040800038B504460D4686F09BFC04F500533DB957
:10409000D3F8FC2EC3F8000F0AB9C3F8FC0E38BDE4
:1040A000D3F8002F801A642882BF0022C3F8002FA3
:1040B000C3F8FC2EF3E7000037B5044600F5924044
:1040C00074307EF03FF804F50052C0F3803592F86A
:1040D000E23EC3F34001A9421DD065F3410304F55C
:1040E000335482F8E23E04346DB14DF0F1FD02220A
:1040F0000B214DF0A5FB094A0221204603B0BDE883
:10410000304050F02FBE4DF0E3FD2A460B214DF01C
:1041100097FB034AF0E703B030BD00BF0CAB0C08BF
:1041200028AB0C0838B50A460C460621054601F0B6
:10413000F7FB28B1054A137843F00803137038BD24
:1041400021462846BDE8384006F080BED4890020CC
:1041500038B50A460D461521044601F0E1FB28B1A9
:10416000094A137843F00803137038BD042104F59D
:1041700033500844054A50F0F5FD29462046BDE875
:10418000384006F063BE00BFD489002038AB0C086D
:1041900038B50A460D461521044601F0C1FB28B189
:1041A000094A137843F00803137038BD042104F55D
:1041B00033500844054A50F0D5FD29462046BDE855
:1041C0003840FFF7AFBF00BFD489002060AB0C08B8
:1041D00038B50A460D461B21044601F0A1FB28B163
:1041E000094A137843F00803137038BD042104F51D
:1041F00033500844054A50F0B5FD29462046BDE835
:104200003840FFF78FBF00BFD489002076AB0C0881
:1042100038B50A460D461121044601F081FB28B14C
:10422000094A137843F00803137038BD042104F5DC
:1042300033500844054A50F095FD29462046BDE814
:10424000384006F003BE00BFD489002088AB0C08BC
:1042500010B500F5005494F8E23E9A0623D4D4F841
:10426000EC0E03681B689847032808D005D802287D
:104270000ED194F8E00EC00914E01B28F9D194F88F
:10428000E00E00F0A000A0F180035842584109E080
:10429000B4F8E00E20F4FE4020F07F0080B2003839
:1042A00018BF012010BD0120FCE7000038B500F563
:1042B0000055044695F8053F184A43F0080300F5F9
:1042C000335085F8053F0221043050F04BFD4DF08E
:1042D000FFFC012217214DF0B3FA2046FFF7B8FF8B
:1042E00040B104F531500122BDE8384015210430B9
:1042F000F9F762BED5F8EC0E03681B6898470628EC
:1043000006D104F5B4401C30BDE8384007F0A6BF24
:1043100020460B21BDE83840FFF704BF9CAB0C08DA
:1043200070B500F500550646D5F8FC2ED5F8003FCF
:104330009B1A41F28832934211D9D5F8EC0E0368EA
:104340001B6D9847044695F8053FC3F3C003A3428D
:1043500013D034B13046BDE87040FFF7A7BF00244A
:10436000F1E74DF0B5FC224617214DF069FA95F8BA
:10437000053F64F3C30385F8053F70BD0B46013B61
:104380001146062B18D8DFE803F00406080A0C13C0
:10439000150006F05BBDFFF7C5BEFFF7F9BEFFF7DE
:1043A000D7BE00F53150012214210430F9F704BEC4
:1043B000FFF70EBFFFF72CBF7047000070B5044633
:1043C00004F500554DF084FC012205214DF038FA2A
:1043D00095F8DA31072B98BF304A204694BFD65C57
:1043E0000126FFF735FF68B12D4A2E492046FFF719
:1043F00021FE04F53150012210210430F9F7DCFDD3
:10440000002614E0D5F8EC0E0368DB6C9847A8B1E1
:1044100004F5405393F8652482B193F96434012B79
:104420000CDC214A21492046FFF704FE01263146D3
:1044300020460322BDE87040FFF7A0BFD5F8EC0E80
:104440000368DB6C984718B1D5F8883A190715D47A
:10445000D5F8EC0E03681B689847032803D1D5F8FC
:10446000883ADA070DD4D5F8EC0E03685B6A9847F2
:1044700068B90C492046FFF7BFFDD8E70A4A094949
:10448000D1E70B4A07492046FFF7D4FDB8E7D5F836
:10449000883A5B07EDD5074AF4E700BF84AC0C0807
:1044A000BCAB0C08C6AB0C08CCAB0C08DFAB0C08E3
:1044B000EFAB0C08FFAB0C0870B5044615464DF089
:1044C00007FC012206214DF0BBF92046FFF7C0FE94
:1044D00098B104F53150012207210430F9F76CFD41
:1044E000134A14492046FFF7A5FD0025294620461A
:1044F0000422BDE87040FFF741BF04F50056EDB25D
:10450000D6F8EC0E0368DB6C984758B1D6F8883AB9
:104510001B0707D535B1084A06492046FFF78AFD33
:104520000125E3E703492046FFF766FDDEE700BF0C
:10453000BCAB0C081EAC0C08CCAB0C08F8B50446A0
:1045400004F500554DF0C4FB012208214DF078F927
:1045500058F026FC95F8C931072B9CBF364AD65C2B
:10456000D5F8103F93F8CB7088BF02265FB9334966
:104570002046FFF741FD0026314620460522BDE8D2
:10458000F840FFF7FBBE2046FFF762FE60B104F57E
:104590003150012212210430F9F70EFD284A274933
:1045A0002046FFF747FDE6E7D5F8EC0E0368DB6C25
:1045B000984778B104F5405393F8652452B193F9C4
:1045C0006434012B06DC1F4A1F492046FFF732FDE9
:1045D0000126D1E7D5F8EC0E0368DB6C984718B1DB
:1045E000D5F8883A190713D4D5F8EC0E03681B6880
:1045F0009847032803D1D5F8883A9A070BD4D5F801
:10460000883ADB0609D40D492046FFF7F5FCB3E7ED
:104610000C4A0A49D9E70D4AC1E7D5F8EC0E036800
:10462000DB69984705460028EDD1094A0349204631
:10463000FFF700FD2E469FE78CAC0C08E7970C08AF
:10464000BCAB0C08CCAB0C0818AC0C0826AC0C08A6
:104650003BAC0C0870B500F50055044695F9C9311E
:10466000ABB3D5F8706E96B386F0AAF905F52E6354
:1046700093ED000ADFED167A9FED161ADFED160AAC
:10468000861B20EE270A8D2023F004FFBCEEC00A13
:1046900010EE103A9E420CD295F8053F9A0716D5B7
:1046A00020460021F9F7E2FD2046BDE87040FFF703
:1046B000D5BC0CD995F8053F9B0708D420460121AD
:1046C000F9F7D4FD2046BDE87040FFF737BF70BD55
:1046D00000007A440000804F000000002DE9F34103
:1046E000074600F5924074307DF02CFD07F500542C
:1046F000C0F38048019086F063F994F8083F434581
:10470000454606460DD007F5335084F8088F04302F
:10471000002D3FD03A4B3B4AC4F80C6F022150F0B9
:1047200021FB94F8083F43B394F8093F2BBBB4F93D
:10473000F63A9FED350A9FED351ADFED350A07EEA3
:10474000903AF8EEE77A40F2571027EE800A23F00D
:10475000A1FEBCEEC00AD4F80C0F10EE103A361AC7
:104760009E420AD9012307F5335084F8093F294AAC
:10477000234B0221043050F0F5FA94F9F53A002B5E
:1047800094F8053F0DDC6FF3451384F8053F02B044
:10479000BDE8F0811A4B204AC4F80C8F84F8098FC9
:1047A000BCE7C3F34012AA42F1D065F3451384F885
:1047B000053F9B06EBD5194BD3F8EC0E03681B693C
:1047C00098470028E3D04DF083FA01221F214DF0D5
:1047D00037F83846FFF73CFD48B107F53150012264
:1047E0002121043002B0BDE8F041F9F7E5BB94F8AF
:1047F000F51A3222384602B0BDE8F041FFF7BEBDDF
:1048000054AC0C0863AC0C0800007A440000804FE4
:104810000000000079AC0C086EAC0C08D84B0020EE
:1048200008B5044B01221A7086F0BEF8024B1860DE
:1048300008BD00BF498800204C880020014B0022A1
:104840001A707047498800202DE9F041044686F02F
:10485000ABF82A4BB4F8BE201988294E9142054680
:104860000ED01A80274B18603378A3B1002434701F
:104870004DF02EFA22461321BDE8F0414CF0E0BF86
:104880003378214FDBB93B782BB11E4B1F4A1B6895
:10489000C31A934201D8BDE8F0810123337004F5B7
:1048A0000053D3F8100F90F8CB3013B103689B6A14
:1048B00098474DF00DFA012213214CF0C1FF3B78CF
:1048C000002BE8D03378002BE5D00E4A104913684E
:1048D000EB1A8B42DFD904F500541560D4F8100FA1
:1048E00090F8CB30002BD6D000217EF0E5FBD4F839
:1048F000100F0368BDE8F0415B6A18474A88002042
:10490000488800204C8800204988002080841E00B0
:1049100040420F002DE9F04100F500550446D5F85E
:10492000EC0E95F8DC700368DB6C9847014650B9D3
:1049300095F9E03E002BA5BFD5F8103F93F8CB00CA
:10494000012180F0010104F5025808F120084046D9
:1049500062F0F4F8D5F8103F93F8CB300646002B00
:104960007BD0002865D03E4B93F9E03E002B04DB62
:1049700002463C49404661F0BBFC95F9A67057B130
:1049800095F9E03E002B0EDA04F5315001220F219B
:104990000430F9F711FB4DF09BF93246BDE8F041C8
:1049A00009214CF04DBFD5F8EC0E03685B699847C0
:1049B00058B195F9E13E002B07DA95F8053FDA0783
:1049C00003D495F8DC30DB07DED53146404662F093
:1049D0001BF9DFED257AB4EEE70AF1EE10FA05DDFA
:1049E0000A220921204600F09BFFD4E7023F032F53
:1049F00011D801A353F827F0E1490108094A010839
:104A0000274A01082D4A01080A221521204600F0F4
:104A100087FF0028BFD10A220621204600F080FF30
:104A20000028B8D1DCE70A221121F6E70A22152175
:104A3000F3E797B195F8DC307BB9094B93F9E03E89
:104A4000002B06DB04F53350084A0521043050F0F2
:104A500089F94DF03DF90022A0E7BDE8F08100BFE3
:104A6000D84B002094AC0C080000C8429DAC0C0848
:104A700070B500F5005300F59245743586B093F893
:104A8000881C044628467DF00BFB02A812F0FCFCB3
:104A900002A904F596500CF02FFF04F58043049A08
:104AA000C3F86C29059AC3F8702928467DF04AFBA3
:104AB00082061AD528467DF053FB04F59245FDEE9B
:104AC000C07A643504F5805417EE901A0222284605
:104AD00017EE906A12F0DEFC94F83C35DB0706D442
:104AE00001223146284612F0D5FC06B070BD0121E6
:104AF000284612F093FD0028F2D0F6E770B500F5D5
:104B0000A04486B0B4F890338B420D46164603D1CC
:104B1000D4F88C33934221D085F052FFD4F88833F7
:104B2000C31A132B1AD9C4F88C63A4F89053C4F891
:104B300088034DF0CDF8044685F04AFF084B094A3A
:104B40001B68CDE90453084B0193084B0093CDE952
:104B50000201074B074920464CF0FCFC06B070BD33
:104B600050880020B4AC0C08CCAC0C086E820C0849
:104B7000B4650C08C7AC0C0838B500F500540D46F8
:104B800094F8E13EC3F380138B420BD021B14DF07A
:104B90009FF811214CF034FE94F8E13E65F3861342
:104BA00084F8E13E38BD0000F0B52DED048B00F532
:104BB00000558BB0D5F8103F93F8CB30064600F582
:104BC0008044002B67D095F9E03E002B63DBD5F8DD
:104BD000EC0E03685B699847002861D1D4F890090E
:104BE0009FED430A6C3026F041FE0AAACDED080A7B
:104BF0008DED091A8DED070A12E9070004AB01AF2C
:104C000083E8070087E80700384626F09DFBD4F8C4
:104C1000903906F592404430D3ED368AB0EE409A92
:104C20004FF036FD27F020FAD4F89839D5F8EC0E7D
:104C3000D3EDDB9A0368DB6CB0EE408A9847DFED7A
:104C40002D7AB4EEE79AF1EE10FA02DC95F8E83E20
:104C50000BB1002838D0DFED287A68EEA78AF3EE92
:104C60000E7AF4EEE78AF1EE10FA2DDCF0EE087A17
:104C7000B4EEE78AF1EE10FA26DCF5EEC09AF1EE1A
:104C800010FA21DAD4F8900903689B6F98470BB0AB
:104C9000BDEC048BF0BDD4F8900903689B6F0DE068
:104CA000D5F8282BD4F89009B2F908200368002A17
:104CB00003DCD5F8E42E022AF0D1DB6F0BB0BDEC9B
:104CC000048BBDE8F0401847D4F89059DFED0B0A8B
:104CD0002B68D3F88060D4F8983940F2AB1093ED8C
:104CE000C90AB7EE001A23F0D5FB2846B047CEE735
:104CF0009F0CB3450080BB44E02E654200000000DD
:104D000000F5005090F8E80E70470000F8B500F587
:104D10000054064694F8E03EB1EBD31F0D4644D054
:104D2000224B00221A6000293BD04CF0D1FF122107
:104D30004CF066FD94F8E03E65F3C71385F001077B
:104D400084F8E03E6DF096FD39466DF06FFD37B1A9
:104D500094F85E311BB985F033FEC4F8600184F825
:104D60005E7115B3B4F8AC315B071ED5D4F8103FB3
:104D700093F8CB30CBB1D4F8EC0E03685B6998475D
:104D800098B9D4F8EC0E036820219B69984760B16C
:104D900006F531500122BDE8F8400D210430F9F745
:104DA0000BB94CF095FF1C21C2E7F8BD50880020DC
:104DB0002DE9F04F2DED0A8B00F500558DB0D5F89B
:104DC000103F93F8CB6000F5A042044601921EB953
:104DD0000121FFF79BFF0BE095F9E02E002A66DA30
:104DE000D5F8EC0E03689B6C98470646002842D025
:104DF0004FF0000B95F9E02EB44E002AC0F2598115
:104E0000D6ED007AB4F9A420B8EE677A1AB9B4F8EE
:104E1000A220A4F8A420B4F8A430DFEDAD6A07EE18
:104E2000903AF8EEE77A67EEA67AB4EEE77AF1EE1A
:104E300010FAACBF012100212046FFF79DFE95F935
:104E4000E02E002A95F8E12EB8BF4BF0010B530677
:104E5000019B93F8742348BF4BF0020B0AB14BF04F
:104E6000080B3268594620460DB0BDEC0A8BBDE8F0
:104E7000F04FFFF743BED5F8103F204693ED0C8A64
:104E8000F9F7C6FAB4EEC80AF1EE10FAB0D5D5F8C3
:104E9000103F93F8A130032BAAD14BF0CFF84FF479
:104EA000801142224BF082F83146204691E7019A68
:104EB00092F87493B9F1000F03D0844A0023136071
:104EC00096E700F5804A93F80780DAF890090368BE
:104ED0005B6F984707460090D5F8EC0E03685B6956
:104EE000984720B1D5F8E43E022B00F0E480B8F1F9
:104EF000000F0CBF4FF0000B4FF4007BB7EE00BA71
:104F000017B14BF4806B009604F59547203738466F
:104F100064F0F2FF0130DAF890099FED6E0A9FED20
:104F20006ECADFED6E8A0CBF012302236C3008EEDF
:104F3000103A26F09BFC0CABCDED0A0A8DED0B1A56
:104F40008DED090A13E907000DF10C0E0DF1180C97
:104F50008CE807008EE80700704626F0F5F904F5A6
:104F60008042DFED5F7AD2F8902992ED36AA2AEEE0
:104F700027AAB4EECC0AF3EE0EBAF1EE10FA04F55D
:104F80009240B4EEEBAAC8BF4BF4807B4430F1EE04
:104F900010FAC8BF4BF4807BF0EE40AA4FF078FBCC
:104FA00027F062F8B8EEC88A04F59240B4EEC80A59
:104FB000F1EE10FA00F1740098BF4BF0800BF0EEA8
:104FC000409A7DF0D9F868EE288AB0EEC09AB4EE27
:104FD000E89AF1EE10FA204648BF4BF0400B09F07A
:104FE00001FD002847D14BF0200BB246384664F053
:104FF00083FF012850D14BF0100BB1463349B8F173
:10500000000F54D0009B002B51D0F4EECCAAF1EE4F
:1050100010FA4CDCB4EEEBAAF1EE10FA47DCF4EE39
:10502000C89AF1EE10FA42D8B4EEE89AF1EE10FA0E
:105030003DD5BAF1000F3AD0B9F1000F37D00A6868
:10504000B4F9A40007EE902AB8EE677A18B9B4F85C
:10505000A200A4F8A400B4F8A43007EE903AF8EE49
:10506000E77A67EE8B7AB4EEE77AF1EE10FA19D5AB
:1050700001320A60BEE604F52D5004304FF0E4FA28
:10508000DFED187A90ED007AB4EEE77AF1EE10FADF
:10509000A9D44FF0000AA9E7384664F02DFF01308B
:1050A000ACD1A8E701212046FFF730FEA2E600229E
:1050B000DFE70121C0E6B8F1000FB0EE08BA0CBF7F
:1050C0004FF0000B4FF4007B1BE700BF508800201F
:1050D000CDCC4C3E9F0CB3450080BB440000C84281
:1050E000E02E65420000484330B500F5B053103360
:1050F000044693E8070089B002AD85E807009FEDFC
:105100001D7ADDED047A77EE877A9FED1B7ACDED7F
:10511000047AD4ED2B7AF0EEE77AF4EEC77A04F550
:105120009240F1EE10FA00F144000BD5B4F9A23030
:1051300007EE903AF8EEE77AF7EE006A86EEA77A85
:1051400084ED2B7AD4F8AC30019301AA29464FF0B4
:1051500011FB2046FFF72CFE2046FEF781F9204682
:10516000FEF758FA2046FEF71FF82046FEF7C8F86B
:1051700009B030BD0AE81C410000003410B50446F7
:105180002DED028B1D2059F02BFA60B304F500536E
:10519000D3F8EC0E00F0C2FA192108EE100A04F55B
:1051A000516043F017F902281AD00338012808D8B3
:1051B00004F52D5004304FF047FA90ED008ABDEE13
:1051C000C88AB8EEC88A9FED090A28EE000ABDEC2D
:1051D000028B04F595402030BDE8104064F012BF0A
:1051E0009FED038AEDE7BDEC028B10BD0AD7233C8F
:1051F00000000000134A0260134A426002F1740189
:1052000081601249C16002F5205101610839416194
:1052100024398161A2F56E61C1610D49016202F517
:105220005761416202F51861816202F68411C16220
:1052300002F6881102F68C124263064A0163826309
:10524000704700BF00BE0C08784D00207475002028
:1052500068750020F02C00201C2953D8DFE801F0ED
:10526000130F171B27232F1F522B52335252373B3A
:105270003E424652524A5252525252524E0000F54B
:10528000A7401830704700F5B5402830704700F54A
:10529000A7405830704700F5A8401430704700F51B
:1052A000AF407030704700F5B2404C30704700F5A9
:1052B000B1404030704700F5B2400430704700F50F
:1052C000B4401C30704700F5B0403030704700F5F6
:1052D000B0406C30704700F5AB40FAE700F5B340E2
:1052E0000830704700F5AF402C30704700F5B540EE
:1052F0006430704700F5B6403430704700F5B74071
:10530000503070470020704773B50B6805461B6C22
:1053100008460C46164698470421034605F53350C7
:105320000E4A009608444FF01DFD4CF0D1FC236856
:1053300005461B68204698470A21024628464CF03D
:105340007FFA074B93F8E13E9B0641BF054A13786D
:1053500043F00403137002B070BD00BFD0AC0C0862
:10536000D84B0020D489002038B50C4A18230546B4
:105370000C464AF0D5FC78B121462846FFF76CFF71
:1053800030B10146064A2846FFF7BEFF002038BD6F
:1053900028464AF00DFCF9E70120F8E750AD0C086B
:1053A000F0AC0C0810B500F50054002384F8D83B8D
:1053B000084B00F5804093F8E01ED0F89009C90929
:1053C00076F09EFCD4F8EC0E0368BDE81040DB6874
:1053D000184700BFD84B002070B505460868036821
:1053E0005B690C461646984790B1306803685B6964
:1053F000984768B905F50053D3F8102F92F8CB20E1
:1054000032B193F9E03E002B02DB2846F9F716F89B
:1054100004480AF099F820680368BDE870409B686A
:10542000184700BF1089002070B500F500550446EC
:10543000D5F8EC0E0B4E0368DB6998473074D5F84D
:10544000EC0E03681B689847F070D5F8EC0E036803
:105450005B6C9847014604F593501030BDE87040EE
:105460003EF0F8BCB589002070B52DED028B244BC1
:1054700093F8053FDB0782B006460D461446B0EEB2
:10548000408AF0EE608A06D500232B60236002B0CC
:10549000BDEC028B70BD57F083FD037F002BF3D072
:1054A000F36A9FED181A1B689FED170AB3F90830CD
:1054B00007EE103AB36A1B68B3F9083007EE903A6A
:1054C000B8EEC77AF8EEE77A67EE000A68EE811A5E
:1054D00027EE800A28EE011A01A9684623F0CEFEC5
:1054E000DFED0A6A9DED007ADDED017A27EE267A7E
:1054F00067EEA67A85ED007AC4ED007AC7E700BFB3
:10550000D84B00200AD7233C530469390000C84215
:1055100070B52DED028B88B0002302930393364BB8
:1055200093F8053F13F0010F0646B0EE408A06AD32
:1055300002AC03D157F034FD037F5BB994E803005C
:1055400085E803009DED060ADDED070A08B0BDEC15
:10555000028B70BDB36ADFED296A1B68B3F90830AE
:1055600007EE903AF36A1B68B3F9083007EE103A79
:10557000B8EEC77AF8EEE77A27EE267A67EEA67AD3
:10558000F1EE476ACDED026ADFED1D6ACDED037ADB
:10559000B0EEC77AB4EEE67AF1EE10FA06D5F0EE88
:1055A000E77AF4EEE67AF1EE10FAC7D403AA2146C0
:1055B0001448F8F773FFDDED027A9DED037AF0EE03
:1055C000E77AB0EEC77AF4EE477AF1EE10FACCBF84
:1055D000B0EE670AB0EE470A204625F003FE04A8A5
:1055E0008DED040ACDED050A25F0AEFE204688EECD
:1055F000000A25F027FEA1E7D84B002053046939A3
:1056000000000034D82B0020094B93F9E02E002A2B
:105610000CDAB5EEC00AF1EE10FA07D9D3F8103F54
:1056200093F8A100C31E58425841704700207047AC
:10563000D84B0020436A1B6893F8CB3043B1054B2D
:1056400093F8E00E00F0A000203818BF012070474A
:1056500001207047D84B002010B5436A04461868F3
:10566000D1B102217DF038FD236A9FED0C1A186834
:105670000368F0EE410ADB6AB0EE410A9847236AFC
:10568000074A1868D2ED6A0A03689FED040A5B6E48
:10569000BDE81040002118470121E3E700000000A9
:1056A000D84B002010B5436A04461868002930D052
:1056B00002217DF011FD236A186876F0F1FA636A21
:1056C0001B6893F8A130012B04D8236A01211868C4
:1056D00077F080F8636918687AF08CF96369186864
:1056E0007AF0E8F963699FED0C0A18687AF00EFC0D
:1056F000636918687AF07CFC236A9FED071A1868C2
:105700000368BDE81040DB6AF0EE410AB0EE410AE2
:1057100018470121CDE700BF0000000013B5044683
:1057200001A90C4809F0EEF910B1019802B010BDC2
:105730006369186879F068F818B9074BD3F86809F5
:10574000F4E7064801AA032111F0DAFE0028F4D09C
:10575000EBE700BFD82B0020D86B00203C75002061
:1057600070B504462DED028B00296AD18368B3F928
:105770006258642DB8BF6425FFF7D0FFA842626865
:10578000A4BF324B93F8E15EB2F93430ACBFC5F33D
:1057900080150125002BDBBF63691B685B4293ED1D
:1057A000C48AC8BF07EE903AB2F93230C8BFB8EE2B
:1057B000E78A002BB8BF5B429BB25B4207EE903A90
:1057C000A368F8EEE77AB3F96268F4EEC87AF1EE0E
:1057D00010FAD8BFB0EE678A2046642EB8BF6426A0
:1057E000FFF79CFF6369A26B1B68D2ED001A93ED73
:1057F000C61AD3ED0E0A311A00EE101AB8EEC00A1E
:1058000023F02AF96368B3F93230002BB8BF5B424A
:105810009BB25B4201EE103A40F29720B8EEC11AFB
:10582000F0EE480A22F036FE63692946186879F0DE
:105830008FF8BDEC028B6369BDE8704018687AF0A0
:10584000D7BB9FED030A0025EEE700BFD84B002031
:1058500000000000436A186803681B6918470000CD
:1058600038B52DED028B03680446D3F88030984795
:10587000236B2A481B68F0EE408AB3F9085009F000
:1058800051F84FF47A72041E4FF000012846D8BF39
:105890004FF4FA7422F03CFE8442B6EE000A2ADD90
:1058A00007EE900AB8EEE77A07EE904A27EE007A04
:1058B000F8EEE77A87EE278A4FF46D7038EEC00A6B
:1058C000F5EE087AB1EE400A80EE270AB7EE001A2C
:1058D000FEEE000A22F0DEFDF7EE007A77EEC07AE7
:1058E00028EE000A20EE080A20EE080AA7EE880A31
:1058F000BDEC028B38BD031B07EE103AC4F57A7479
:10590000B8EEC77A07EE904A27EE007AF8EEE77A0B
:1059100087EE278A38EE008ACEE700BFD82B00201A
:105920002DE9F0472DED028B00F5A04300F5005660
:1059300093F8944383F894230546D6F8EC0E036855
:1059400082B01B68884617469847404521D11A2FD8
:1059500086F85C7109D140B905F5804506F6BC268C
:10596000D5F890393268C3F8FC208C4B93F8E13EAF
:10597000980606D40124204602B0BDEC028BBDE897
:10598000F087BC42F6D0864A137843F002031370C6
:10599000F0E7022F0DD0B8F11B0F12D105F5A8408A
:1059A0003946143002B0BDEC028BBDE8F04701F07F
:1059B00055B941462846FFF7D7FC04460028EAD1EE
:1059C000D9E741462846FFF747FC0446019018B93D
:1059D00028464AF0EDF8CEE7D6F8103F93F8CBA072
:1059E00003685B699847019A05F5B04330338AF044
:1059F00001099A4208BF0120BAF1000F08D10198AD
:105A0000036849465B689847044648BB654A22E0FC
:105A100096F9E03E002B80F2B380002800F0B080C1
:105A2000DFF878A1DAF8EC0E03685B699847044662
:105A3000002840F0A5800198FFF712FFAAF500505A
:105A4000B0EE408AF8F7E4FCB4EEC08AF1EE10FA4A
:105A500040F39680544A01992846FFF755FC8AE79F
:105A600005F53B5101AA2C312846FFF7B5FC0198FA
:105A7000C6F8EC0E86F85C7103681B6898473A46D6
:105A8000014605F57C604BF0EBFA05F5335000213B
:105A9000043056F0BDFB96F9A63023B105F502504F
:105AA000203061F0D5F8D6F8EC0E03681B689847F3
:105AB000C21E05F580435042504106F68C2183F802
:105AC000200AD3F890290968C2F8F81006F6BC211C
:105AD000D3F890290968C2F8FC10B8F1010F02D080
:105AE000B8F10B0F06D106F6A426D3F89039326828
:105AF000C3F8FC202846FFF797FC284B93F8E13EBB
:105B00009B063FF540AF35E796F8A030002B3FF4F9
:105B100076AFB6F8BC30D9077FF571AF96F8DC30B8
:105B2000002B3FF46CAFD6F8103F93F8CB30002B2E
:105B30003FF465AF96F85C310A2B7FF460AF96F9BD
:105B4000E03E002BFFF65BAF184A01992846FFF7AD
:105B5000DBFB00240FE7164809F046F90028D3D1F3
:105B6000D6F8EC0E03685B6998470028CCD0019802
:105B700003685B69984704460028C5D10D4A6AE767
:105B8000019803681B6998470028E4D0084809F089
:105B900019F904460028DED1074A5CE7D84B0020FB
:105BA000D48900202E180E0818AD0C083CAD0C0846
:105BB000D82B00202AAD0C089AC80D080148FFF721
:105BC000AFBE00BFD82B002013B504468DED010AEF
:105BD00064F02AF96369A26B1B6892ED001A93EDD9
:105BE0000E0AD3EDC60A01A962F0ACFF9DED010AD1
:105BF00002B010BD436A186803685B6A184700006A
:105C000038B5436A1C6894F8CB10054661B9204644
:105C10007DF062FA6B6A1B6893F8A10018B1012845
:105C200014BF0320022038BD164803783BBBFFF7A2
:105C3000EBFC20BB144A92F8E03E03F0A003202BBB
:105C400017D0B5EEC00AF1EE10FA10D592F8E23E88
:105C50005B070CD4012120467DF03EFA6B6A1B687D
:105C600093F8A130012B0CBF02200320DBE70221B7
:105C7000F1E7204602217DF02FFA0420D3E701202E
:105C8000D1E700BF10890020D84B002010B52DEDC2
:105C9000028B134B93F8053FDB07044604D59FEDB9
:105CA000110ABDEC028B10BD57F07AF9037F002B6F
:105CB000F5D0636B186857F09DFAA368DFED0A7A98
:105CC00003F6AC0292ED008A03F50B63D3ED000AF4
:105CD00028EE278A23F08CFA28EE000AE1E700BFBD
:105CE000D84B0020000000000000C8420148F8F72F
:105CF00003BC00BFD82B00200148F9F77FB800BFD4
:105D0000D82B00200148FFF70BBE00BFD82B002086
:105D100070B57E4D2DED028B95F8E13E8CB00026DE
:105D2000044658060496059603D56369186878F00A
:105D3000DFFB95F8053FD9075DD463689B899A0717
:105D40001BD573484EF080FCDFED727A90ED007A3F
:105D5000B4EEE77AF1EE10FA0FDD4BF0B9FF3D211A
:105D60004BF04EFD6C4809220521FFF7D9FD20B903
:105D7000092202212046FFF7C5FF636893F95430DA
:105D8000CBB365489FED658AF9F738F8E3689FED76
:105D9000647A1B68D3ED0A7AF4EEC87AF1EE10FA51
:105DA000B8BFF0EE477AB6EE000A27EE800A20462A
:105DB000FFF7AEFB8DED040AB0EEC00AB4EEC80AE0
:105DC000F1EE10FACDED050A06D5F0EEE00AF4EE9C
:105DD000C80AF1EE10FA0ED495F8E23E1B0704D47F
:105DE0004BF076FF49214BF00BFD95F8E23E43F076
:105DF000080385F8E23E95F8E33E09966FF38203C7
:105E000085F8E33E60690A9609AE324604A9006847
:105E1000012378F0D7FB6369186879F04BFE63695A
:105E2000186878F023FFA3688DED060ACDED070A08
:105E30008DED081AD3ED007AF5EEC07AF1EE10FA86
:105E400051DDB5F99C319FED378A00EE903AF8EEBE
:105E5000E00A2046CDED030AFFF760FCA368DDED04
:105E6000030AD3ED001A9FED2B0AB7EE002A07EEC6
:105E7000900A31EE822AB8EEE71A22EE082A61EE85
:105E8000881A22F047FADFED287A20EE270ADFEDA4
:105E9000277A20EE270AA8F081FBDFED257A20EE95
:105EA000270A06A820EE088A25F04EFAB4EEC08A2A
:105EB000F1EE10FA17D5C8EE006A63699DED067A17
:105EC000DDED077A27EE267A67EEA67A8DED067A63
:105ED000CDED077A1B68D3F88823C3F89423D3F851
:105EE0008C23C3F89823236A12491C683046FCF7B8
:105EF0002DFB0B9B009396E80C0006A9204675F03D
:105F000081FF0CB0BDEC028B70BD00BFD84B0020F0
:105F10003075002000002F44D82B002000000034F2
:105F200000007A430000C8420AD7233C35FA8E3C71
:105F30000AE81C410488002013B504460191FFF7CC
:105F4000E7FE0199204602B0BDE81040FFF708BC0B
:105F50000148FEF7DBBE00BFD82B00200048704789
:105F60009C5800200148F8F7B5BA00BFD82B002094
:105F700030B50F4D87B0002304466946D5F898091F
:105F800000930193029378F089FED5F8980902A94D
:105F900078F0D8FE009B0393019B04930222029B9E
:105FA000059303A9204611F0ADFD204607B030BD92
:105FB000D86B0020002070470020704700207047F9
:105FC0000020704700207047002070470020704775
:105FD0000020704700207047002070479FED010AA5
:105FE000704700BF0000000000207047002070478D
:105FF0000020704701207047002070470020704744
:106000000120704700207047012070470120704731
:106010000020704701207047012070470020704722
:106020000048704768AD0C080048704768AD0C0820
:10603000836893F8C038DB0706D5002380F83C302E
:10604000024B0222C3F8E42E01207047D84B0020F7
:1060500090F83C3043B9836893F8C038DB0742BFFF
:10606000034B0122C3F8E42E002380F83C30704734
:10607000D84B0020012380F83C3070472DE9F043D5
:106080002DED0C8BF0EE409A20EE000A97B0002523
:10609000A0EEA00A04468946B0EE41CAF0EE60AA1E
:1060A00090461F4601950295039504950595069522
:1060B000A8F08AFCF7EE00CAB4EEEC0AF1EE10FA92
:1060C000C8BFCCEE807AA36803F67C0203F50863B0
:1060D00092ED009A9FEDC5DAD3ED000AC4BF69EED8
:1060E000A79A6AEEA7AAB0EE690A23F081F8A3681E
:1060F00029EE0D9A03F67C0203F50863D2ED008ABF
:10610000D3ED000A29EE009AB0EE6A0A23F070F887
:10611000A36868EE8D8A03F6940203F69803D3ED24
:10612000000A92ED008A68EE808AB0EE4C0A23F0F5
:106130005FF8636828EE0D8A93F9703028EE008AC4
:10614000002B00F0D980236A9FEDA90A18686C30F3
:1061500025F08CFBB0EE60AACDED080A8DED091A92
:106160008DED070A22F040F9BDEEC0BAA14940F614
:10617000B8321BEE100A22F0BBF9434207EE903A08
:106180006368F8EEE77A93ED1A7A67EE877AB0EEF5
:106190004A0ACDED017A22F027F9FDEEC0BA40F6A9
:1061A000B83294491BEE900A22F0A2F94242636889
:1061B000039507EE902A93ED1B7A93F97030F8EE71
:1061C000E77A022B67EE877ACDED027A6ED18A4BA1
:1061D000B3F99C310AEE103AB8EECBBAB8EECAAABF
:1061E000236AB4EECABAF1EE10FA1A683DDDA3686C
:1061F000DFED820AA16B92ED051AD1ED001A03F6CC
:106200007C0393ED007A27EE0D7A3AEE4B0AC7EE47
:10621000200A22F021FCDDED017A37EE800A8DEDB7
:10622000010AB8EEEB0A236AB4EECA0AF1EE10FADC
:106230001A6834DDA368A16B92ED061AD1ED001A3D
:1062400003F67C03D3ED000A20EE8DDADFED6B0A56
:106250003AEE400ACDEE200A22F0FEFBDDED027A96
:1062600037EE800A8DED020A20E0B1EE4A0AB4EE64
:10627000C0BAF1EE10FAD4D5A368A16BDFED5F0AC6
:10628000D1ED001A92ED051A03F67C0393ED007A26
:1062900027EE0D7A30EE4B0AC7EE200AB9E7B1EED1
:1062A0004AAAB4EECA0AF1EE10FAC3D4236AD3F8AC
:1062B00000C00CF184030FCB12AD85E80F000EAEC9
:1062C0000AAD86E80F0085E80F0004AB01AA294655
:1062D000604676F033FA636893F97030022B16D17A
:1062E000DDED047A39EE279ADDED057A78EEA78A9E
:1062F000DDED067A38EE278A89ED009AC8ED008A2E
:1063000087ED008A17B0BDEC0C8BBDE8F083F0EE92
:10631000E99AF0EEEAAAF4EEE9AAF1EE10FA48BF23
:106320006D46CDED009ACDED0AAAD5ED007ADFEDF0
:10633000340AB0EECCCAF4EECC7AF1EE10FAD8BF43
:1063400035468DED0ECA95ED007ADFED2E7A87EE9B
:10635000270AAD20B7EE001A3CEEC00A22F09AF8E8
:10636000E369D3ED937A04A820EE270A25F07EFA9C
:10637000F0EEC07A8DED061AB0EEC91A31EE671A4A
:106380008DED040AB0EEC11A39EE000ACDED050A12
:10639000B520F1EE410A22F07DF8B0EE409A9DED75
:1063A000050AB0EEE81AF0EEC07A31EE671A38EE60
:1063B000800AB0EEC11AF1EE410ABA2022F06AF862
:1063C000F0EE408A9DED060AB0EEC81AF0EEC07AF3
:1063D00031EE671A38EE000AB0EEC11ABF20F1EEB6
:1063E000410A22F057F8B0EE408A85E70000C84223
:1063F0009F0CB34548F4FFFFD84B002000007A44BF
:106400000000000000A08C4530B52DED028B836AA2
:106410003E4D044687B0186856F0ECFEE36A1868F3
:10642000B0EE408A56F0E6FE636B8DED010A186807
:1064300056F0E0FE05ABB0EE401A03A92046DDEDB4
:10644000010A04AAB0EE480AFFF718FE636A18684A
:1064500090F8CB10002939D17CF03EFE2046FFF7A2
:10646000FFF9636A1B6893F8A1100129B0EE408A16
:106470003BD0032942D051B9236A0121186877F033
:106480005FF8236A186875F0F5FB9FED218A236A8F
:10649000A268186892F8C02803689DED030ADDED34
:1064A000040A9DED051A92074CBFDB6B9B6B984766
:1064B000236AD5ED6A0A1868036800215B6EB0EEA6
:1064C000480A984707B0BDEC028B30BD95F9E13E14
:1064D000002B06DBD5F8E43E022B04D190F8A13066
:1064E0000BB90121B8E70221B6E7236A186877F0F3
:1064F00027F8236A186875F0D3FBC6E7D979002915
:10650000C5D12046FFF724FDC1E700BFD84B0020CE
:1065100000000000836893ED140AB5EEC00AF1EEA6
:1065200010FA01DCFFF796B97047000070470000D1
:1065300000207047012070470220704700207047FC
:1065400000207047012070470020704781F0010053
:1065500070470000012070470120704700487047D5
:1065600000AE0C08004870470CAE0C0838B5436903
:106570000446186878F06AFA18B96369186879F0FF
:10658000E9FB636920461D68FFF7ECFC6368B3F91B
:106590003820B3F9363000EE903A434201EE102A2B
:1065A00000EE103AB8EEC11AF8EEE00AB8EEC00AF2
:1065B000284678F037F9636920461D68FFF7D2FC5A
:1065C0006368B3F93820B3F9363000EE903A4342AD
:1065D00001EE102A00EE103A2846B8EEC11AF8EE85
:1065E000E00AB8EEC00A78F097F9012038BD000043
:1065F00030B52DED028B0446436985B01D68FFF769
:10660000B1FC6368B3F93820B3F9363000EE903A44
:10661000434201EE102A00EE103AB8EEC11AF8EE2D
:10662000E00AB8EEC00A28465B4D78F0FBF8204639
:10663000FFF762FBB5F99C3108EE103A236A18683F
:1066400003689B6E9847B8EEC88AF0EE400A02AA2B
:1066500001A9B0EE480A2046FEF706FF2046FFF7E4
:1066600015FB236B1B68B3F90830F0EE408A00EE8F
:10667000103A2046B8EEC00AFFF738FB2046B0EECD
:10668000408A8DED030AFFF76DFC6368B3F936307D
:1066900001EE103A434200EE903AB8EEC11AF8EE1D
:1066A000E00A2B20B0EE480A21F0F4FE20468DEDE2
:1066B000030AFFF7A5FA042813D8DFE800F0032F38
:1066C000252A4B00236A186875F0D4FA236A002142
:1066D000186876F07FF863699FED300A186879F0E2
:1066E00015FC236ADDED020A18689DED010A0368B6
:1066F000B0EE681ADB6A98476369186879F078FC2D
:1067000005B0BDEC028B30BD236A0121186876F01C
:1067100061F8236A186875F0C3FADCE7204D2B781E
:1067200063B963689FED1F1ADFED1C0A93ED040A3D
:10673000452021F0AFFE284608F0EEFE20469DEDF4
:10674000030AFFF741FA16488DED030A03A908F082
:106750001DFFC6E7636A022118687CF0BDFCB5F92D
:106760009C31114800EE103A02AA01A9B8EEC00A05
:1067700061F018FF20469DED030AFFF725FA0B484C
:106780008DED030A08F0DCF963699DED030A1868D2
:1067900078F0CEF8A5E700BFD84B0020000000003D
:1067A0001089002000007A4408760020A4570020B9
:1067B0000020704790F8B931002B14BF1B20032034
:1067C00070470000002070470120704790F890014A
:1067D000062804D0A0F1090358425841704701200F
:1067E00070470000012070470120704790F8B90100
:1067F000034A044B002814BF10461846704700BFD8
:10680000A4AE0C08B5DB0D0890F8B901034A044B9F
:10681000002814BF10461846704700BFB0AE0C08E1
:10682000B5DB0D0890F890010A3818BF01207047B9
:1068300090F8B9312BB9044BD3F8D80A00F0010015
:1068400070470020704700BFD84B002090F890316F
:1068500023B9034B187880F001007047002070477F
:10686000F488002038B590F89041012C054601D0FD
:10687000002038BDC368186803681B699847002862
:10688000F6D1EB681B68204683F8B848F1E70000B2
:10689000C3681B68002283F8B828012070470000F5
:1068A00070B52DED028B002380F8B931B0F870304F
:1068B000012B84B004460D4601D8002946D0636AF6
:1068C000254E1B6893F8CB3073BB2448072384F80C
:1068D00090310368022B02D10021FBF777FC9FED7A
:1068E000208AE368F0EE480A1868B0EE481AF0EE25
:1068F000481AB0EE480A01257AF064FE84ED738AE6
:1069000084ED748A84ED758A84F8B85104F59A7020
:1069100025F094FC134803F0B3FD96F8E23E6FF3C4
:10692000C30386F8E23E11E096F9E03E002BCCDA94
:1069300004F13C0027F050FD05460028C5D1204653
:10694000FFF70CFB084A02214EF00CFA284604B06F
:10695000BDEC028B70BD00BFD84B00200488002026
:106960000000000098840020B8AE0C0810B5044662
:10697000064890F85434012B03D100F58A6025F0C5
:10698000C5FC002384F8B93110BD00BFD87B0020BE
:1069900010B52DED028B094B0446D3F89C09B0EEDF
:1069A000408A7AF085F99FED060A28EE008A0120D8
:1069B00084ED748ABDEC028B10BD00BFD86B002043
:1069C0000AD7233C10B52DED028B094B0446D3F8B2
:1069D0009C09B0EE408A7AF07BF99FED060A28EE1A
:1069E000008A012084ED758ABDEC028B10BD00BFCA
:1069F000D86B00200AD7233C10B52DED028B094B34
:106A00000446D3F89C09B0EE408A7AF06FF99FED06
:106A1000060A28EE008A012084ED738ABDEC028B01
:106A200010BD00BFD86B00200AD7233CC3681B6889
:106A3000186978F04DBA000038B5D0F894310446A2
:106A40000D461BB983F0BCFFC4F8940183F0B8FF76
:106A5000D4F89431C01A4FF47A73B0FBF3F0B4F861
:106A60009231984209D32046FFF778FA2B88044ADE
:106A700006214EF077F9012038BD0020FCE700BF69
:106A8000D4AE0C0890F89031052B05D1054BD3F806
:106A9000A439D86878F094B9C36818680368DB68CB
:106AA000184700BFD86B002008B590F89031052B2F
:106AB0000BD1094BD3F8A439D868243024F044FC16
:106AC000BCEEC00A10EE100A08BDC368186803685F
:106AD0009B689847F4E700BFD86B002090F890318E
:106AE0008B4206D00A2B80F8901102D10148FCF7A6
:106AF000E9BF7047D82B002073B501231E4E80F8E4
:106B00007530D6F8EC3E834205460A4614D101247E
:106B100085F8B941D6F8EC0E019203681B689847D6
:106B2000019A014615484AF09BFA96F8E13E9A060A
:106B30001BD4204602B070BD01910321FFF7E2F89B
:106B4000019A04460028E2D185F875004BF0C0F8A0
:106B50001B220A214AF074FE96F8E13E9B06E8D516
:106B6000074A137843F0040303E0054A137843F01F
:106B700002031370DDE700BFD84B0020983B0020D4
:106B8000D489002030B585B004460D4601466846DC
:106B9000FFF7EEF9694604F13C0028F0CFF9C8B9D7
:106BA0004BF096F81B220A214AF04AFE0D4B93F84F
:106BB000E13E9B0604D50C4A137843F0040313709E
:106BC0002046FFF7CBF9094A04214EF0CBF800200C
:106BD00005B030BD2946204605B0BDE83040FFF77E
:106BE0008BBF00BFD84B0020D4890020E8AE0C0832
:106BF00030B585B004460D4601466846FFF7B8F942
:106C0000694604F13C0028F0BDF9C8B94BF060F8C2
:106C10001B220A214AF014FE0D4B93F8E13E9B061D
:106C200004D50C4A137843F0040313702046FFF791
:106C300095F9094A04214EF095F8002005B030BDC1
:106C40002946204605B0BDE83040FFF755BF00BFDC
:106C5000D84B0020D489002024AF0C087FB505460E
:106C60000E4605F13C0401466846FFF781F9694686
:106C7000204628F087F9C0B92046694628F05EF919
:106C8000044690B94BF024F81B220A214AF0D8FDA3
:106C90000D4B93F8E13E9B060FD42846FFF75EF9B3
:106CA0000A4A04214EF05EF804E031462846FFF718
:106CB00023FF0446204604B070BD054A137843F014
:106CC00004031370E9E700BFD84B00205CAF0C0849
:106CD000D489002030B5044685B00F4808F072F81A
:106CE0000546B0B1072384F8903100230193029345
:106CF0000393E36801A9186879F074FFE3681868E2
:106D0000036801A95B680022984704480021FBF74B
:106D10005DFA284605B030BDD82B0020048800203D
:106D2000F0B5424FD7F87029D7F86C392DED028BAA
:106D30001343D7F86829134387B005460C460CD196
:106D400049F07CF940F275124FF4801107B0BDECA8
:106D5000028BBDE8F04049F029B980697BF000FA68
:106D60002046B0EE408A10F0BFFB03283AD1EB6812
:106D700001A918687AF012F8064698B3DDED017A99
:106D80006368009338EE678A294BDFED2A7A93F91E
:106D9000E03E9FED290A2948002BA8BFB0EE670A04
:106DA00038EE008A009BBDEEC88A002118EE102A3A
:106DB0009342ACBF00930092FBF708FA6B69186826
:106DC00078F0C8FFDDED007A1D48B8EEE70A3146DD
:106DD00008F058FE00212846FFF780FE07B0BDEC02
:106DE000028BF0BD94E80F0002AE86E80F00D7F8E2
:106DF0006C3904936A46D7F87039059302213046FE
:106E000010F07EFB78B94AF063FF022215214AF0A8
:106E100017FDDDED037AF8EEE77A77EE887AFDEE7E
:106E2000E77ACDED007A0026AEE700BFD86B0020F0
:106E3000D84B0020000000000000C8420488002059
:106E4000F488002030B52DED028BC36887B004466E
:106E500018680D4679F096FF00284BD194F89021E0
:106E600000230093019302936AB93148039303A965
:106E70000493059308F036FE28B1039B0093049B0E
:106E80000193059B029394ED730A9FED2A8AE368B0
:106E9000DDED000A9DED011ADDED021A1868B4EE71
:106EA000C80AF1EE10FAAABFDFED237A9FED230A9C
:106EB00020EE270A7AF086FBD4ED747AF4EEC87AD5
:106EC000F1EE10FA07DBE3689FED1B0A186827EE66
:106ED000800A79F0EDFED4ED757AF4EEC87AF1EE21
:106EE00010FA07DBE3689FED140A186827EE800AA2
:106EF00079F0EEFEE368294618687AF08BFA0546C9
:106F000088B10F4B1B68022B09D0032B03D10D4B0B
:106F100093F9CD311BB10A480021FBF777F9012124
:106F20002046FFF7DBFD284607B0BDEC028B30BDE5
:106F3000F4880020000000340000C8420000000077
:106F400004880020D84B002010B52DED028BC368BB
:106F5000DFED348A1B684269D3ED0A0A9FED328A5D
:106F600093ED060AF4EEE80A0446F1EE10FA106812
:106F7000B8BFF0EE480A77F03BFAE36862691B6835
:106F80001068D3ED0A0A93ED060AF4EEE80AF1EE72
:106F900010FAB8BFF0EE480A77F0A2FA63691868F1
:106FA00077F032FC18B96369186878F06DFCE36813
:106FB00062691B68106893ED080A93ED0C1AD3ED13
:106FC000070AB0EEC00A77F02DFCE36862691B681F
:106FD000106893ED080A93ED0C1AD3ED070AB0EE92
:106FE000C00A77F099FC6369186877F02FFD18B92B
:106FF0006369186878F0AEFE00210C48FBF7E6F8EC
:107000000B4863F097F80B4AB2F8E23E23F4816331
:10701000A2F8E23EBDEC028B20460221BDE8104002
:10702000FFF75CBD0000003400007A4304880020B4
:1070300078760020D84B002010B50C4B0446D3F8CE
:10704000A40990ED0B0A90F8502000F11C0179F092
:10705000CFFA07480368022B02D00821FBF7B6F8E5
:1070600020460521BDE81040FFF738BDD86B002051
:1070700004880020F0B52DED028B4A4DDFED4A8AE1
:10708000B0EE408A8FB00446D5F8A4090E461746E4
:1070900079F024F9F0EEC87AF4EEE87AF1EE10FA1D
:1070A00007D49FED420AD5F8A40928EE000A79F02A
:1070B0007BF9D5F8A40990ED0B0AB0EEC00A0FB128
:1070C000B1EE400A79F060F90023D5F8A4090793DE
:1070D00002AA07A90893099379F082F9DFED347ABF
:1070E0009DED027AB4EEE77AF1EE10FA56DD022257
:1070F00007A90AA810F006FD71680191304610F04A
:10710000F3F9019902460AA810F0C4F9E3680AA944
:1071100018687AF07FF910B92648FDF7C7F8A0691A
:107120007BF01CF802684368D5F8A409049303A90E
:107130001C30039224F03AF805A88DED050ACDED38
:10714000060A24F001F91C4B1B68022B1BD0D5F852
:10715000A4391948D3ED0A7AF4EEE87AF1EE10FA80
:10716000B8BFD3ED047AF4EEC07AF1EE10FA4FF026
:10717000000110D5DFED117AB4EEE70AF1EE10FA56
:1071800009DDFBF743F804212046FFF7A7FC0FB009
:10719000BDEC028BF0BDFBF719F8F4E72046FFF7D2
:1071A0004BFFF4E7D86B0020000000340000C84219
:1071B00000009643D82B0020048800200000FA43EA
:1071C00008B50748D0F8D83A9B0704D50121A0F5A7
:1071D0000050F6F7E7FFBDE80840024808F0B4BAEF
:1071E000D84B0020F488002030B589B00446FEF763
:1071F00021FA30B10021204609B0BDE83040FEF749
:1072000051BA636A022118687BF066FFE368186868
:1072100003685B69984701461048FCF731FF6369D2
:10722000186878F0E5FE236A1D686369186877F0CE
:107230001DFD05AC20460A498DED020ACDED030A7D
:107240008DED041AFBF782F9079B009394E80C007C
:1072500002A9284674F0D6FD09B030BDD82B002015
:107260000488002038B50446FEF7E4F9054628B145
:1072700020460021BDE83840FEF714BA636A0221B7
:1072800018687BF029FF29462046BDE83840FEF704
:1072900053BE00000148002105F0FABBF485002030
:1072A00030B5174D9FED170A05F5804389B00446A8
:1072B000D3F8A40979F036FA01462846FCF7E0FE37
:1072C0006369186878F094FE236A1D68636918681A
:1072D00077F0CCFC05AC20460B498DED020ACDEDD4
:1072E000030A8DED041AFBF731F9079B009394E82C
:1072F0000C0002A9284674F085FD09B030BD00BF1E
:10730000D82B0020000000000488002030B589B090
:107310000446FEF78FF930B10021204609B0BDE8E0
:107320003040FEF7BFB9636A022118687BF0D4FED3
:10733000E368186803685B69984701461048FCF7E2
:107340009FFE6369186878F053FE236A1D686369BD
:10735000186877F08BFC05AC20460A498DED020ACF
:10736000CDED030A8DED041AFBF7F0F8079B0093AF
:1073700094E80C0002A9284674F044FD09B030BD21
:10738000D82B00200488002030B52DED028B83B06F
:107390000446FEF74FF920B9636A1B6893F8CC30B6
:1073A00043B90021204603B0BDEC028BBDE830405C
:1073B000FEF778B994F89831DA071DD4E3681D68B0
:1073C0002B6828469B689847D5ED097A94F8983140
:1073D000B4EEE70AF1EE10FA4CBF0122002262F38C
:1073E000000384F8983107D4204603B0BDEC028B2B
:1073F000BDE83040FFF7F8BE94F898319B0734D4CD
:10740000E368DFED458A1B686269D3ED0A0A9FEDE8
:10741000438A93ED060A1068F4EEE80AF1EE10FADA
:10742000B8BFF0EE480A76F0E3FFE36862691B68D4
:107430001068D3ED0A0A93ED060AF4EEE80AF1EEBD
:1074400010FAB8BFF0EE480A77F04AF86369186896
:1074500077F0DAF918B96369186878F015FA94F8D2
:10746000983143F0020384F898312D4BD4F8A021D1
:10747000D3F868399B1A07EE903AB8EEE78AF1EE36
:10748000047AB0EEC87AB4EEE77AF1EE10FA38D5A5
:1074900094F8983143F0040384F89831204684ED41
:1074A000678AFEF735FC6369A26B1B68D2ED001A90
:1074B00093EDC61AD3ED0E0AB1EE480A21F0CCFACC
:1074C00063691B6840F2AA4093EDC31AD3EDC40A66
:1074D00020F0E0FF2046FEF777FB12488DED010A11
:1074E00007F02EFB63699DED010A186877F020FA1A
:1074F0006369186803B0BDEC028BBDE8304078F0DA
:1075000077BDD4ED677A68EE277AF5EEC07AF1EEB2
:1075100010FAC3D5BCE700BF0000003400007A4376
:10752000D86B0020A457002030B52DED028B83B01E
:107530000446FEF77FF820B9636A1B6893F8CC30E5
:1075400043B90021204603B0BDEC028BBDE83040BA
:10755000FEF7A8B86369DFED347A1B6894ED710A11
:1075600093EDC31AD3EDC40A20EE270A40F2C440BB
:1075700020F090FF2046FEF727FB236A1868036877
:107580009B6EB0EE408A9847284BB3F99C3107EECA
:10759000903AB4F8BC316425F8EEE77A13FB05F3B2
:1075A000B4EEE70A07EE103A94F9BE31F1EE10FAA4
:1075B000D8BFF0EE407A13FB05F39FED1D0AF8EEFD
:1075C000C76A07EE103AF4EE407AB8EEC77AF1EEE9
:1075D00010FA58BFB0EE670A6846CDED006A8DED2F
:1075E000017A23F003FF236ADDED010A1868B4F87D
:1075F000C03102689DED000A126B13FB05F301EE2A
:10760000103A0121B8EEC11A90476369B0EE480AFA
:10761000186877F08DF96369186878F0E9FC03B0B1
:10762000BDEC028B30BD00BF0000C842D84B00202B
:1076300000007A4430B590F8B83185B00446F3B113
:1076400068460FF021FF404869460AF0A5F950B19D
:1076500004F13C0027F05EFC002384F8B83104F507
:107660009A7024F0EBFD94F890310A2B2DD8DFE8C6
:1076700003F0294C50544C582C5C602C640000F5ED
:107680009A7024F0DBFD04F13C0590B194F8403091
:10769000012B0ED194F89031012B0AD1284627F006
:1076A000A7FA50B12046FEF759FC284A02214DF0B6
:1076B00059FB284627F0CAFAD5E72046FEF74EFCCC
:1076C000234AF3E72046FFF77BFD94F844303BB9AB
:1076D00094F8463023B994F840309A1E53425341EF
:1076E00094F8B9216AB363BB84F8B931194CD4F862
:1076F000EC0E03681B6898472D220146A4F58250C2
:1077000005B0BDE8304049F0ABBC2046FFF76CFD4A
:10771000DBE72046FFF7A6FDD7E72046FFF7BAFDD7
:10772000D3E72046FFF7BCFDCFE72046FFF7EEFD8D
:10773000CBE72046FFF728FEC7E72046FFF7F4FE19
:10774000C3E705B030BD00BF983E0020A8AF0C08CD
:10775000D0AF0C08D84B00202DE9F0412DED028B65
:10776000074684B008460E460FF0BEFE032880464A
:107770006D4628D1FB68186879F062F9012822D19A
:107780002148294607F0BEF90446B0B17B69DDED1A
:10779000007A1B68F8EEE77A93EDF27A77EEC77A13
:1077A0004246FDEEE77A17EE901AC829CDED007A31
:1077B000B8BFC82130460FF06DFE204604B0BDECC6
:1077C000028BBDE8F081114B0FCB85E80F003046EE
:1077D0000FF08AFE014628460FF020FF04460028DD
:1077E000EBD07B69DDED017A1B68B8EEE78AD3ED5B
:1077F000F27A284638EE678A0FF076FEBDEEC88A28
:10780000024618EE101AD5E7D82B00203C75002050
:1078100010B543699FED126A1B68D3EDF06A93EDD2
:10782000F17AD3EDF27A86B066EE866A27EE067AB2
:1078300067EEC67A68460C46CDED006A8DED017A9A
:10784000CDED027A23F0D6FF03A920468DED030A81
:10785000CDED040A8DED051A10F0A8F906B010BDA3
:107860000AD7233C30B5083204461D460FCA84E8C7
:107870000F00134301BFAB68A360EB68E36063686C
:1078800085B093B920460FF02FFE03AA0146284683
:107890000FF036FE60B10399019120460FF024FEEF
:1078A0000199024620460FF0F5FD204605B030BD97
:1078B000696801912846F1E730B50B6985B0044647
:1078C0000BB94B6953B30023C4F8B43108310FC965
:1078D0006D4685E80F0029462046FFF73DFF98B921
:1078E000124B0122D3F8681928460FF0D3FD4AF055
:1078F000EFF90222152149F0A3FF2046FEF72EFBE7
:107900000B4A02214DF02EFA29462046FFF79AFA3B
:1079100010B90848FCF7CAFC05B030BD0123C0F817
:10792000B43105B0BDE83040FFF70EBBD86B002086
:1079300004B00C08D82B002070B51A4B04460E4634
:107940000FCB88B06D4685E80F0020462946FFF72B
:107950005FFFE368186879F015FA98B1E368186872
:1079600003681B69984768B1E3682946186879F08D
:107970007BF838B948F062FB40F295624FF4801111
:1079800048F014FB214604A82B463246FFF76AFF55
:1079900004A92046FFF756FA10B90348FCF786FC05
:1079A00008B070BD3C750020D82B002070B5154B79
:1079B0000C4606460FCB88B06D4685E80F00294679
:1079C0003046FFF725FF2B462246314604A8FFF735
:1079D00049FF6288A388122A4FEA132305D1227E29
:1079E000D20744BF03EB83035B00227A07EE903A91
:1079F000C2F34002B8EE670A04A93046FFF73AFB2B
:107A000008B070BD3C75002038B504460D46FFF740
:107A100093FF0023C4F89431AB88A4F8923138BDA9
:107A20007FB50D460446FFF787FF05F108010FC932
:107A30006E4686E80F00134306D1234BD3F86C291A
:107A4000D3F870390292039304F5D07201213046C5
:107A50000FF056FD94F8983170B923F0050343F008
:107A6000050384F898312046FEF778FA174A062174
:107A70004DF078F904B070BD23F0070384F8983115
:107A80000023C4F89C31E36862691B68106893EDB9
:107A9000080A93ED0C1AD3ED070AB0EEC00A76F08F
:107AA000C1FEE36862691B68106893ED080A93EDF4
:107AB0000C1AD3ED070AB0EEC00A76F02DFF0821AC
:107AC0002046FFF70BF8D5E7D86B002030B00C0844
:107AD0002DE9F0438DB06D4688461C460746134697
:107AE0000A4601462846DDE91469FFF7BBFE95E822
:107AF0000F0084E80F0007A80FF0C6FCB8F80430A8
:107B0000F3B9B8F80010013105AA89B207F13C00B9
:107B100026F01AFCA0B1234605AA39462846FFF7ED
:107B2000A1FE95E80F0086E80F00BDF81630A3F11E
:107B300052025342534189F800300DB0BDE8F08342
:107B400094E80F0086E80F000023F4E770B58B88F7
:107B500092B004460D461646002B44D10DA80FF0F6
:107B600093FC298801310BAA89B204F13C0026F06C
:107B7000EBFB002837D0BDF82E10132903D014D802
:107B80001039012913D833462A46214603A8FFF7A6
:107B900069FE03AB214607A80BAAFFF763FEE36863
:107BA00007A9186879F076FC01E0522901D012B0DB
:107BB00070BD07AD03A80FF067FC28460FF064FC0A
:107BC0000DF10B03CDE90053324603AB0BA9204660
:107BD000FFF77EFFE0689DF80B3000682A4603A996
:107BE00079F02EFCE3E70120E1E7000070B5214BBE
:107BF00004460E460FCB88B06D4685E80F00204640
:107C00002946FFF705FEE368186879F0BBF898B1DC
:107C1000E368186803681B69984768B1E3682946F8
:107C2000186878F021FF38B948F008FA40F2166277
:107C30004FF4801148F0BAF9214604A82B46324689
:107C4000FFF710FE04A92046FFF7FCF820B90A4808
:107C5000FCF72CFB08B070BD0023C4F89431B38846
:107C6000A4F8923104AA31462046FFF76FFF00289E
:107C7000F0D1ECE73C750020D82B0020F0B5324B5A
:107C800004460E460FCB91B004AD85E80F002046A8
:107C90002946FFF7BDFDE368186879F073F898B1DD
:107CA000E368186803681B69984768B1E368294668
:107CB000186878F0D9FE38B948F0C0F94FF4DF629F
:107CC0004FF4801148F072F90CAF08A80FF0DCFBFC
:107CD00038460FF0D9FB0DF10F03CDE900732A46AA
:107CE00008AB31462046FFF7F3FEE0689DF80F3001
:107CF00000683A4608A979F0E9FE20B91348FCF774
:107D0000D5FA11B0F0BD0023C4F89431B388A4F8BB
:107D1000923108AA31462046FFF718FF0028EDD01F
:107D20000B4B1B68022B09D0032B03D1094B93F992
:107D3000CD311BB106480021FAF768FA012120462F
:107D4000FEF7CCFEDDE700BF3C750020D82B0020FD
:107D500004880020D84B002037B504460D4682F039
:107D60002FFEC4F8A801D5ED027AF5EEC07AF1EE47
:107D700010FA17DD9FED137A67EE877AFCEEE77A4B
:107D8000C4ED697A2046FEF7E9F8D4F8A4214FF44F
:107D90007A73B2FBF3F30C4A062103B0BDE830401E
:107DA0004CF0E0BF5EF0EAF90023009395F90D2056
:107DB00095F90E3095F90C105EF07CF9C4F8A40129
:107DC000E0E700BF00007A4448B00C0810B5B1F9F4
:107DD0000A30A0F8BC3191F90C3080F8BE31B1F90D
:107DE0000D30A0F8C031B1F90F3007EE903AF8EE3F
:107DF000E77A0446C0ED717A82F0E2FD0A21C4F808
:107E0000C8012046BDE81040FEF768BE38B50446FC
:107E10000D4682F0D5FDC4F8B001D5ED027A9FED94
:107E2000047A67EE877AFDEEE77AC4ED6B7A38BDA7
:107E300000007A444A7C06480B46003A91F910103B
:107E4000D3ED030A93ED020A18BF0122FAF7E8B94D
:107E50000488002070B51B4E0446D6F8EC0E03686B
:107E600086B01B680D469847042806D16B88102BF6
:107E70000FD0732B20D000201CE0D6F8EC0E036846
:107E80001B6898470328F6D194F89031062BF2D15D
:107E9000ECE705F108010FC902ACDFED0B0A84E83D
:107EA0000F00002309480093B0EE600A1A462146ED
:107EB00002F028F906B070BD20462946FFF7BAFF48
:107EC0000120F7E7D84B0020000000009884002034
:107ED00038B5D1F8093007EE903AF5EEC07AF1EEF8
:107EE00010FA05460C4605DD0B7A022B03D01ED98D
:107EF000032B0ED038BD154B9FED150AD3F89C0906
:107F000027EE800A78F0D4FED4F80930C5F8D031D5
:107F1000F0E70E4B9FED0E0AD3F89C0927EE800A7E
:107F200078F0D6FED4F80930C5F8D431E2E7074B33
:107F30009FED070AD3F89C0927EE800A78F0D6FE59
:107F4000D4F80930C5F8CC31D4E700BFD86B002095
:107F50000000C84210B5044C237813B1034862F006
:107F6000E3F8207810BD00BFF48800207876002068
:107F700013B5094B01910446D3F89C0903681B69AA
:107F8000984730B10199204602B0BDE81040FEF795
:107F900053BD02B010BD00BFD86B002090F89831DF
:107FA00013F0010018BFC3F380007047094A03466D
:107FB00092F8590A68B192F8582A043A012A07D867
:107FC0005B6A1B6893F8A100431E584258417047F2
:107FD00000207047D87B002010B5044682F0F0FCEA
:107FE000D4F8B031C01AD4F8AC3123EAE373984224
:107FF0004FF0000084BFC4F8AC01012010BD0000A8
:1080000010B503680446DB6D9847D4F8AC3123EA19
:10801000E37398424FF000003CBFC4F8AC0101206C
:1080200010BD000008B504480321FAF7CFF8BDE8F9
:1080300008400148FAF7B6B90488002070B51C4B17
:108040000446D3F89C0903681B690E469847054609
:1080500010B90025284670BDD4F894315BB982F080
:10806000AFFCB4F89231C4F8940123B1114A5378AB
:1080700043F00103537082F0A3FCD4F89421B4F8C8
:108080009231801A4FF47A72B0FBF2F09842E0D34A
:1080900023B9084A537843F0010353702046FDF793
:1080A0005DFF3388044A06214CF05CFED2E700BF36
:1080B000D86B0020D4890020D4AE0C0810B590F8FD
:1080C0009031042B0446164B0AD1D3F89C0903685F
:1080D0001B69984718B12046FEF7AEFF002010BD7F
:1080E0000A79D3F8A439DFED0F6A93ED0E6A07EE33
:1080F000902A0A7E920748BF9FED0B7AF8EE677AC6
:1081000048BF67EE877A86EE267AB0EEC77AB4EE7D
:10811000E77AF1EE10FAACBF01200020DFE700BFE4
:10812000D86B0020DB0FC9400000803B13B5094B22
:1081300001910446D3F89C0903681B69984730B144
:108140000199204602B0BDE81040FEF775BC02B0B0
:1081500010BD00BFD86B002010B5044682F030FC83
:10816000D4F8A831C01AD4F8A43198424FF00000D6
:1081700084BFC4F8A401012010BD000038B5054635
:108180000C4682F01DFCD5F8C831C01A23894FF483
:108190007A725343984294BF0020012038BD0000FA
:1081A000C368186808B190F8B808704710B5012185
:1081B00004460A4803F0ECFF28B120460321BDE83D
:1081C0001040FEF78BBC47F039FFBDE8104040F28D
:1081D0006B124FF4801147F0E9BE00BFF485002018
:1081E00090F89031022B04D0032B04D1034803F004
:1081F0009FBF012070470020704700BFF48500201A
:1082000038B50C4BD3F8D85A90F89031032B04466C
:1082100005F004050AD1084803F0A2FF94F8903154
:1082200035B110B9023B5842584138BD0020F5E73E
:108230000120FAE7D84B0020F485002010B50F4A42
:10824000137843F0800313700D4B93F9E02E002A4E
:10825000044609DBFEF73EFD70B920460822BDE862
:1082600010400921FDF74EBDBDE8104001220E214E
:1082700003F64440F5F7A0BE10BD00BFD48900202E
:10828000D84B0020F8B5D0F8B44105465CB1012CBC
:108290001AD047F0D3FE40F643024FF4801147F066
:1082A00085FE012407E0184BD3F89C0903681B697D
:1082B000984710B900242046F8BD2846FEF744FE32
:1082C0000123C5F8B431F6E7104F97F9E03E002BD3
:1082D000F0DA436A1B6893F8A160012EEAD13C30C2
:1082E00026F088F804460028E5D1D7F8103F93F827
:1082F000CB3033B132460D2107F64440F5F75CFE32
:10830000D9E73446D7E700BFD86B0020D84B002010
:1083100038B5674BD3F8EC2E664B9A4204460D46AF
:1083200001D0002096E04B885D2B75D8512B2FD8BB
:10833000103B9AB20F2A49D92046FDF70FFE6B88F1
:108340005D4A04214CF00EFD7DE0BC3B0D2BF3D8C3
:1083500001A252F823F000BF4784010847840108B6
:1083600039830108398301083983010839830108F9
:1083700039830108478401083983010847840108CB
:1083800039830108398301083983010847840108CA
:10839000523B0B2BD0D801A252F823F09384010852
:1083A000398301085D84010871840108398301085B
:1083B00039830108398301083983010839830108A9
:1083C0003983010839830108998401080F2BB3D838
:1083D00001A252F823F000BF6B8401082383010837
:1083E000798401087F8401088D8401087184010863
:1083F0005D84010839830108398301083983010844
:108400003983010839830108398301083983010858
:108410003983010885840108732B46D006D8702B58
:1084200040D0722B88D1FFF7EBFD1AE04AF2CF6201
:10843000934234D080D8C92B0DD8BB2B85D8B23B02
:10844000012B3FF679AF2046FDF788FD298850F0D3
:10845000ABFD012038BDCF2BF5D06DE72046FFF7EF
:1084600079FD00283FF45DAFEDE7FFF7E7FDF8E7A2
:108470002046FFF707FFF4E7FFF720FEF1E7FFF7DD
:1084800077FDEEE7BDE83840FFF788BDFFF78EFDCA
:10849000E7E7FFF74BFEE4E7FFF75EFEE1E7FFF7F4
:1084A0006DFEDEE7FFF798FDDBE7FFF7BBFDD8E7E2
:1084B000D84B0020EC7F002058B00C0890F8903189
:1084C000032B0BD0062B06D0012B0AD1C3681868EA
:1084D00003681B681847044801F006BA034803F014
:1084E000B1BE0020704700BF98840020F4850020B2
:1084F0008B88012B05D00B693BB94B692BB9CB6835
:108500001BB904480021FAF75DBA0248002208317D
:10851000FAF77ABAD82B002010B54B885D2B0446A9
:108520000A464BD8512B05D8103B99B20F291FD9B9
:10853000002091E0523B0B2BFAD801A151F823F017
:1085400093860108318501084D860108638601087C
:10855000318501083185010831850108318501081F
:108560003185010831850108318501089B860108A4
:108570000F2BDDD801A151F823F000BF5B86010865
:108580006D860108758601087D8601088D860108C3
:10859000638601084D86010831850108318501088F
:1085A00031850108318501083185010831850108CF
:1085B000318501083185010885860108B32B76D005
:1085C00016D8732B70D00ED8702B6AD0722BAFD107
:1085D000D1ED027A9FED3A7A67EE877AFDEEE77A7F
:1085E000C0ED6B7A37E0B22BA2D1FFF771FC32E01D
:1085F000C92B23D8BB2B9BD9BC3B0D2B98D801A1F1
:1086000051F823F057860108578601083185010883
:10861000318501083185010831850108318501085E
:10862000B586010831850108B58601083185010844
:108630003185010831850108B58601084AF2CF620B
:1086400093427FF475AFFFF7C1FB04E002F108012C
:108650002046FEF765FB012010BD1146FFF7C6FA64
:10866000F9E711462046FFF727F9F4E71146FFF72F
:1086700063F9F0E71146FFF799F9ECE71146FFF7C8
:10868000C3F9E8E71146FFF7CBF9E4E7FFF78EFD02
:10869000E1E71146FFF7F2FADDE71146FFF75CFB71
:1086A000D9E7FFF7B3FBD6E7FFF7C4FBD3E7FFF744
:1086B0001FFFD0E7034802F10801F9F74FFECAE7B0
:1086C0000000C84204880020704700007047000086
:1086D0007047000090F8280080F00100704700000B
:1086E000024B436040F6050303817047000102041A
:1086F00090F85501704700000F2070470020704728
:1087000000207047002070470020704700487047E5
:1087100004B10C080048704710B10C0808B50948AE
:1087200000F50053D3F8283BB3F9083000EE103AB7
:10873000B8EEC00AF5F7E0FEBDE808400248FDF7D4
:1087400043BA00BFD82B0020C481002010B51448C4
:108750002DED028B1C4600F5005300F58040B3F967
:108760009C31D0F8900908EE103A036882B09B6EF5
:10877000CDE900219847B8EEC88AF0EE400ADDE95D
:108780000021B0EE480A0748FCF76EFE0548FDF7E9
:108790007DFA84ED000A02B0BDEC028B10BD00BF73
:1087A000D82B0020C4810020F8B51C4D05F50054DD
:1087B00005F580462846D6F89879F5F78BFEB4F98A
:1087C000D83101EE103AB4F9D63100EE903A434276
:1087D00000EE103AB8EEC11AF8EEE00AB8EEC00AA0
:1087E000384676F01FF82846D6F89869F5F772FEF5
:1087F000B4F9D83101EE103AB4F9D63100EE903A1E
:10880000434200EE103A3046B8EEC11ABDE8F840D7
:10881000F8EEE00AB8EEC00A76F07EB8D82B002059
:1088200038B5144C04F5804504F57C64D5F89009FE
:1088300003689B689847692100F19402204648F03C
:10884000DBF8D5F890090368DB6898476A2100F1E6
:108850009402204648F0D0F8D5F8900903681B69C7
:1088600098476B2100F194022046BDE8384048F05B
:10887000C3B800BFD82B0020014806F0A3BA00BF40
:10888000D82B00203C3080F0E7B9000008B547F055
:10889000D5FBBDE8084072224FF4801147F086BB3B
:1088A00008B547F0CBFBBDE8084066224FF48011C5
:1088B00047F07CBB08B547F0C1FBBDE8084080220B
:1088C0004FF4801147F072BB73B51E4E0546D6F8C3
:1088D000EC0E0268126B9047044670B396F9E13EC5
:1088E000002B2DDBD6F8103F93F8CB402CB396F835
:1088F000E03E03F0A003202B22D1D6F8EC0E026854
:1089000012689047052808D0D6F8EC0E0268126865
:108910009047A0F110035C425C410B4A02F67413CD
:108920000193D6F8403C0093D2F89839D2F89029B8
:108930002146284680F03EF90446204602B070BD2C
:108940000024FAE7D84B0020D86B00203C30FFF71A
:10895000BBBF000038B5114D04461148F6F74EFA7A
:1089600095F9E03E002B14DA236A93F8A120012A3E
:1089700006D0D5F8EC0E0021BDE83840FCF792BED9
:108980000D2105F64440F5F717FB95F9E03E002B65
:10899000EFDB2046BDE8384080F048BCD84B0020D3
:1089A000D82B00203C30FFF7D5BF000001207047D6
:1089B0000120704701207047012070471120704747
:1089C000012070470020704700207047002070474A
:1089D0000048704754B20C08004870475CB20C085D
:1089E00038B5436904461D68806979F0BDFB23F002
:1089F0003BFBDFED1B0A284675F0FAFC6369A069B2
:108A00001D6879F0B1FB23F02FFBDFED150A284636
:108A100075F066FD6369186876F036FF6369DFED0F
:108A2000110A18689FED0E1AB0EE600A75F0FAFE92
:108A30006369DFED0C0A18689FED091AB0EE600A51
:108A400075F06AFF6369186876F000F818B9636911
:108A5000186877F07FF900232364012038BD00BF38
:108A600000803B4400007A4370B52DED028B88B046
:108A70000446FCF7DFFD70B120460021FCF712FE32
:108A800063699FED310A186808B0BDEC028BBDE840
:108A9000704077F03BBA636A022118687AF01CFBD9
:108AA0002A4B93F8E13E5B0603D56369186875F0BD
:108AB0001FFD9FED258A60698DED018A8DED028A8B
:108AC0008DED038A8DED048A03AA01A900680123B4
:108AD00075F078FD6369186876F0ECFF236A1D680D
:108AE0002B68DE6C6369186876F0C0F80122CDED62
:108AF000060A8DED071A05A98DED050A2846B0EE88
:108B0000480AB0476369B0EE480A186875F010FF6C
:108B10006369186877F06CFA236C8BB181F050FFB1
:108B2000E36BC01A236C98420AD309480C22052132
:108B3000FCF7F6FE20B906480C220221FCF7F0FEF5
:108B400008B0BDEC028B70BD00000000D84B0020C7
:108B5000D82B002038B504460D4681F031FFC4E91A
:108B60000F0538BD0720704701207047002070476F
:108B7000002070470120704700487047F4B20C088D
:108B800000487047FCB20C0838B52DED028B00236D
:108B900080F83C30C368DFED338A1B684269D3ED4F
:108BA0000A0A9FED318A93ED060AF4EEE80A0446BC
:108BB000F1EE10FAB8BFF0EE480A106875F018FC34
:108BC000E36862691B681068D3ED0A0A93ED060A30
:108BD000F4EEE80AF1EE10FAB8BFF0EE480A75F0CC
:108BE0007FFC636920461D68FDF7BCF96368B3F933
:108BF0003820B3F9363000EE903A434201EE102AA5
:108C000000EE103AB8EEC11AF8EEE00AB8EEC00A6B
:108C1000284675F007FE636920461D68FDF7A2F936
:108C20006368B3F93820B3F9363000EE903A434226
:108C300001EE102A00EE103AB8EEC11AF8EEE00A82
:108C4000B8EEC00A284675F067FE084BD3F8A409B1
:108C500077F0EAFC06480821F9F7B8FABDEC028B78
:108C6000012038BD0000003400007A43D86B00209A
:108C70000488002030B52DED048BC3689FED898AF0
:108C80001B684269D3ED0A7ADFED870A93ED060A85
:108C9000F4EEC87AF1EE10FA0446A8BFF0EE670AC7
:108CA000106889B075F0A4FB636920461D68FDF764
:108CB00059F96368B3F93820B3F9363000EE903AC9
:108CC000434200EE103A01EE102A2846774DB8EEE6
:108CD000C11AF8EEE00AB8EEC00A75F0A3FDD5F8A7
:108CE000A40977F01DFEA5F5005393F8053FD907B9
:108CF00047D4D5F8A4391A8BD20742D593ED0A9AF6
:108D0000B4EEC89AF1EE10FAB8BF93ED049AE36A94
:108D1000186854F06FFAD5F89C39D3ED067AA36B36
:108D200020EE270AD3ED007AF0EE498AE0EE278A9A
:108D3000B0EE490AF5EEC08AF1EE10FAD8BFDFEDC9
:108D40005C8AF0EE680A1FF0A1FA28B9D5F8A409E8
:108D5000B0EE680A77F028FB636893F95130272B4F
:108D60000FD0A36A186854F045FAF0EEC07AF4EE1A
:108D7000C87AF1EE10FAB0EE407A20D5002384F8DC
:108D80003C30236B1B68B3F9083000EE103A2046E4
:108D9000B8EEC00AFCF7AAFF2046FCF715FF2046F4
:108DA000B0EE408AFCF746FC002848D0002120465F
:108DB00009B0BDEC048BBDE83040FCF773BCD5F8BE
:108DC000A4399FED3C0AD3ED0F7AD3ED0B6AA36B68
:108DD00027EE800AF4EEC86AD3ED007AF1EE10FABD
:108DE00067EE277A10DB9FED341ADFED310A55204C
:108DF00037EE800A1FF04EFB012384F83C30D5F893
:108E0000A40977F0C1FABCE79FED2C7AF4EEC76AAB
:108E1000F1EE10FA05D89FED261ADFED290A592048
:108E2000E6E7F0EEE66AF4EEC86AF1EE10FAE3D592
:108E300094F83C30002B08BFB0EE670ADCE7636AA9
:108E4000022118687AF048F91E4805F079FEB0EE64
:108E5000480AD5F8A40977F065FC01461A48FBF7E3
:108E60000FF96369186877F0C3F8236A1D686369AE
:108E7000186875F0FBFE05AC204614498DED020A1A
:108E8000CDED030A8DED041AF9F760FB079B009303
:108E900094E80C0002A9284672F0B4FF09B0BDECBA
:108EA000048B30BD0000003400007A43D86B0020F2
:108EB00000000000E02E65420000B442000000B453
:108EC0000000B4C2A4570020D82B00200488002042
:108ED00008B5064BD3F8A439D868243022F034FA08
:108EE000FCEEC07A17EE900A08BD00BFD86B0020D8
:108EF000024BD3F8A439D86875F062BFD86B002054
:108F00000B207047012070470020704701207047F8
:108F1000002070470048704794B30C080048704721
:108F20009CB30C080120704708B5DFED237AF4EEFE
:108F3000E70AF1EE10FA2DED028BF0EE408AB0EE6A
:108F4000608A35DDDFED1D7AF4EEE70AF1EE10FA06
:108F50002ED5F6EE007A70EEE77ADFED196A9FED16
:108F6000190ADFED190AF0EEE77A87EEA67A872074
:108F7000B7EE001A30EE470A1FF08CFADFED137AD5
:108F80009FED131ADFED130A20EE270A8A2020EE48
:108F9000280A1FF07FFA30EE080ABDEC028BDFEDE5
:108FA0000A0ABDE808408D20B7EE001A1FF072BA19
:108FB0009FED050AEFE700BFAC1C5A3ED578493F4C
:108FC0008FC2753E9A99993F00000000FAEDEBBA06
:108FD0009A99993E9A9999BE70B57E4EB6F99C3190
:108FE0002DED048B00EE903AF8EEE00A82B00446D4
:108FF00001AA6946B0EE600AFCF736FAA06979F07A
:10900000B3F8E369D0ED008AD3ED946AD3ED977A93
:1090100090ED016AA3689FED701ADFED700A27EEEC
:10902000E80A68EEA68A03F69403E6EE278A054668
:109030003B20DFED6B7AB0EEE87AB4EEE77AF1EE42
:1090400010FA58BFB0EE677ADFED667AC7EE275A9E
:10905000F7EE007A77EEE57A9DED007A67EE877A93
:1090600093ED007A67EE877A9FED5F7AA6EE260A87
:1090700087EE879A1FF00EFA3C209FED571ADFED1E
:10908000570AB0EE408AB0EE680A1FF003FA626B2E
:10909000564B1268DFED567AB2F90820D3ED006A1C
:1090A0009FED541ADFED540A07EE102AB8EEC77A86
:1090B000F0EE408A27EE277ADFED507AA6EEA77A07
:1090C0004520F4EE007AA7EE678ABAEE000A28EE91
:1090D000000A83ED007A8DED000A1FF0DBF9DDED6B
:1090E000017A9FED477A474B8DED000AF0EEE77A63
:1090F000F4EEC77AF1EE10FA51D593ED007ADFED78
:10910000427A77EE277AB2EE007AF4EEC77AF1EE81
:1091100010FA58BFF0EE477AC3ED007A67EEA87AEE
:10912000CDED017A636A186890F8CB10002939D127
:1091300079F0D2FF636A1B6893F8A110012938D037
:1091400003293FD039B9236A186873F043FB236AB7
:10915000186872F08FFD236ADDED010A18689DED35
:10916000000A0368B0EE491ADB6A9847204695ED7D
:10917000028AFCF775FB2046F0EE400AB0EE480A82
:10918000FFF7D2FE236A62681868D2ED020A03680C
:1091900001215B6E984702B0BDEC048B70BD0022CC
:1091A0001A60BFE796F9E13E002BB4BF012102210E
:1091B000BEE7236A186873F00DFB236A186872F023
:1091C0006FFDC8E7D9790029C5D12046FCF7C0FE5C
:1091D000C1E700BFD84B002000000C4400000CC4C5
:1091E0000000FA4400409C450000344254880020AE
:1091F0000AD7233D00A08C4500A08CC58FC2753FC7
:1092000000000034588800208FC2F53C0E207047C3
:1092100000207047002070470020704700207047F2
:10922000002070470048704734B40C08004870476D
:1092300034B40C0870B52DED028B436A1B6893F8AB
:10924000CB300446FBB9052384F848302046FCF7B0
:1092500007FB636A02211868B0EE408A79F03CFF90
:1092600094F95030E2696BB3D2F8F8515D4394F849
:109270004820052A4FD8DFE812F02B005F00840059
:10928000B100DF001E01836A1B68B3F90830002BB0
:10929000B8BF5B429BB2B3F57A6FD4D2C36A1B6886
:1092A000B3F90830002BB8BF5B429BB2B3F57A6FBD
:1092B000C9D281F085FBE36CC01A40F6C413984212
:1092C000C1D8C3E794F95150D2F8FC215543CEE7F9
:1092D000226A94F9511010689FED801A49F64042B5
:1092E0005343514300EE103A00EE901A0268F8EE34
:1092F000E00A926BB8EEC00A9047DFED797A41F24E
:1093000093139D4238EE278A05DD94F950308BB1D6
:10931000012384F84830236A62681868D2ED020A93
:109320000368B0EE480ABDEC028B5B6EBDE870408E
:10933000002118470223ECE7226A9FED681A1068A3
:1093400049F64042534300EE103A0268B8EEC00AB4
:10935000926BF0EE410A9047DFED627A38EE678A51
:1093600005F50C55B5EEC08AF1EE10FA05F12705AA
:1093700043F2BA43D8BF9FED598A9D42CBD804230C
:10938000C7E7236A9FED551A186894F9513049F6DA
:109390004042534300EE903A0268F8EEE00A926BC6
:1093A000B0EE410A9047DFED4F7AE36938EE678A05
:1093B000D3F8F831B5EEC08AF1EE10FAD8BF9FEDC0
:1093C000478A002BB8BF5B4242F228329342A2DDAB
:1093D00041F294139D429EDD03239AE7236A9FED99
:1093E0003F1A186894F9513049F64042534300EE51
:1093F000903A0268F8EEE00A926BB0EE410A9047AC
:10940000DFED387AE36938EE678AD3F8F831B5EEE4
:10941000C08A03F50C53F1EE10FA03F1270344F26E
:109420004E62D8BF9FED2D8A93423FF674AF2E4B0C
:109430009D42FFF670AFA2E7236A94ED111A1868F7
:10944000D4ED100A036894ED0F0A1B6B00219847B6
:10945000DFED237A94F95020E36938EE278A1AB3B6
:1094600093ED7E7AD4ED0F7AB8EEC77A77EEC77AAD
:109470009FED1E7AF0EEE77AF4EEC77AF1EE10FA7D
:109480003FF649AF0D2294F849101948FCF748FA05
:10949000024618B901461648FCF742FA48F018FC93
:1094A000162148F0ADF936E793ED7F7AD4ED107AC6
:1094B000B8EEC77ADAE70D2294F849100C48FCF7A9
:1094C0002FFA024618B901460948FCF729FA48F074
:1094D000FFFB02220D2148F0B3F91CE70000000059
:1094E000CDCC4C3E8FC2753E6DEEFFFF0000FA43BF
:1094F000D82B0020F7B5474D0446D5F8EC0E03688D
:109500005B6B984718B90026304603B0F0BD95F95B
:10951000E13E002B5EDBA36A1B68B3F90830002B29
:10952000B8BF5B429BB2B3F57A6FECD2636A1B683B
:1095300093F8CB60002EE6D095F9E03E002BE2DBFD
:10954000D5F8EC0E03681B689847002784F849009B
:1095500084F8487081F034FAE36AE064A4F850704B
:109560001B68B3F90830B3F5967F42DD012384F818
:10957000513048F0ADFB152148F042F9B5F99C3166
:1095800001EE103AE369B8EEC11A93ED7E0A8DED53
:10959000011AF1EE410A5320B8EEC00ACDED000ADF
:1095A0001EF078FFE36984ED0F0A93ED7F0A9DEDCD
:1095B000011ADDED000AB8EEC00A54201EF06AFF61
:1095C000E36984ED100AD3ED807AF8EEE77AC4ED12
:1095D000117A99E7D5F8EC0E03681B6898470128C3
:1095E00091D0D5F8EC0E03681B689847002892D1FB
:1095F00089E713F5967F01DAFF23B8E7A36A1B68B2
:10960000B3F90830002BACBF0123FF2384F850309E
:10961000AFE700BFD84B00200420704701207047FF
:10962000002070470120704700487047CCB40C08F8
:1096300000487047D4B40C08012909D0232907D069
:10964000042905D0034BD3F8DC0A00F00100704771
:1096500001207047D84B0020C36B23B990F841001C
:1096600080F001007047002070470000034BD3F8E2
:10967000DC0A80F00400C0F380007047D84B002063
:10968000012380F84230184670470000002380F81C
:10969000423001207047000070B52DED028BC36889
:1096A0000446186890F9BB3886B0B0EE408A0BB318
:1096B00090F8BC68F6B177F0C3F901281AD12748B1
:1096C00019213EF0B7FE07EE900AF8EEE77AF4EEC5
:1096D000C87AF1EE10FA0DDD214BB3F93E3B07EEEF
:1096E000903AF8EEE77AF4EEC87AF1EE10FA18DB69
:1096F000002012E01B4B0FCBFDEEC87A02AD85E8CF
:109700000F0017EE901A012228460DF0C3FE01AAA1
:10971000022128460DF0F4FEE8B906B0BDEC028B3C
:1097200070BDBDEEC88A8DED018A002529460E4820
:10973000E563F8F74BFD6369186876F00BFBDDED28
:10974000017A0A48B8EEE70A314606F09BF984F838
:1097500041500120E1E70026E7E700BFE83800209C
:10976000D84B00203C75002004880020F48800209D
:1097700010B52DED048BC2689FED149A12684369F1
:10978000D2ED0A0ADFED128AF4EEC90AF1EE10FA00
:109790000446B8BFF0EE680A1868B0EE408A74F06C
:1097A00027FEE268636912681868D2ED0A0AF4EECF
:1097B000C90AF1EE10FAB8BFF0EE680AB0EE480A36
:1097C00074F08EFEBDEC048B012010BD000000344F
:1097D00000007A4313B5C36842691B68F0EE400A83
:1097E00093ED080A93ED0C1ACDED010A0446B0EE94
:1097F000C00A106875F016F8E36862691B681068A3
:1098000093ED080A93ED0C1ADDED010AB0EEC00AE3
:1098100075F082F8012002B010BD000010B52DEDEA
:10982000028BC36842691B68044693ED0C1AD3EDA2
:10983000070A1068B0EE408A74F0F4FFE3686269CA
:109840001B68106893ED0C1AD3ED070AB0EE480AB6
:1098500075F062F8BDEC028B012010BD1FB5C36B23
:10986000022B0BD0032B1DD0012B22D1C36818680B
:109870000368DB6805B05DF804EB1847806978F091
:109880006DFC0D4B59689A6802911B68019301A900
:1098900003921FF013FEFDEEC07A17EE900A05B09A
:1098A0005DF804FB4369186805B05DF804EB75F0DA
:1098B00087BA0020F3E700BF90880020C36B012B1C
:1098C0000AD003DC2BB19FED070A7047023B032B44
:1098D000F9D84369186802E0C3681B68186975F015
:1098E000F7BA00BF0000000030B5C26B012A89B092
:1098F0000C4604D0022A0AD0002009B030BDC3684B
:10990000186803681B6809B0BDE8304018470B4B66
:10991000586899681B680193094B02901B78039162
:10992000002B04AD18BF032201A928460EF0EAF867
:1099300095E80F0084E80F000120DEE79088002002
:10994000D48800207FB5C36B022B0FD0032B23D00C
:10995000012B25D1C368186803689B689847BCEE43
:10996000C00A10EE100A07B05DF804FB806978F0B9
:10997000F5FB0D4B014658689A6804901B680393E9
:1099800003A8059221F012FC01A88DED010ACDED8E
:10999000020A21F0D9FCE2E7436918682430F8E7AD
:1099A0009FED020ADDE700BF908800200000000064
:1099B00010B52DED028B01239FED1C8AC363C36894
:1099C000044684B018688DED018AF0EE480AB0EEC6
:1099D000481AF0EE481AB0EE480A8DED028A8DED75
:1099E000038A77F0EFFDE3688DED018A8DED028A41
:1099F0008DED038A186801A977F0F4F8E368186818
:109A0000036800225B6801A9984730B946F016FB4D
:109A1000BB224FF4801146F0C9FA05480021F8F73F
:109A2000F5FB04B0BDEC028B10BD00BF00000000D0
:109A30000488002030B589B00446FBF7FBFD70B107
:109A40001D4805F015FD014618B1636A1B6893F8BF
:109A5000CC10204609B0BDE83040FBF723BE636A56
:109A60000221186879F038FBE368186803685B69BD
:109A7000984701461048FAF703FB6369186876F0C7
:109A8000B7FA236A1D686369186875F0EFF805ACCA
:109A900020460A498DED020ACDED030A8DED041A28
:109AA000F8F754FD079B009394E80C0002A92846A0
:109AB00072F0A8F909B030BDD82B0020048800202E
:109AC00010B52DED028BC368DFED298A1B68426952
:109AD000D3ED0A0A9FED278A93ED060AF4EEE80A11
:109AE0000446F1EE10FAB8BFF0EE480A106874F0C0
:109AF0007FFCE36862691B681068D3ED0A0A93ED86
:109B0000060AF4EEE80AF1EE10FAB8BFF0EE480AE1
:109B100074F0E6FCE36862691B68106893ED080A5C
:109B200093ED0C1AD3ED070AB0EEC00A74F07AFE7A
:109B3000E36862691B68106893ED080A93ED0C1ADC
:109B4000D3ED070AB0EEC00A74F0E6FE6369186848
:109B500076F000F96369186875F096FE06480021F2
:109B6000F8F754FB054B00221A70BDEC028B10BDB8
:109B70000000003400007A4304880020D4880020CC
:109B80000223C363FFF79CBF0523C363FFF798BF9E
:109B90000423C363FFF794BF10B50446FFF7F8FF33
:109BA000074A0023936053601360064A9360536032
:109BB0001360002384F8403084F84230012010BD47
:109BC0009C880020A88800200323C363FFF778BF88
:109BD00030B50623C363C36842691B6893ED080A66
:109BE00093ED0C1AD3ED070A044685B01068B0EE69
:109BF000C00A74F017FEE36862691B68106893ED91
:109C0000080A93ED0C1AD3ED070AB0EEC00A74F0FF
:109C100083FE6369186874F019FF18B963691868DE
:109C200076F098F880F0CCFE0C4D0346284601A94A
:109C300040F8043B236A1B6800245B6F0393019484
:109C4000029420F0F9FE0023EC61AC616C616C625F
:109C50002C6285F82C3005B030BD00BF6088002034
:109C6000024BD3F8DC0AC0F3C0007047D84B002089
:109C70002DE9F0432DED028B9946C36B274C062B43
:109C800085B080460E461746B0EE408A36D0FFF7C4
:109C90009FFF96E80F00224D85E80F0097E8070028
:109CA000103585E8070084F82D900023B9F1000FE6
:109CB00030D084ED0A8A636280F082FE03AB2060BC
:109CC00002AA01A9304620F0E9FF94ED092ADFED50
:109CD000157AD4ED0A1A9DED031ADDED020A9DED09
:109CE000010AD8F83C10104822EE272A3A46F7F726
:109CF00013FA05B0BDEC028BBDE8F083B9F1000F9B
:109D0000C7D194F82D30002BC3D04369186876F082
:109D100021F8BEE7A36284ED098ACDE760880020C0
:109D2000648800200AD7233CD82B002038B50B4D7F
:109D30000446284605F008FD2B786BB194F84130B5
:109D400053B90123064884F841305CF093FBBDE829
:109D50003840044860F0E8B938BD00BFF4880020FE
:109D6000784C00207876002070B52DED028B88B0FD
:109D70000446FBF75FFC054680B1294805F078FBF7
:109D8000014618B1636A1B6893F8CC10204608B0EE
:109D9000BDEC028BBDE87040FBF784BC636A9FEDAD
:109DA000218A1868022179F097F960698DED018A9E
:109DB0008DED028A8DED038A8DED048A2B4603AA70
:109DC00001A9006874F0FEFB63698DED008A1868D4
:109DD0000368B0EE480A2A4669465B68984763699B
:109DE000186875F067FE6369186876F001F9236AF0
:109DF0001D682B68DE6C6369186874F037FF0122F8
:109E00008DED050ACDED060A8DED071AB0EE480A74
:109E100005A92846B04708B0BDEC028B70BD00BF55
:109E2000D82B002000000000A1B1DFED0F7A20EE5A
:109E3000270A33B1DFED0D0A0D4801220021F8F7A2
:109E4000EFB922B160EEA70A0948F8F767BADFED6B
:109E5000070AF9E722B10648B0EE600AF8F79ABAA5
:109E60000348F8F7D3B900BF0AD7233C000000002D
:109E7000048800202DE9F0432DED028B8BB00446C1
:109E8000164606A802220F461D46B0EE408AF0EEA6
:109E9000608A0DF037FE284806A95CF0ADFC8046CC
:109EA00058B947F015FF0522162147F0C9FC404676
:109EB0000BB0BDEC028BBDE8F083E36B032B02D04B
:109EC0002046FFF781FE9DF858309DF854209DF8FC
:109ED0005010F0EE680AB0EE480A2046FFF7A4FFE3
:109EE00080F06EFD154BD7F800901860144BD7F832
:109EF00004E0D7F808C0134AC3F80090C3F804E0A0
:109F0000C3F808C00023137096E807000E4F0F4EE9
:109F1000CDF80C9087E8070095E8070086E8070071
:109F2000CDE90076E16B0A48CDF810E003AACDF840
:109F300014C0F7F7AFF8BAE7784C00205C8800202F
:109F400090880020D48800209C880020A8880020C9
:109F5000D82B002010B588B00024059406940794EF
:109F60009DF82C4002949DF82840CDE9003405ABC3
:109F7000FFF780FF08B010BD2DE9F04F2DED028BEB
:109F80008FB091469DF86C709DF868B0002F14BF9B
:109F90000322022204460AA80D46B0EE408A9A46E1
:109FA000F0EE608A0DF0AEFD4D480AA95CF024FC8D
:109FB000064658B947F08CFE0522162147F040FCB2
:109FC00030460FB0BDEC028BBDE8F08F454AE36B25
:109FD000D2F8DC2A12F0400F0DF11C082AD0012B18
:109FE00002D02046FFF7E4FC5B46F0EE680A5246DA
:109FF000B0EE480A49462046FFF716FFE3681868A6
:10A0000003683A465B682946984700230493059302
:10A01000069307930893099304AB0093CDF804804B
:10A020003B462A46E16B3048F7F734F8012384F8C1
:10A030004030C5E7022B02D02046FFF7A1FD002FDC
:10A0400049D0E3684146186876F0A8FE40B9226816
:10A0500003905268012120469047039B1E46AFE7BC
:10A06000224B1B782BB963699DED070A186874F0C1
:10A07000A1FD52464946DFF874A0DFF884905B46A4
:10A08000F0EE680AB0EE480A2046FFF7CDFE2968D8
:10A090006A68AB68164D8AF80070164F29606A60CE
:10A0A000AB600023BB607B603B60C9F80830C9F837
:10A0B0000430C9F8003080F083FC0F4B6A682968CF
:10A0C0001860AB680892CDE90079099307919AF876
:10A0D00000304246A6E763699FED080AC6E700BF65
:10A0E000784C0020D84B0020D82B0020D4880020AA
:10A0F000908800209C8800205C88002000000000E0
:10A10000A88800202DE9F0472DED028B8EB0044683
:10A110006F489DF860A00E469046B0EE408A994682
:10A12000F0EE608A5CF068FB054658B947F0D0FD58
:10A130000522162147F084FB28460EB0BDEC028BA9
:10A14000BDE8F087634BD3F8DC3A590648D5E36B9A
:10A15000012B02D02046FFF72BFCE368314618683C
:10A1600077F058F9054618B947F0B2FD0222E0E74A
:10A1700053464A46F0EE680AB0EE480A4146204689
:10A18000FFF752FED6ED027AE16B0391F8EEE76A33
:10A19000D6ED037ACDED056AB8EEE77AD6ED017A11
:10A1A0008DED067AF8EEE77A3046CDED077A0DF0C0
:10A1B0009BF900220BAB089209920A920B920C9227
:10A1C0000D920193C21E08AB009303995342534171
:10A1D00005AA4148F6F75EFF012384F84030ABE75B
:10A1E0000027E068089709970A97006805AB08AA56
:10A1F000314677F0CFF8054600289DD0E36B022B5F
:10A2000002D02046FFF7BCFC5346F0EE680A4A46EF
:10A21000B0EE480A41462046FFF706FE9DF814308E
:10A22000002B50D0E3680BA9186876F0B7FD804684
:10A2300030B9236801215B682046984745467BE793
:10A24000264B1B782BB963699DED0B0A186874F0D7
:10A25000B1FC234B089A1A60099ADFF89080DFF866
:10A2600090905A60DFF874A00A9A9A609DF81430B2
:10A270008AF80030C8F80870C8F80470C8F8007090
:10A28000C9F80870C9F80470C9F8007080F098FB2C
:10A29000D6ED027A134BE16B1860F8EEE76AD6ED63
:10A2A000037ACDED0B6AB8EEE77AD6ED017A8DED43
:10A2B0000C7ACDE90089F8EEE77A9AF80030CDED16
:10A2C0000D7A0BAA85E763699FED070ABEE700BF19
:10A2D000784C0020D84B0020D82B0020D4880020B8
:10A2E000908800205C880020000000009C880020EE
:10A2F000A88800202DE9F0470E4611461A46C36B88
:10A300008AB0052B9DF84C9005460DD0CDED050A81
:10A3100004928DED030A0291FFF736FCDDED050A8C
:10A32000049A9DED030A0299184C194F9DF8483084
:10A33000DFF868A0DFF868802846FFF775FD002386
:10A340000022A36063602360BB607B603B608AF88F
:10A35000002096E8070088E8070080F031FB0D4BED
:10A360001860B9F1000F0ED06268A36821680791E8
:10A3700008920993CDE900789AF80030E96B064815
:10A3800007AAF6F787FE0AB0BDE8F087908800209C
:10A390009C8800205C880020D82B0020D4880020D6
:10A3A000A88800202DE9F0470F461946C36B8AB0F4
:10A3B000042B9DF85090054616460BD0CDED050AAE
:10A3C0008DED040A0391FFF7E3FBDDED050A9DED3A
:10A3D000040A03991A4C9DF84C309DF84820DFF888
:10A3E00070A0DFF870802846FFF71EFD0023A360F1
:10A3F0006360236000238AF8003097E8070088E84C
